:020000040000FA
:1000000000A002024D8B0000452F0000A94F000008
:1000100000000000000000000000000000000000E0
:1000200000000000009C0100489C0100452F0000DA
:100030000000000000000000452F0000E9A10000C2
:10004000FD2B0000452F0000452F00006D8B0000A8
:1000500019610000BD840000D52E0000C92F0000EA
:10006000ED0E0000290E0000452F0000492F000072
:10007000ED60000035B90000ED8A0000198B00002A
:10008000452F0000452F0000452F000075AD0000F2
:1000900095AD0000452F0000452F0000452F0000C2
:1000A000B9AD0000C3AD0000B12C00003D890000D7
:1000B000452F000025850000000000000000000022
:1000C0000348854600F00CFE00480047C5FD0000CF
:1000D00000A0020230B50B46014600202022012478
:1000E00009E00D46D5409D4205D31D469540491B6C
:1000F0002546954040191546521E002DF1DC30BDB5
:1001000070B500242546002801DA01244042002968
:1001100001DA01254942FFF7DDFFAC4200D0404241
:10012000002C00D0494270BD03460B439B0703D00F
:1001300009E008C9121F08C0042AFAD203E00B78AC
:100140000370401C491C521EF9D27047D2B201E024
:100150000270401C491EFBD270470022F6E710B522
:1001600013460A4604461946FFF7F0FF204610BD25
:1001700030B505462A460B4610781C78521C5B1C8D
:10018000002801D0A042F7D0002C03D0002802D0D4
:100190006D1CEFE7284630BDCAB2401E4178401CB6
:1001A0008A4202D00029F9D100207047421C017810
:1001B000401C0029FBD1801A704710B5002200E0D6
:1001C000521C835C8C5CA34201D1002BF8D1D8B2C5
:1001D000E1B2401A10BD30B504460020034600E0ED
:1001E0005B1C934203D2E05CCD5C401BF8D030BD79
:1001F00003460A780270401C491C002AF9D11846AF
:10020000704730B505460020034600E05B1C934272
:1002100005D2EC5CC85C201A01D1002CF6D130BDAF
:1002200070B5064614F04AFF046805460A2200210C
:10023000304600F0E1FB2C6070BDF8B502464A4044
:10024000D40F42004B0052085B089A4202D2024689
:10025000084611464A0023D0C30D4A00DDB2120EF3
:10026000AD1A202D35DA49020126490AF6058A1908
:10027000002C00D0524220214F1B1146B9402A4188
:100280001018C20D9A4221D0002C17D0012D08DC85
:10029000DA05801AD20F8019D207DBB200F0ECFB2E
:1002A000F8BDDA05801A012340001B06C01880182B
:1002B0005A428018CA0F1043490007E04908C20794
:1002C0001143DA05801A80194008801800F0CCFB31
:1002D000F8BD61000122511A001BF7E70122D20785
:1002E0005140AAE70122D2075040A6E7024670B566
:1002F0004A40D30FDB0740002DD04A002AD0010E20
:10030000140E000212020919400A520A8418E5016B
:1003100004465443000A120A2E045043A4194219F9
:10032000200CC543AA18120C0125AD03521C52190A
:1003300012047F39240400D0521C104301D4400021
:10034000491EC2B20C06C0092018401C4008802A71
:1003500002D003E0002070BD40084000002900DA10
:100360000020184370BD70B502464A40D50F4000CA
:100370004A00ED0740085208002814D0002A12D085
:10038000C40DD30D41020120C0055202490A520A90
:10039000E41A091812187D34914201D3641C00E05C
:1003A0004900002C01DA002070BD0023914201D3E6
:1003B000891A0343400849000028F7D100290AD0D0
:1003C000914202D10121C90705E0914201D20121E8
:1003D00001E00121C943E005C018401900F044FBC9
:1003E00070BD0000F0B507460846584087B0C00F02
:1003F000049048000E46590040084908BC1A88413C
:1004000005D2384631461E4617460B46024658006E
:10041000400810434CD0300D039040055900400D6A
:10042000490D0590401A0290402872DA1803012104
:10043000000B09050843019004980092002805D09C
:100440000199524200208841009201900298402177
:100450000A1A0199009800F09BFA05460C466B4673
:1004600007CB00F0B6FAC0197141039A0E0D0023B4
:10047000D71756401A467A40164344D0049A002AA9
:100480002DD0029A012A039A15DC1205C01A914157
:1004900001263605001C7141D20F059ED20700933C
:1004A000019202962A46234600F02CFB07B0F0BDCD
:1004B00038463146FAE71605224A0F46B218C01AE6
:1004C000B74101210905001C4F4100187F41114629
:1004D00018187941E20F10436D19644113E0E207E7
:1004E0006D0815436408C2071443039A01261205D8
:1004F000C01A91413605001C7141CE0740083043B7
:100500004908C01851412A46234600F0EEFACDE7CB
:10051000FFE7049801224000C117121A00238B4103
:1005200004983146C417381AA141EEE730B40124CB
:10053000E407634030BC55E730B40124E407614070
:1005400030BC4FE70000E0FFF0B51FB488B00B9956
:100550000998002448400999C00F490049080991A9
:10056000C0070B990090490049080B910999089818
:10057000A64608431CD00B990A98084318D009983E
:1005800001244000420D4800410D09982405000354
:10059000000B204309900B980003000B20430B90A5
:1005A00050181C494018002201901446104605E0DE
:1005B000002001460DB0F0BD032801DA034600E03B
:1005C00003239C46C11A0AAE0AE05F0008ADED5B4A
:1005D0004F00F75B7D430027AA187C41491C5B1E36
:1005E0006145F2DD410004AB5A522104120C0A436A
:1005F000240C401C0828DFDB01980290009970460B
:1006000001910090059B049A0799069800F07AFAE8
:10061000D0E700000DFCFFFFF0B50C465C4085B054
:10062000E40FE40703944C00002664085900944644
:10063000490802460296224321D062460A431ED050
:100640006200570D4A000E032303550D0124024694
:100650002C492405781B1B0B360B401823432643DB
:10066000614600901C46501AB44103D30098401CC8
:10067000009002E0921800985B41002803DA002005
:10068000014605B0F0BD0020012109050746864658
:1006900011E064461D46141BB54106D36546521B46
:1006A000B341744607430C43A646CD0740084908AA
:1006B000284392185B4105460D43EAD11046184382
:1006C00013D06046194650407140084306D060463A
:1006D000101AB34106D20122002306E000220123B2
:1006E000DB0702E00122D243531000987446010553
:1006F000381C6141029C039D0019694100F0F5F925
:10070000BFE70000FD0300000122D207002800DB44
:10071000101A002900DB511A814201D801207047CC
:10072000002070470122D207002800DB101A0029A0
:1007300000DB511A814201D201207047002070472E
:100740000122D207002800DB101A002900DB511A11
:10075000814201D301207047002070470122D20757
:10076000002800DB101A002900DB511A814201D950
:1007700001207047002070470122D207002800DBCB
:10078000101A002900DB511A814201D10120704763
:100790000020704710B5002904DB0C460121C90771
:1007A0004042A141002B04DB1C460123DB075242DF
:1007B000A34142404B401A4301D0002010BD01200C
:1007C00010BDC217C10F504010B54018CA0796237C
:1007D000002100F051F910BD10B5002296231146FA
:1007E00000F04AF910BD00000EB5C217C10F50400D
:1007F000CA0740180021054B0293019200910A4656
:100800000B4600F07FF903B000BD00003304000088
:100810000EB505490291002100910A460B4601914F
:1008200000F070F903B000BD33040000C20F4100B6
:1008300040020123400ADB05D207090EC0187F29B8
:1008400001DA00207047962903DC9623591AC84024
:1008500001E096398840002AF4D0404270474100B8
:1008600040020122400AD205090E80187F2901DAD0
:1008700000207047962903DC9622511AC840704721
:10088000963988407047000070B5CD0F4A000903C3
:100890000123090B1B0519430B4BED070024520DD7
:1008A0009A4201DA002070BD074B34339A4203DCD0
:1008B0009A1A00F07DF802E00449511888402C4350
:1008C000F1D0404270BD0000FF030000CDFBFFFFF0
:1008D000C20FD207400040080BD0C10D0723DB0137
:1008E000C91840020905400A1143C20840071143D4
:1008F0007047002001467047CB0FDB07490010B559
:10090000490802460A4307D00A0D07240903E401F7
:10091000090B121B002A01DC002010BDC900440F86
:100920000C43C100E018D205801800F09DF810BDFE
:10093000F0B51FB40646002082B005464024019160
:1009400000901BE0019922460F46304600F030F837
:10095000049A059B801A994110D3104619462246E5
:1009600000F016F8361A8F41019722460120002127
:10097000009F00F00DF838184D4100902046641E8D
:100980000028DFDC019B00982946324607B0F0BD05
:1009900010B5202A04DB0146203A9140002010BD0A
:1009A000914020239C1A0346E3401943904010BD18
:1009B00010B5202A04DB0846203AD040002110BDA3
:1009C0000B46D340D0402024A21A91400843194638
:1009D00010BD10B5202A06DBCB170846203A10417F
:1009E000C1170B4306E00B461341D0402024A21A46
:1009F00091400843194610BDF7B5009C0F460026EC
:100A00002578641C002D05D000F07CF90068405D5D
:100A1000C007F5D12B2D02D02D2D18D0641E3946DC
:100A20002046029A00F072F9002F04D03968A142E2
:100A300001D1009939607105022400290BDA404286
:100A4000002803DD14F03AFB0460A007FEBD01207E
:100A500080020643E3E70028F8DA14F02FFB046075
:100A60000048FEBDFFFFFF7F002904DA401C49005B
:100A700001D140084000704770B40024050C05D136
:100A80001024000402D1002921D01124050E01D127
:100A900000020834050F01D10001241D850F01D18A
:100AA0008000A41C002801DB4000641C002908D041
:100AB00020252E1B0D46F540A14000D001212943E1
:100AC000084301061B1B000ADB1D02D5002070BC79
:100AD0007047DB05181880180029F8DA401C490017
:100AE000F5D170BC40084000704710B5002B08DA03
:100AF0000024401C614192185B411A4301D1400817
:100B0000400010BDF0B51FB482B005460C0003D004
:100B1000084614F0A5FA02E014F0A2FA20300246CA
:100B2000009021462846FFF733FF049B059A0446B0
:100B30000F4618431143084314D0184610431BD0E6
:100B4000009840210A1A18460599FFF731FF05461B
:100B50000E46009A05990498FFF71AFF084305D03E
:100B6000012004E02046394607B0F0BD0020C1173F
:100B700005430E432C43374300990E986305401AF2
:100B80007905E40A00220C43FD0A0A3002D5002050
:100B90000146E9E70105101969410C9C0D9D0019FA
:100BA0006941FFF7A2FFDFE770B54B005B08034325
:100BB0000BD04B005C0D002633466542B341D41781
:100BC000AD1AA34102DB0020014670BD12053018AA
:100BD000514170BDFEB500231A461B1A8A4103DB42
:100BE0000020014603B0F0BD4A000D0301212D0B8A
:100BF0000905520D0D43D10702D100186D41521E57
:100C00005110FF31FF310131002704463E4638467E
:100C1000009701910246012100200905FFF7C8FE57
:100C2000C3197141F818324684468E464A416146DE
:100C30002846611A904104D36046241A95417646AD
:100C40001F46241900986D41401C00903428E1DDB6
:100C5000F91930467041091BA84103D20022D24342
:100C6000134601E00022134601980105381C71412A
:100C7000FFF73BFFB6E700004A0009030123090B19
:100C80001B0519430A4B10B5520D9A4202DA002097
:100C9000014610BD064B34339A4203DC9A1AFFF723
:100CA00087FE10BD034BD218FFF772FE10BD000087
:100CB000FF030000CDFBFFFF10B5002904DB01247A
:100CC000E40740428C412146002B04DB1C460123F3
:100CD000DB075242A341994200D1904210BD00006F
:100CE000064C0125064E05E0E36807CC2B430C3C7F
:100CF00098471034B442F7D3FFF7E6F99893010010
:100D0000B89301000048704714660100F7B582B03F
:100D1000029C00272078641C15460197302802D0D9
:100D2000002D15D015E020780127641C782804D008
:100D3000582802D0002D09D00BE0002D01D0102D35
:100D400007D1002710252078641C02E0082500E068
:100D50000A250026009610E000990127694308182B
:100D6000020C294680B2714300908E1838048642E6
:100D700001D3012001902078641C294600F019F865
:100D80000028E9DA0398002805D0002F01D0641E5E
:100D900000E0029C04600198002806D014F08EF94F
:100DA00002210160C81E05B0F0BD0099300408435F
:100DB000F9E73A2800D23038202302469A43412AE4
:100DC00001D310463738884201D30020C043704712
:100DD00070B58C180578401C6B075B0F01D1037848
:100DE000401C2A1106D10278401C03E006780E70E0
:100DF000401C491C5B1EF9D12B0705D40023521E51
:100E00000DD40B70491CFAE70378401CCB1A921CD6
:100E100003E01D780D70491C5B1C521EF9D5A142E0
:100E2000D8D3002070BD000010B52148016A8A07A0
:100E300015D44A0715D4C90732D01E498A89002A19
:100E400015D0531E8B8182688C6904C48C610A6939
:100E50001B040DD0002A22D10121016010BD022106
:100E600000E00421C16113488021416110BD0A697D
:100E7000012A09D1026801239A430260C361FF205D
:100E8000683099300C4A106001204861CA69002A14
:100E900005D0886909898B00C01A904710BD10BD24
:100EA000FF226832054806A109A311F06DFDC04676
:100EB00008D0014048A8010280E200E06477010008
:100EC0004144435F49525148616E646C6572000051
:100ED000556E65787065637465642041444320698C
:100EE0006E746572727570740D0A000070B582B010
:100EF00000230193444801688A6A4C681325254001
:100F0000132D02D1CB689B07DB0F4361930772D48B
:100F100053070AD4D30711D1130724D5048F838E26
:100F20001C1B102C0EDD102310E004208862022010
:100F3000032142A212F084FD02B070BD012088623C
:100F400002B070BD048F1B1B1C0610D0DBB2002446
:100F5000058FC66A75192D5D0D74641CA342F7D107
:100F6000048FE3180387D20607D400212FE04B6AD1
:100F70000824A3434B62D206F7D5CB68C28E448FB8
:100F8000141B5B04DB0EA34201D3438FD31ADAB2E6
:100F9000002A16D0097D438F046BE1540199012A80
:100FA00010D001231C46890145582D7D41184E8FD4
:100FB0009B19096BCD54641CE3B201999A42F2D893
:100FC00000E000218B01C3185C8FA2185A878A01A8
:100FD00081184B8FCC8EA3420BD301230B61805819
:100FE00000224262CA6B002A03D03A31098801A864
:100FF000904702B070BD02208862044804A1084AEC
:1010000008A311F0C1FCC04694A001027D77010045
:101010004145535F49525148616E646C65720000EE
:10102000CE02000041455320696E707574206F76C2
:101030006572666C6F770D0A000000004145532011
:101040006F757470757420756E646572666C6F77F9
:101050000D0A0000F0B581B001243F2900D993E0CA
:1010600003468068456B2D688E0001A7BE59B746C0
:10107000AF110000CB110000A7110000A711000064
:1010800089110000891100008911000089110000F8
:1010900089110000891100008911000089110000E8
:1010A0008911000089110000DD110000F911000014
:1010B00089110000891100008911000089110000C8
:1010C00089110000891100008911000089110000B8
:1010D00089110000891100008911000089110000A8
:1010E0008911000089110000891100008911000098
:1010F0008911000089110000891100008911000088
:101100008911000089110000891100008911000077
:101110008911000089110000891100008911000067
:101120008911000089110000891100008911000057
:101130008911000089110000891100008911000047
:101140008911000089110000711100007111000067
:101150007111000071110000711100007111000087
:101160007111000071110000711100007111000077
:10117000434800690024022809D001280DD0002826
:1011800002D103CA06F0D2FF204601B0F0BD03CA67
:1011900006F0BEFF204601B0F0BD03CA06F0DCFF3A
:1011A000204601B0F0BD022931D0022430E0344D98
:1011B00000242C616C619E49354A02F081F968690E
:1011C000401C6861204601B0F0BD02F0B3F928462A
:1011D00003F0CAFB0024204601B0F0BD284909698C
:1011E0000C234B432749CA58C918496802F068F9CB
:1011F0000024204601B0F0BD0024204606F042FF46
:101200000128C1D11E483030204900241CE00124AF
:101210001B490F690C26314679431A4A51188968CF
:10122000214208D000247D1C15490D614C61052D1B
:1012300010D3154906E012494869401C486103284B
:1012400012D32E4900241846224602F009FC2046FB
:1012500001B0F0BD6E430B498A598919496802F003
:101260002FF9204601B0F0BD0E20009000240A2284
:101270002846214602F0E4FB204601B0F0BDC046FE
:10128000FCAC010218660100FC6D0100DC6D010080
:1012900061840100B0B504291ED804468068C046A8
:1012A0007944097949008F4402191D15080016492F
:1012B00016A202F005F90020B0BD10490022204618
:1012C00002F0CEFB0E480168491C0160032901D1E0
:1012D00001F0DCFA0020B0BD0120B0BD02F02AF917
:1012E0000020B0BD00250321284606F0DBFE05499D
:1012F00020462A4602F0B4FB0020B0BDEC6D010090
:101300005CAD01026C6E0100881300004154453051
:101310000D0A0000B0B582B001240A2910D88368F4
:101320007944097949008F440E2905050B0B0B0BF5
:101330000B0B1A00194909680024224602F090FBA1
:10134000204602B0B0BD506814490860144915A287
:10135000184602F0B5F80024204602B0B0BD0024C3
:10136000019403CA09A201AB03F054FC0228E7D19F
:10137000019806F00DFF204602B0B0BD184602F0FD
:10138000D9F80024204602B0B0BDC0462B435351CB
:101390003A2025642C252A0D0A00000060AD0102C8
:1013A0008813000041542B4353510D0A00000000E4
:1013B000B0B582B00546002406F0E4FE01280DD148
:1013C00008498C60E86B426853684B600094019256
:1013D0006A4602F045FB204602B0B0BDE443204619
:1013E00002B0B0BDCCA30102B0B50546881E0228EC
:1013F0000AD3A868012913D0002915D10C490DA2E0
:1014000002F05EF80020B0BD0220014606F04AFE60
:10141000064900242846224602F022FB2046B0BDA1
:1014200002F088F80020B0BD0120B0BDBC6D010005
:101430008813000041542B4346554E3D300D0A00A1
:1014400080B5E0B00320C101684613F0F1FD094802
:101450000078002803D001F049FC002802D00020C9
:1014600060B080BD03206A46014612F0E9FA002010
:1014700060B080BD64AB0102F0B597B0102014904D
:10148000642013902648109002200E90E120400224
:101490001690244E304614301290052040021190D0
:1014A00001240F940EA9204609F056FE0027FD43A3
:1014B000002802D0284617B0F0BD0C36304603F0A5
:1014C00061FA0028F6D118480B901848099018487E
:1014D000089018480790184806903920059017483A
:1014E0000490174803900D960B2040020C900A9030
:1014F000144E03A9304602F04DF80028DAD10096C8
:1015000001940F4C104911A2124B204602F05CFAD4
:101510001149204602F08CFA3D46284617B0F0BD2E
:1015200090F0010294A9010290FA010290100202C7
:101530000D26000081260000DD2500007C6F0100E3
:101540002CAD0102282F02025C6D01004149523787
:10155000383045007C6E01004114000010B503488E
:101560000024047013F0B8F9204610BD7CB90102C4
:1015700080B501F079F9002080BD0000F0B58DB094
:101580000D4600240C940B940A9409940894079433
:1015900006940594029080680490406B0068019066
:1015A00006F06CFD07465BA105220392FEF729FEBB
:1015B0005A4E00281ED05AA105223846FEF721FEB9
:1015C000002817D058A105223846FEF71AFE002839
:1015D0000FD059A105223846FEF713FE002809D086
:1015E00057A105223846FEF70CFE002807D156A663
:1015F00000E04FA605A82021324603F0DDFB0120C4
:101600003F2D00D936E0C0467D442D796D00AF44B2
:101610003340474A57313131313131313131643022
:1016200031313131313131313131313131313131AA
:10163000313131313131313131313131313131319A
:101640003131313131311F1F1F1F1F1F1F1F1F1F3E
:10165000BE48416A04290CD1039A426284620C207C
:1016600050433D490A580818416805AB049801F0F9
:1016700027FF20460DB0F0BDB44D00206862A8627F
:10168000CD49364A049801F01BFFA86A401CA862A5
:10169000EFE7049801F04EFF019803F065F9E8E7E1
:1016A000AA48406A04E0A949486AC21E012A1CD817
:1016B000A649421C4A628C62062AD0D325491AE008
:1016C000A2494A6A052AD5D1062048628C6221497E
:1016D0000298224602F0C4F9CBE79C48406A0C21EC
:1016E00041431D4842584018BEE7886A401C886242
:1016F000032805D316490022029802F0B1F9B8E791
:101700000E20009000210A220198029B02F098F915
:10171000AFE7C04634363030300000008984010025
:1017200034363030320000003436303031000000C2
:10173000554E494E455400003436303036000000D6
:10174000343630303300000043544E45540000001E
:101750005C6D0100AC6D010054660100F583010071
:1017600070B5022956D30F2907D1784C217A012967
:1017700005D1002222728F494AE0012070BD86689F
:1017800003F026F9002006F085FC012803D1002093
:10179000032106F087FC0025284606F073FC01288B
:1017A00004D130346A490022204631E0304600F04E
:1017B000EFFD00282ED03046FFF7FAFD002829D093
:1017C00006F09CFC012807D15F498D60F06B4268F0
:1017D000E26252684A601AE0022006F053FC0128D7
:1017E00008D159498D61F06B4268E26252684A61E2
:1017F00010310CE0022006F04DFC01280AD15249BC
:101800008D62F06B4268E26252684A6220312A4679
:1018100002F026F9002070BD10B582B00346012009
:10182000272931D87944097949008F442C132D2D6B
:10183000162D2D2D2D2D2D2D2D2D2D2C2D2D2D2DF0
:101840002D2D2D2D2D2D1C2D2D2D2D2D2D2D2D2DD9
:101850002D2D2D2908F04EFA15E0DF4900221846FB
:1018600002F0FEF80FE00020019003CA08A201ABCD
:1018700003F0D0F9012806D1019808F059FB02E0E5
:10188000024801210172002002B010BDFCAC01022F
:101890002B51495552433A2022636C6F7365642281
:1018A0002C25640D0A000000B0B502294AD30F2987
:1018B00014D18568002006F0EDFB012803D100203B
:1018C000032106F0EFFB0024204606F0DBFB012895
:1018D00006D1D94830301E49002231E00120B0BD88
:1018E0002846FFF765FD00282CD006F007FC0128EC
:1018F00008D115498C60E86B4268CF4BDA625268B8
:101900004A601CE0022006F0BDFB012809D10E4907
:101910008C61E86B4268C84BDA6252684A611031E8
:101920000DE0022006F0B6FB01280BD106498C62BF
:10193000E86B4268C04BDA6252684A622031224644
:1019400002F08EF80020B0BD60A00102FCAC0102E4
:10195000DC6D010080B5022905D3042905D19E491B
:10196000002202F07DF8002080BD012080BDC0462D
:10197000B0B50546881E02280AD3A868012913D0ED
:10198000002915D10C490DA201F09AFD0020B0BD2F
:101990000220032106F086FB064900242846224641
:1019A00002F05EF82046B0BD01F0C4FD0020B0BDDD
:1019B0000120B0BDFC6D01008813000041542B4391
:1019C00046554E3D310D0A0010B50F290BD00129A7
:1019D0001DD000291DD1FFF7C1FD0020022106F016
:1019E00061FB002010BD0446002006F04BFB0128DF
:1019F00003D10020022106F055FB002006F04AFB2F
:101A0000012804D104490022204602F029F80020D0
:101A100010BD012010BDC046EC6D0100F0B581B0D5
:101A20000124322928D805468768786B0668C046A5
:101A30007944097949008F442F3F1919191F1F1F35
:101A40001F1F1F1F1F1F221F1F1F1F1F1F1F1F1FA3
:101A50001F1F1F1F1F1F1F1F1F1F1F1F1F1F1F1F96
:101A60001F1F1F1F1F1F1F1F1F1F26001E4900248F
:101A70002846224601F0F4FF204601B0F0BD1B4885
:101A8000017800291FD0184900242846224601F079
:101A9000E7FF204601B0F0BD0024FC6239693846FA
:101AA00088470028FAD011480470FC62FFF756FD01
:101AB0000E20009001220EE0304602F055FF002477
:101AC000204601B0F0BD01210170FFF751FD0E204D
:101AD000009000240522304621462B4601F0B0FF3D
:101AE000204601B0F0BDC0467C6D010064AD01022E
:101AF00010B586B0034601203B2900D956E0C04608
:101B00007944097949008F44505051513351515112
:101B100051515151515151515151515151515151B5
:101B200051515151515151515151515151515151A5
:101B300051515151515151515151515151391D1D15
:101B40001D1D1D1D0020059003CA02AA009218A2A7
:101B500005AB03F05FF8022827D1039A029817A17A
:101B6000FEF74FFB002820D1059808F0E1F91CE0B2
:101B7000B5490022184601F073FF16E000200290DC
:101B80000590049003CA05AA019204AA00920DA22E
:101B900002AB03F03FF8032807D1049A0599029895
:101BA00008F06CFA029808F007FA002006B010BDA1
:101BB00025642C2025700D0A00000000434C4F5373
:101BC000454400002B524543454956452C25642C7D
:101BD00025643A0D0A256500CC6D0100012901D864
:101BE0000020704701207047B0B50546881E0328C5
:101BF0000BD2104606F08AFA0F48C16A0024284624
:101C0000224601F02DFF2046B0BDAC6801290BD063
:101C100000290ED106F034FA0346084908A22046EE
:101C200001F04EFC0020B0BD204601F083FC0020F6
:101C3000B0BD0120B0BDC046FCAC0102881300005D
:101C400025730D0A0000000070B582B001240F2931
:101C50003DD803468568686B0668C04679440979B3
:101C600049008F4407141E343434342F373434344D
:101C70003434434E6648002404708461C4610121F9
:101C800001716649664A284601F01AFC1FE02846A1
:101C900001F050FC304602F067FE0024204602B0FE
:101CA00070BD5B48002404718269042111430278ED
:101CB000002A2ED0052958D1016A491C016259D247
:101CC000624961E0524B18780024002831D0204648
:101CD00002B070BD4E4B1878012816D103CA1833D4
:101CE00051A202F097FF002002B070BD48480024C6
:101CF00084610121017100784849002812D1484AC5
:101D000011E0434E307900281BD00024204602B059
:101D100070BD052932D10024012101708461C461A4
:101D200001713E493F4A284601F0CAFB204602B0F5
:101D300070BD03CA183340A202F06CFF204602B007
:101D400070BD002006F0A6F9012803D10020032170
:101D500006F0A8F90024204606F094F9012816D1CF
:101D600030362D49002430464BE000210162C16924
:101D7000491CC1610E20009000241CE0C169491C6F
:101D8000C161652915D330490024184639E0284639
:101D9000FFF70EFB00289AD006F0B0F9012812D107
:101DA0001C4900248C60E86B4268F26252684A6009
:101DB00027E00E20009002223046214601F040FE2E
:101DC000204602B070BD022006F05CF9012809D15E
:101DD000104900248C61E86B4268F26252684A61E3
:101DE00010310EE0022006F055F9012800D06EE710
:101DF000084900248C62E86B4268F26252684A62C9
:101E00002031224601F02CFE204602B070BDC046B3
:101E1000FCAC010260A00102DC6D0100881300002F
:101E20001E840100298401002B43475245473A2074
:101E3000252A2C25640000002B435245473A2025D3
:101E40002A2C256400000000CC6D01008C6D01007F
:101E5000B0B584B001243B2900D937E013460546CC
:101E60008068C0467944097949008F443F4932323D
:101E7000322F2F2F2F2F2F2F2F2F2F2F2F2F2F2F6F
:101E80002F2F2F2F2F2F2F2F2F2F2F2F2F2F2F2F62
:101E90002F2F2F2F2F2F2F2F2F2F2F2F2F2F2F2F52
:101EA0002F2F1D1D1D1D1D1D0024039403CB01AAF2
:101EB00000921C4A03AB02F0ADFE022806D1029A42
:101EC000019819A1FEF79DF900281FD0204604B003
:101ED000B0BD1848006808F02BF8174900242846C0
:101EE000224601F0BDFD204604B0B0BD11490B6093
:101EF0001E2112A201F0E4FA0024204604B0B0BD75
:101F000001F018FB0024204604B0B0BD0948006869
:101F100008F00EF808490022284601F0A1FD2046ED
:101F200004B0B0BD89850100434C4F5345204F4B51
:101F30000000000068AD01029C6D010041542B437C
:101F40004950434C4F53453D25640D0A00000000A5
:101F5000F0B589B0044601203B2900D9AAE0164615
:101F6000A7687A6B1568C0467944097949008F449F
:101F7000536AA071A1A1A1A1A1A1A1A1A1A18AA11E
:101F8000A1A1A1A1A1A1A1A1A1A1A1A1A1A1A1A141
:101F9000A1A1A1A1A1A1A1A1A1A1A1A1A1A1A1A131
:101FA000A1A1A1A1A1A11D1D1D1D1D1D00270897F7
:101FB00003CE06AA0092414A08AB02F02BFE02288B
:101FC00077D13F4805680898854272D1079A069EE6
:101FD0003CA130460592FEF714F9002847D03DA1F8
:101FE0003046059AFEF70DF9002840D03CA1304656
:101FF000059AFEF706F90028314E5AD1284607F017
:10200000B1FF7068401C706003283CD303207060EF
:10201000306807F02FFF36E029480660304607F0A9
:102020007DFF05902648006807F04CFF0490244887
:10203000006807F053FF0499019102900598012868
:1020400027D02EA026E0384601F074FA284602F088
:102050008BFC2EE01A4D286807F084FF6868401C4E
:10206000686003280FD300226A6022490DE0144EF5
:102070007760284607F08CFF306808F0A3F8002846
:1020800001D01B4900E00C490022204601F0E8FC89
:102090000FE019A000901A491AA23846334601F001
:1020A0000FFA0E2000900021B4222846234601F0AA
:1020B000C7FC002009B0F0BD9C6D010089850100BE
:1020C0000CAA0102414C524541445920434F4E4E07
:1020D00045435400434F4E4E454354204F4B000060
:1020E000434F4E4E454354204641494C00000000AA
:1020F0003C6E01005C6D010054435000554450009B
:102100008813000041542B43495053544152543DCD
:1021100025642C222573222C222573222C25750D53
:102120000A000000B0B582B014468A1E022A12D3FB
:102130008568012917D000291CD1204607F0B4FE7C
:1021400000901E210EA22846234601F0B9F9002472
:10215000204602B0B0BD09490024224601F080FCAF
:10216000204602B0B0BD284601F0E4F90024204624
:1021700002B0B0BD0124204602B0B0BD4C6E0100DB
:1021800041545E4845415254434F4E4649473D31C4
:102190002C25642C25750D0A00000000F0B583B0D5
:1021A00014468A1E022A1CD38568012921D00029E1
:1021B00026D1164F3C60204607F068FEFDF7F6FF7B
:1021C0000646386807F062FE7108009101901E21F2
:1021D0000FA22846234601F073F90024204603B0DD
:1021E000F0BD09490024224601F03AFC204603B024
:1021F000F0BD284601F09EF90024204603B0F0BD52
:102200000124204603B0F0BD9C6D01006CAD0102BD
:1022100041545E4845415254424541544845583D19
:1022200025642C25752C25730D0A0000F0B585B0AA
:10223000044601203B2900D988E0A5687944097942
:1022400049008F444257825E8383838383838383E1
:10225000838383836383838383838383838383836E
:10226000838383838383838383838383838383833E
:10227000838383838383838383831D1D1D1D1D1D92
:102280000020049003CA02AA0092314A04AB02F073
:10229000C1FC022859D12F4885680498854254D141
:1022A000039E029F2CA138463246FDF7AAFF002864
:1022B0003DD02BA138463246FDF7A3FF002844D17C
:1022C000284607F035FE29493BE0224CA260104623
:1022D00007F010FE002838D002F005FEE06000286C
:1022E00033D0A36840680090234924A2284601F017
:1022F000E7F82AE017480021C160284601F01AF9E2
:1023000023E01448806807F013FE19E001F082F919
:10231000012804D10F48C16803C901F0ABFA0D4888
:10232000C0680CC81349284601F00AF90DE0284698
:1023300007F0E0FD0028074907D0C96802F0A9FDB1
:102340000B490022204601F08BFB002005B0F0BDB8
:10235000898501000CAA010253454E44204F4B00D1
:1023600053454E44204641494C000000CC6D0100CD
:102370009C6D0100204E00008813000041542B4347
:10238000495053454E443D25642C25750D0A0000E7
:10239000F0B583B0074602F01BFB0026304607F07D
:1023A000B3FD032835460BD10421284607F0FCFE77
:1023B000F86B51492A4601F053FB304603B0F0BD9B
:1023C00002970024204607F09FFD0428254609D1E6
:1023D0000298C06B49492A4601F042FB2646304626
:1023E00003B0F0BD0027384607F08EFD05283D46B6
:1023F00009D10298C06B40492A4601F031FB3E46A4
:10240000304603B0F0BD01970125284607F07CFD5A
:102410000328029FC8D00125284607F075FD04282F
:10242000D6D00125284607F06FFD0528019FE0D092
:102430000225284607F068FD0328029FB4D0022534
:10244000284607F061FD0428C2D00225284607F07F
:102450005BFD0528019FCCD0254C2068401C032142
:10246000FDF74EFE0D46084607F04EFD0628029F7A
:1024700008D1284607F03EFD002803D002F033FDC6
:1024800000282AD1681C0321FDF73AFE0D460846B4
:1024900007F03AFD062808D1284607F02BFD002852
:1024A00003D002F020FD002817D1681C0321FDF79E
:1024B00027FE0D46084607F027FD0021CE430628DB
:1024C00000D07AE7284607F015FD002800D174E710
:1024D00002F009FD002800D16FE72560F86B05497F
:1024E0002A4601F0BDFA0026304603B0F0BDC046D2
:1024F00070AD01025C6E01001C6E01002C6E0100CB
:1025000080B58AB010200790642006900948039097
:102510000220019001200290E12149020991C34962
:102520001431059105214902049101A908F014FE16
:102530000AB080BD90F00102B0B582B001220F292F
:102540003ED803468068446B2468C04679440979C4
:1025500049008F44071F2527343535353535353546
:1025600035350A152749002204E02649CA68092A98
:1025700020D8521CCA601649164A00F0A1FF1EE07E
:10258000002005F07FFD012819D11E4830300E498A
:10259000002212E000F0CEFF204602F0E5F90EE046
:1025A0000D4908E00E20009000210122204601F094
:1025B00047FA04E005490022184601F051FA0022CA
:1025C000104602B0B0BDC046DC6D0100BC6D01001C
:1025D00088130000358401006C6D010080B5012076
:1025E00008F0A2FD80BD00000648416B00200029D4
:1025F00005D0054A914203D049680029FAD17047B5
:1026000001207047FCAC0102AC6D0100B0B514466E
:102610000D460846114602F0E5FA012802D1285D70
:10262000002805D001202946224608F0E9FEB0BD69
:10263000002C13D06019401E00780A280ED1814862
:1026400000780028EED000F051FB0028EAD10320EA
:102650000A4A01462B4611F0F3F9E3E7794800787E
:102660000028DFD000F042FB0028DBD10320034A22
:1026700001462B4611F0E4F9D4E7C046D3830100AC
:10268000F0B585B0054604A800240470E743002D8A
:1026900012D0EA68002A0FD0686A00280CD0A86A15
:1026A000002809D0401EE96A814200D38EE004A9C7
:1026B00028469047002803D03C46204605B0F0BD90
:1026C0005A4EE86A411CE962696A049A0A54E86A47
:1026D000696A002202920A54E86A092806D1696AE6
:1026E00009225148FDF777FD00283ED03078411E81
:1026F000022908D802F06CF9B168401A4C498842A6
:1027000064D84A4E30780A2820D0012823D16E6A36
:102710003A213046FDF740FD002847D0019002984D
:102720000390E96A03AB304642A202F073FA022832
:102730004CD10398002849D00A213C4A11700199D4
:102740000818696A401AC01C50602FE07068E96A76
:1027500081422BD13AE004A800780A280FD00D2836
:1027600014D101202863E86A1AE00120307002F0D9
:102770002FF9B0603078411E0229BBD9C3E7296B1D
:10278000012904D102202863E86A03E0296BE86A82
:10279000022905D1022817D10298E862286305E0D2
:1027A000012803D1686A00783E280FD0A86AE96A38
:1027B000401E81420AD2EA6804A9284690470028B0
:1027C0001A4E00D17DE777E702982863E96A686AC4
:1027D00002F008FA012822D1E86A002811D0696ABB
:1027E0004018401E00780A280BD1164800780028AF
:1027F00015D000F07BFA002811D16B6A032012A2D9
:102800000AE010480078002809D000F06FFA00288C
:1028100005D16B6A032010A2014611F011F903489B
:102820000470204605B0F0BD187D010094A9010296
:10283000DC0500002B524543454956452C252A2CE2
:1028400025643A0064AB01025B4154205265637613
:102850005D202573000000005B41542052656376C3
:102860005D2025730D0A000010B50C2400212046C0
:1028700005F0ACFC29480AF080F80121204605F05B
:10288000A5FC27480AF079F810BDC0460C240025A5
:102890002046294605F09AFC204E30460AF06DF895
:1028A00001272046394605F091FC1D480AF065F8DD
:1028B0004B20C101384608F007FD1A49132228466B
:1028C0002B4611F04FFEE1204102384608F0FCFC97
:1028D000C8200AF052F8FF200004134908608A4912
:1028E0000860124908601249086001460246034622
:1028F00006F09CFA2046294605F068FC30460AF0AE
:102900003CF82046394605F061FCBFF34F8F09487B
:1029100009490160BFF34F8F00BFFDE7DC050000F0
:10292000B80B00006CA70102843D0202D8380202F5
:10293000743D02020CED00E00400FA05B0B5012080
:102940000DF0D6FB1E4D2870132802D10DF088FC27
:10295000B0BD0F2003F024FB6870287033282AD103
:1029600020243721204603F078FB2120032103F0A7
:1029700074FB2220402103F070FB2320082103F088
:102980006CFB3020AA2103F068FB0E48022101876E
:10299000322003F062FB3320012103F05EFB5F2154
:1029A000204603F05AFB0F2003F0FAFA68700A2061
:1029B00009F0F8FFB0BD03480021C187B0BDC04693
:1029C000D0A8010202C30102F0B583B04A48002733
:1029D00007704A4E307883490978814236D1707A3F
:1029E000202833D1464802210160BF4B0120987254
:1029F0001F833079D872B27A1A737079B17909026B
:102A00000C189C839C820092520091190B313D4D11
:102A100032352846FDF788FB3B48FF21016001A8BD
:102A20000480B14CA178002913D03848027843784B
:102A30001B029A1801AB1B88934204D0801C7F1C98
:102A4000B942F3D10F46E782312904D9002003B0FF
:102A5000F0BD0027E7820098002812D00B365F48AF
:102A600002880020337874782402E31893420AD055
:102A7000B61CAD1C401C009B8342F3D19A4C009EB7
:102A80001AE0002618E0C6B2304600F041F8298866
:102A9000954CE78AE07A584AD055D019627B3223A8
:102AA000C2547800194A13185986A1788F4203D16D
:102AB000A38A1352491CA170CAB2207B864207D157
:102AC000BBB2934204D100F023F8002003B0F0BD64
:102AD0000028BBD1A38A02AC23800906F3D00B499E
:102AE0000B784C782402E31802AC24889C42ADD0C9
:102AF000891C521EF4D1E6E75FAB0102883D020259
:102B000040A8010298AC0102F85B020234AC010259
:102B1000F0B581B0304C212100916172724FF87094
:102B20002E4909886170BA8A62712D4B1B88E37146
:102B30007D6B7D622B4E36782670090AA170110AD2
:102B4000A171190A2172284941434819274945189A
:102B5000BD630EF015FD40190FF01AFA06460D463A
:102B60002348007C0FF0A0F8224909882222A154B2
:102B700082B2D20B801802B2D0175210B21868413C
:102B8000130E009D6355130C202563553B6EA376F1
:102B90001D0AE5761D0C25771B0E6377234622332D
:102BA000090A5970A277BA65F865BA66F866100A1C
:102BB000E0770EF04FFDB862BB6B2821012520465F
:102BC0002A4612F031F97D713871F88A0A490918DC
:102BD0000020487601B0F0BD1E3E020270AB01023B
:102BE00078AB010263AB0102C0F30000200C0100CE
:102BF00044A0010272AB0102C4AB010270470000A5
:102C0000F0B585B0204804902048039020480290F9
:102C100020480190204F3C46183401A920460AF074
:102C200043F93D4608353E46103620462946324691
:102C30000AF028F82046294632460AF023F8B868F8
:102C4000F9680024154B2246FDF7E6FC144A154BA3
:102C500012F034FF02460B4613492046FDF766FC8E
:102C6000124B2246FDF770FCFDF746FE3860B8684F
:102C7000F96822462346FDF78DFD002800D03C6010
:102C8000002005B0F0BDC0464F29010051290100C8
:102C9000BD2801001529010030A9010200AA8F40BA
:102CA0006C45D9CC955BC83F0000F03F40A5E5409E
:102CB00070470000002909D000220378D3189AB287
:102CC000401C491EF9D1D84380B27047014880B2F8
:102CD0007047C046FFFF000080B5012012F082F867
:102CE00001480021017280BDE0AA010280B500F018
:102CF00031FB002802D07648406880BD012080BDAD
:102D000080B58AB00020079006900590802104913C
:102D100011490391022101910290E1214902099197
:102D200001A908F019FA002801D00AB080BD0B49AA
:102D30000B480C4A42500C490C4A42502D21490183
:102D40000B4A4250B321C9000A4A425001F0D0FC5C
:102D500006F0DAFA0AB080BD902E02029405000057
:102D6000303002021D2E00009C050000712E000074
:102D7000112E00009D2E0000F0B581B000F0EAFA9F
:102D8000534E002806D07068002803D101F070FB74
:102D900001B0F0BD00F0DEFA002813D07068012801
:102DA00010D000F0D7FA00280AD07068032807D1A5
:102DB000694600240C70204608F0B6F9002805D0BA
:102DC00001B0F0BD00F0BEF901B0F0BD0F4F0AE058
:102DD0007C606D46287808F033FC0020294608F016
:102DE000A3F90028ECD1684600780328F0D17D686B
:102DF00001F0EEFD002D07D07968401AC928E8D30C
:102E0000746001203870E4E77860E2E750AB0102BB
:102E100080B50146002008F087F980BD83B0B0B5C9
:102E2000FFB082B0044685918692879300F092FAB3
:102E300001460020002914D025494968002910D1F5
:102E400085AB8093012041026D462846224612F050
:102E5000EFF82846FDF7AAF902460020294608F0B7
:102E6000CFFA7FB002B0B0BC02BC03B00847C04686
:102E700080B582B001A9087000F06CFA014600200C
:102E8000002908D012494968002904D1002001A96D
:102E9000012208F0B5FA02B080BDC04610B5044664
:102EA00000F058FA0146002000290BD00849496873
:102EB000002907D12046FDF779F902460020214676
:102EC00008F09EFA10BDC0460149486000207047D6
:102ED00058A00102B0B582B0194C2068056801A95C
:102EE0000020087007E090470198401C01A9087075
:102EF000C0B2082822D2012211048140294209D0FF
:102F00002268516080002018826A002AECD001A853
:102F10000121E8E7130283402B4201D0022104E0A3
:102F200082402A42E0D00321134622685360800089
:102F300020188268002AD7D001A8D4E702B0B0BD1B
:102F4000D8A20102FEE7000010B509480168CA696D
:102F500020231343CB610269032A08D10122930580
:102F60000C689C430C605102C26E0A43C26610BDDD
:102F70004CA3010281B010B581B00393002807D0A3
:102F8000C16A002904D003AB0093C46A0021A047A2
:102F900001B010BC01BC01B00047000080B5024682
:102FA00008480068002807D091B2120C03889A42A2
:102FB00003D040690028F9D180BD002200F0ACFCAC
:102FC00080BDC046242F0202F0B581B05C4C206861
:102FD000856BE80707D0E168002904D00020884706
:102FE000206801218163A80707D52169002904D041
:102FF00001208847206802218163680707D561693D
:10300000002904D002208847206804218163280712
:1030100007D5A169002904D003208847206808212A
:103020008163E80607D5E169002904D004208847B8
:10303000206810218163A80607D5216A002904D0E1
:1030400005208847206820218163680607D5616ACA
:10305000002904D006208847206840218163280683
:1030600007D5A16A002904D007208847206880215D
:1030700081630126E80507D5E16A002904D03702FB
:103080000820884720688763A80507D5216B002999
:1030900004D077020920884720688763680507D530
:1030A000616B002904D0B7020A2088472068876333
:1030B000280507D5A16B002904D0F7020B2088470B
:1030C00020688763E80407D5E16B002904D0370343
:1030D0000C20884720688763A80407D5216C002945
:1030E00004D077030D20884720688763680407D5DC
:1030F000616C002904D0B7030E20884720688763DD
:10310000280407D5A16C002904D0F7030F208847B5
:1031100020688763E80307D5E16C002904D03704F1
:103120001020884720688763A80307D5216D0029F0
:1031300004D07504112088472068856301B0F0BD74
:10314000DCA3010210B582B001A90020087007F0CD
:10315000EBFF002809D101AC207800F009F800202D
:10316000214607F0E1FF0028F5D002B010BD0000B5
:10317000F0B587B0624E3168032910D002294FD0D4
:10318000002900D0B5E0242800D0B2E0842001213D
:103190003150022030602420307107B0F0BD0A2881
:1031A00000D0A4E08427F059411CF151341D0A21BC
:1031B0002154F0590025255452A12046FCF7D8FF90
:1031C000002857D0F15903A80090504A05AB20467B
:1031D000029101F01FFD022835D101950499039851
:1031E00001F080FC059A1178069B022B06D3521C35
:1031F0005B1E15786940521C5B1EFAD1C0B2814239
:10320000019D20D143A205AB2046029901F002FDA9
:103210000F2870D10598FDF703F83D49087016E0B6
:1032200084217258531C7350B218107171587E2942
:1032300003D30020306007B0F0BD0D2859D1032022
:10324000306007B0F0BD32488178491C8170F05978
:10325000801985703B48418C002928D02F462C4D81
:103260002978C08C01280AD1002916D0204607F001
:10327000E5FD1CE026484178491C417037E00029F3
:103280000BD0314D2978491C2970C9B288420ED81B
:10329000204607F0D3FD2F7009E0A888401CA880C5
:1032A00080B23C2803D3204607F0C8FDAF80184801
:1032B0000078052810D8C04678440079400087443B
:1032C0000205080B0E13FF2000020AE01F48FF2131
:1032D0000CE0FF20000400E01D48FF3001E0FF206B
:1032E00000041A49086002E01848194901600020EA
:1032F000306007B0F0BD0648C178491CC170A6E730
:10330000A82F02024747412C00000000687B010003
:1033100020A9010224252A2C252A2C252A2C252AFD
:103320002C252A2C252A2C25702C252A2C252A2CC4
:10333000252A2C252A2C252A2C252A2C252A2C2501
:103340002A2A000002C3010274AD0102843D020278
:1033500000FFFF00014800787047C04684A80102C2
:1033600070B5174E304618303146083132461032AB
:1033700009F088FCB068F1680024124B2246FDF782
:103380004BF9114A114B12F099FB02460B461049BA
:103390002046FDF7CBF80F4B2246FDF7D5F8FDF799
:1033A000ABFA05463060B068F16822462346FDF767
:1033B000F1F9002801D034602546284670BDC0468A
:1033C00030A9010200AA8F406C45D9CC955BC83F5B
:1033D0000000F03F40A5E540F0B58DB0002862D078
:1033E0000446406800285ED0A06840285BD8E56AA3
:1033F000002D58D00746204640300026039003E0B9
:10340000019E4AE0039848E0402101220691FCF722
:103410009DFEAE4202963ED20020314601900990B8
:103420000398069B3E46002EEAD0606A0491405CF9
:1034300007900998401C0590002104270891651801
:10344000EA5C012A17D10A966268D3191B1F1B6810
:10345000099E9E5D0798864208D1059D5B5D002B05
:103460000A9E22D00898401C089003E040350022B4
:103470002A70A668069B0837491CB142DFD308981A
:103480000028BFD00499491CE06A81420598099040
:103490000398C8D301E003983E463746E56A029E8A
:1034A000761CAE42B0D30DB0F0BD616A0B91E16AFB
:1034B0000C91D1590BAA204600F09CF80DB0F0BD3C
:1034C00081B0B0B583B00D460446079307AB0293B5
:1034D0008069E16911F0ACFD206265480078002840
:1034E00003D1216AA06900F001FA6369A169226A27
:1034F000204698470146A06B002905D069460C601C
:103500000021224B0A460CE001F02EFA7D208100BA
:103510002846FCF7DFFD0246A06B69460C600021DF
:103520001B4B01F07DFA002003B0B0BC02BC01B01F
:103530000847C04680B5806B01F016FA002080BDB8
:1035400070B582B00D460446466911461A46B0472A
:103550000146A06B002907D069460C6000210B4B87
:103560000A4601F05DFA0EE001F0FEF97D208100CF
:103570002846FCF7AFFD0246A06B69460C600021AF
:10358000034B01F04DFA002002B070BD7936000007
:103590008F36000070B50D460446802101F09EFA7A
:1035A0002868E06368686060A868A060E868E06018
:1035B0002869206168696061A869A061E8690026DE
:1035C0002662E061286A6062686A2663E662A06239
:1035D000A86A60632046383001F0D4F9002802D090
:1035E000F643304670BD21480168216004603046D2
:1035F00070BDC04670B514460D460646881E0328A9
:1036000002D8B06B01F0B0F9F06B2946224600F009
:1036100083F970BD16480178012048407047C046C4
:1036200070B512480468002C1FD0114E11A52169F5
:1036300020468847002815D1307800280DD1E16A4E
:10364000606A01F0CFFA0146606A012903D0E16A9D
:1036500000F010F9284600F0E3F82046FFF7BCFE22
:103660000020E0622468002CE1D170BD182F020216
:10367000102F02020D0A000010B50446806B01F005
:1036800073F9E06B0521002200F046F910BD10B57A
:103690000446806B01F068F9E06B0421002200F021
:1036A0003BF910BDF0B581B000910646C7680468CB
:1036B000A01C3946FCF70EFD00257068814201D13F
:1036C000ED430BE0601C3946FCF704FD31603269C4
:1036D0005143B06808180099FCF726FD284601B050
:1036E000F0BDB0B5012400250560446008300EC06F
:1036F000B0BD70B50E460446C1680068401CFCF7BA
:10370000E9FC00256068814202D1ED43284670BD86
:1037100022695043A16841183046FCF705FDE16875
:103720006068401CFCF7D6FC6160284670BDB0B5EF
:10373000002400280DD0054600688842FDD3401AB9
:10374000286068684018E968FCF7C4FC6960204696
:10375000B0BDE4432046B0BDB0B5002400280ED073
:103760000546006840182860EA689042FDD8A868BD
:1037700040181146FCF7AEFCA9602046B0BDE443FA
:103780002046B0BDF0B583B0164602460027F84388
:10379000002E22D01C46002B1FD00D46D168136886
:1037A00099421AD9CB1AAB4217D392680192521997
:1037B0008A423A4607D9019A8A1A0292029A521903
:1037C0009342029A09D3029201981018FCF782FCE6
:1037D0003160029840192060384603B0F0BD40685F
:1037E00070478068704702460020002A04D01060AD
:1037F00050609060D1607047C0437047002803D08C
:10380000016848424841704701207047002805D0B0
:103810000168C068411A484248417047012070471A
:1038200083B070B5FFB082B00446859186928793CD
:10383000FFF790FD002814D036484068002810D1CA
:1038400085AB80930A4E711C6D462846224611F0C6
:10385000EFFB0246B04200D332460020294607F073
:10386000CFFD00207FB002B070BC02BC03B008479F
:10387000FF010000F0B593B00C460546FFF76AFD66
:10388000002806D023484168002902D10078012889
:103890001FD0002013B0F0BD284639463246029BA7
:1038A00001F0E8F83046FCF781FC0D213154301866
:1038B0000A2141700295002585703046FCF776FCA0
:1038C00002462846029D314607F09AFDED19E41B99
:1038D000DFD003AE402130460291FCF73EFC0120D0
:1038E0000090102C2746D7D31027D5E7B0B50C464B
:1038F0000546FFF72FFD01460020002908D00549A5
:103900004968002904D100202946224607F078FDA5
:10391000B0BDC04658A00102F0B583B014460D46B4
:1039200006464088012818D1306900280CD0A9002B
:10393000405801782D2910D0F368716809686A46EB
:103940001160506010A205E0F36870680068694675
:1039500021C115A23046FFF70DFB7768FB683046A2
:10396000294622469847012808D00AE0C368304615
:103970002946224698477F68012802D178680028A6
:10398000F4D103B0F0BDC04646534D3A252D3873EF
:103990002053544154453A252D323873204556451D
:1039A0004E543A25730D0A0046534D3A252D38736F
:1039B0002053544154453A252D32387320455645FD
:1039C0004E543A25750D0A00F0B581B0002828D074
:1039D0001E460C460546079B06980090002068622C
:1039E000A862E862104909886B8029800F4B1F6824
:1039F0006C60009BAB602B460C33C4C3A861E861CC
:103A00002862481C0849088008480560002C08D036
:103A10006C60002128460A46FFF77EFFA468002C50
:103A2000F6D101B0F0BDC046D4380202242F020204
:103A300002460020002A01D0D1627047C04370477F
:103A400010B582B004AC24881B881B041B196C467B
:103A50002360024B00F0E4FF02B010BD9D2F000078
:103A6000F0B597B01646029105464268002A30D05C
:103A700001966A6001210024284616462246FFF777
:103A80004BFF3046029FBE4232D003A85021FCF7C4
:103A900064FB32467268002F0CD003AF029811C746
:103AA0004068083F824209D0394608313C46002828
:103AB0000F46F4D1002A019EDBD10AE0019E38684E
:103AC0006860002128463246FFF726FF7F68002FF6
:103AD000F5D102988468002C08D06C60002128463B
:103AE0003246FFF719FFA468002CF6D117B0F0BDDD
:103AF00000212846019E3246FFF70EFFE9E700004D
:103B0000F0B581B0044680680A4601282DD84329C3
:103B100065D0442A6DD07E2A00D0C8E0226E002AEB
:103B200000D1C4E0616E012900DAC0E08A4200D110
:103B3000BDE04B1C934200D3C4E07E4AA518621836
:103B4000813200928E1C002701E07F1CA06829684A
:103B5000012801D12A2001E00098C05D8847F019B2
:103B6000216E8842F1D3BD1CADE0413903290CD848
:103B70007944097949008F4401477C8E0321002252
:103B8000204600F0DDF801B0F0BD7E2A00D08EE0C6
:103B90000026E66626676079012800D987E0206E56
:103BA000002800D1C1E0626E012A00DABDE0904237
:103BB00000D1BAE05F4BE158E518571C874200D3AB
:103BC0009CE0A018813000900098805D8847761CAA
:103BD000B8192968226E9042F6D3761C8FE0216EC8
:103BE000626E8A4263D253496158012861D12A200A
:103BF00062E0606E01285ADB401E60664D48215825
:103C00000820884701B0F0BD0020E0662067607999
:103C100001284CD8E06F002849D0A06F09300A2154
:103C2000FCF76EFA606F88421FD0401C0A21FCF737
:103C300051FA61672920C00025186426714369186C
:103C400020468030FCF7D4FAFCF7B0FA20666066B4
:103C5000B320C700E15938488847606F704328187F
:103C6000E1598847E159354888470120607101B022
:103C7000F0BD0020E0662067216E606E884216D29B
:103C80002C49615820188022805C8847606E401C57
:103C9000606601B0F0BD0020E0662067606E01281C
:103CA00005DB401E6066234821580820884701B084
:103CB000F0BDA0188022805C8847606E401C606662
:103CC00001B0F0BD01251B4EA15920208847A6193F
:103CD0003168082088476D1EFAD1216E606E8842D7
:103CE00008D2211881228A5C8023CA54401C216E8C
:103CF0008842F6D3481E206601B0F0BD0126202080
:103D00008847296808208847761EFAD1216E606EA0
:103D1000884208D2211881228A5C8023CA54401C20
:103D2000216E8842F6D3481E20660020607101B0E3
:103D3000F0BDC0469C050000A8870100AB870100CC
:103D4000F0B583B0044609292ED16079012800D945
:103D500067E1256E002D00D161E1206F002809D1B7
:103D6000012020672046E430214680312A46FCF7B6
:103D7000DBF9A566E56E00F037FD854200D347E12B
:103D80002546E435E06E00F033FDA26E2946FCF7CF
:103D900038FA002800D122E1E06E461CE66600F009
:103DA00023FD8642EED333E10026E6662667481EF1
:103DB000072800D935E1C04678440079400087449F
:103DC00003416576AAB6C5EB6079012800D928E1E0
:103DD000206E622832D81546F24EA1591046884707
:103DE000206E616E401E884208DB211880228A5CAA
:103DF0008123CA54401E616E8842F6DA6018802121
:103E00004554606E471C6766216E491C21668F42CF
:103E100014D2A51920188130029000260298805DE6
:103E200029688847761CB819216E8842F6D3002786
:103E30002968082088477F1CBE42F9D100206071A4
:103E400003B0F0BD206E002800D1ECE061790129BB
:103E500000D1EFE0002900D027E121468031002584
:103E60000D54A06F64224243A0182922D20080186A
:103E7000FCF7BEF9A06F082800DC451CA567E06FC1
:103E8000401C0A2800D30A20E0670EE1607901286F
:103E900000D9C6E0E06F002800D1C2E00A2800D0B7
:103EA0001DE1606FA16F884200D141E120E160799E
:103EB000012800D9B5E0E06F002800D1B1E0A06F83
:103EC00009300A21FCF71CF9606F88421FD0401CA2
:103ED0000A21FCF7FFF861672920C0002518642635
:103EE0007143691820468030FCF782F9FCF75EF9CF
:103EF00020666066B320C700E159AB488847606F11
:103F000070432818E1598847E159A848884701209B
:103F1000607103B0F0BD606E012800DA81E0401EE0
:103F20006066A04821580820884703B0F0BD216E84
:103F3000606E884275D29B49615820188022805C4F
:103F40008847606E401C606603B0F0BD6079012850
:103F500067D8206E002800D105E1606E012800DAE4
:103F600001E1904EA15908208847A519A159206E5A
:103F7000626E0292824200D3DEE0029827188037F8
:103F80000026B85D8847761C029880192968226E41
:103F90009042F6D3761CD0E06079012841D8206E9B
:103FA000002800D1FAE0626E012A00DAF6E09042C1
:103FB00000D1F3E07B4BE158E518571C874200D352
:103FC000D5E0A018813002900298805D8847761C69
:103FD000B8192968226E9042F6D3761CC8E0B32047
:103FE000C500615975A088476559E06E00F000FC76
:103FF000A847E06E00F0FCFB014620468030FCF74D
:10400000F7F8FCF7D3F820666066E06E401CE066C7
:10401000E56E00F0E9FB854201D30020E066002058
:10402000607103B0F0BDB320C000215862A0884782
:1040300003B0F0BD532000012518676F6426304699
:10404000784320182921C900029141182846324698
:10405000FCF76AF8A06F09300A21FCF751F88F428B
:104060000095019601D13E4617E0781C0A252946A5
:10407000FCF730F80E46019A574302982118C819E8
:1040800013467343C918FCF74FF8A06F093029464F
:10409000FCF736F88E423746E7D1019A5643A0190D
:1040A000029940180099FCF73FF8B320C600A159C7
:1040B0003FA08847204600F051FC2046803000F0A9
:1040C00057FB0025284600F049FC25666566A06F71
:1040D0000A306067A15937A0884703B0F0BD0A21B4
:1040E000081AA26F8018FBF7F5FF606F88421FD097
:1040F00009300A21FBF7EEFF61672920C00025186F
:1041000064267143691820468030FCF771F8FCF78B
:104110004DF820666066B320C700E1592248884701
:10412000606F70432818E1598847E1591F48884754
:104130000120607103B0F0BD012620208847296866
:1041400008208847761EFAD1606E401E606605E042
:10415000211881228A5C8023CA54401C216E884227
:10416000F6D3481E20660020607103B0F0BD012622
:1041700020208847296808208847761EFAD1216EBA
:10418000606E884208D2211881228A5C8023CA543A
:10419000401C216E8842F6D3481E206600206071C4
:1041A00003B0F0BD9C050000A8870100AB870100AB
:1041B0000D0A00003E0000000D0A3E000D1B5B4A88
:1041C0003E000000F0B581B0491E072900D9C9E0C2
:1041D00015460446B320C0002618C0467944097924
:1041E00049008F44030DBFBF2C384466206E6228FF
:1041F00000D9B7E07168A06801287FD12A207EE04D
:10420000A268216E0B461343002B72D0012A00D105
:10421000B3E0002A00D0A5E02546803500266E5484
:1042200021588FA088470120A0602666666610345A
:10423000102120462A4600F0BFFD01B0F0BD606E9F
:10424000012800DA8EE0401E606679482158082077
:10425000884701B0F0BD216E606E884200D381E0D6
:1042600073496158A268012A7ED12A207FE0206E1E
:10427000002877D0606E012874DB716808208847B9
:10428000206E656E854200D394E060198030009006
:1042900000277168A068012801D12A2001E0009858
:1042A000C05D88477F1CE819216E8842F1D37D1CD0
:1042B00081E0206E002855D0616E012952DB8842D2
:1042C00050D04D1C854200D38EE0601881300090A4
:1042D00000277168A068012801D12A2001E0009818
:1042E000C05D88477F1CE819216E8842F1D37D1C90
:1042F0007BE021585548884701B0F0BD28468847E3
:10430000206E616E401E884208DB211880228A5C84
:104310008123CA54401E616E8842F6DA60188021FB
:104320004554606E471C6766216E491C21668F42AA
:1043300018D220188130009000257168A0680128EB
:1043400001D12A2001E00098405D88476D1C781952
:10435000216E8842F1D30024716808208847641CCC
:10436000A542F9D101B0F0BD20188022805C8847B9
:10437000606E401C606601B0F0BD224680320027AE
:1043800057542766254620354021284600F014FD65
:1043900020461030294600F0B3F9316800283DD09E
:1043A00024A08847316829488847A7602766676640
:1043B00001B0F0BD01257168202088477168082090
:1043C00088476D1EFAD1606E401E606605E02118B8
:1043D00081228A5C8023CA54401C216E8842F6D315
:1043E000481E206601B0F0BD012571682020884775
:1043F0007168082088476D1EFAD1216E606E884270
:1044000008D2211881228A5C8023CA54401C216E64
:104410008842F6D3481E206601B0F0BD0CA0884744
:104420000220A06027666766677101B0F0BDC046D4
:104430009C0500000D0A55736572207665726966E9
:1044400079206661696C65642E0000009B8701001D
:104450000D0A57656C636F6D65210D0A3E00000003
:104460000D0A70617373776F72643A200000000068
:10447000F0B587B006A800270770A0480468002C94
:1044800000D12EE1994E01972D204501615906A8D2
:104490008847002800D020E1601905909248201834
:1044A000049020468030029020468130009000F039
:1044B0008FFA06A90D7829461B39402900D92EE02C
:1044C0007944097949008F44324646464646464675
:1044D000464646464646464646464646464646467C
:1044E0003A464646464646464646464646462020C4
:1044F00020204646464646464646464646464646A8
:10450000464646464646464640002179022922D183
:1045100020462946FFF7F4FA04202071D6E07E2DCC
:1045200019D12179032916D17E212046F2E721797C
:1045300004220A43042A0ED101202071C6E0217909
:10454000022908D103202071C0E02179012902D17C
:1045500002202071BAE02771E168411AB1420ED3FE
:10456000002121666166A160E060284609380228C2
:1045700000D2ABE0082D19D00D2D05D03AE0A0688F
:10458000012807D80D2D0AD102210D222046FFF760
:1045900019FE9BE00D2D33D102210D223AE0284671
:1045A0000938022800D291E0082D23D1206E00287E
:1045B00000D18BE0606E012800DA87E00498016882
:1045C00008208847206E656E854265D2029846199C
:1045D000002704980168A068012801D12A2000E082
:1045E000F05D88477F1CE819216E8842F1D37D1C5D
:1045F0003E4E52E0012120462A46FFF7E3FD65E0EA
:104600000A2D63D0092D03D0082D07D1072100E022
:10461000092100222046FFF793FB57E0E766276752
:104620006079012852D8206E6228049830D8016839
:1046300028468847206E616E401E884208DB21189C
:1046400080228A5C8123CA54401E616E8842F6DA59
:10465000601880214554606E461C6666216E491CB8
:1046600021668E42049F13D2009908180390019D81
:104670000398405D396888476D1C7019216E884227
:10468000F6D30026396808208847761CB542F9D150
:10469000019F6771154E19E00125049F396820209C
:1046A00088473968082088476D1EFAD1606E401E21
:1046B000606605E0211881228A5C8023CA54401C70
:1046C000216E8842F6D3481E2066019F0598016836
:1046D00006A88847002800D1E9E62468002C00D00D
:1046E000D2E607B0F0BDC0469C050000110E0000E8
:1046F00002490A68026008607047C0461C2F020227
:104700000020704780B506480068002805D005499C
:104710004158002901D004A08847002080BDC04630
:10472000202F0202940500001B5B481B5B4A00001F
:10473000F0B50023DA43002818D0002916D0012450
:10474000814D804E2A68002A09D1DA0087582F60EF
:10475000821852686A603268521C32605B1C002208
:104760004F2C03D80835641C8B42EBD31046F0BDA8
:10477000F0B595B0044600E0641C20782028FBD0FA
:1047800000282DD02046FBF711FD2018811E497806
:10479000202909D10121C943401800214170411E3F
:1047A000007820280846F8D0202101AA14232046AA
:1047B00000F013FB009063480668002E10D000251F
:1047C000614F38682146FBF7F8FC002804D0083711
:1047D0006D1CB542F5D303E07A6801A900989047B3
:1047E000002015B0F0BDC046564800687047C0466E
:1047F00054490968814203D9C00053490858704799
:1048000000487047D77C0100564800687047C04692
:10481000F0B581B04B4E3168002900D18FE04A4F8E
:1048200020370720C04300900420484C12E00020AD
:10483000002873D001228D4273D2002879D04449D8
:104840004258002A6FD039684248904720680028B3
:1048500069D16EE005462068002801D1024600E0DB
:1048600001222B1F8B425CD200280ED0384A82587E
:10487000002A06D0009880003958364890472068B2
:104880003168002804D1024603E000200028FAD055
:104890000122EB1E8B4244D200280FD02C4A8258B2
:1048A000002A07D00098800038188168294890476E
:1048B00020683168002804D1024603E00020002867
:1048C000FAD00122AB1E8B422BD200280FD0204AF7
:1048D0008258002A07D000988000381801691D48C6
:1048E000904720683168002804D1024603E0002088
:1048F0000028FAD001226B1E8B4212D2002896D0DB
:10490000134A8258002A07D000988000381881691D
:10491000104890472068316800288BD102468D42AC
:104920008BD3002A05D00A494158002901D00AA09A
:104930008847681D283731686A1C8A428AD300205C
:1049400001B0F0BDB8A6010234A40102202F02027A
:1049500094050000B58701000D0A000001490860B8
:104960007047C046202F0202014600201F2901D9AE
:10497000C043704718224A43344901238B50891899
:104980008860704710B50021CC4300280BD00A4A3C
:104990001368002B09D01832491C2029F8D306D1FE
:1049A00006A0FEF73DFF204610BD01231360016005
:1049B0000024204610BDC046D435020274696D65DE
:1049C000722049442069732066756C6C0D0A0000E2
:1049D000264800687047C04670B520241B4D234E02
:1049E0002868022817D13068A968EA68401A9042FE
:1049F00011D96969002907D02879002807D0022039
:104A000028603068A86004E00120286003E00120ED
:104A10002860286988471835641EE1D170BDC046FA
:104A2000F0B5044600201F2C01D9C043F0BD059D00
:104A300018266643054C0227A751A41921710B497A
:104A400009682646083626C66361F0BDD4350202E1
:104A500006480168491C0160054841680268002356
:104A6000521C02604B4143607047C0465CC7010264
:104A700060C70102F0B50446002000292DD0002CAB
:104A80002BD0002A29D0059D012D01D0022600E05F
:104A900003264E43761C9E421FD8002023785F09D0
:104AA0001E09052F01D3373600E0303616540F2685
:104AB00033400A2B01D3373300E0303316187370BC
:104AC000831C012D03D12026D654C01C00E01846BB
:104AD000641C491EE2D100211154F0BD80B5FBF7E2
:104AE0003CFB80BDB0B5002923D000231A4601E06D
:104AF000573C07E004781201302C1D4611D3392CA5
:104B000002D8303C25460CE0412C1D4609D3462CEA
:104B100001D8373CF6E72546613DEDB2062DE7D3D7
:104B20000025ECB21219491E401C0029E2D11046A2
:104B3000B0BD00221046B0BDB0B50278002A24D026
:104B4000441C0021084601E0573A08E023460001D2
:104B5000D5B2302D0C4611D3392D02D8303A144637
:104B60000CE0412D0C4609D3462D01D8373AF6E723
:104B70001446613CE4B2062CE6D30024E2B280186D
:104B80005C1C1A78002AE1D1B0BD0020B0BD000045
:104B900070B588B00D460646002407940694059427
:104BA0000494FBF703FB014604A86A46906005A83D
:104BB000506006A810600A4A07AB304600F02AF899
:104BC000042808D107982870069868700598A8707E
:104BD0000498E87000E0E443204608B070BDC04689
:104BE000BE87010010B50246012000290DD0002328
:104BF000D45C202C02D37F2C04D307E00D2C01D0F1
:104C00000A2C05D15B1C8B42F2D310BD002010BDD5
:104C1000002010BD81B0F0B584B009930023039348
:104C2000002800D1C2E0002A00D1BFE009AB039305
:104C30001678002E00D1A8E05623DB430093002312
:104C40001D46002900D1A2E0252E3FD1971C5278A5
:104C50001446643C0023142C43D8C0467C44247979
:104C60006400A7440A99A3A3A3A3A3A3A3A3A3A3F4
:104C70004CA3A3A3A3A3A3A35F000297039A131DAE
:104C80000393126801920122002317461E460478FE
:104C9000FF0703D02D2C01D1164607E02746303FF1
:104CA000092F09D80A275F433B19303B491E401C96
:104CB00000270029EBD13946029A019C002C03D031
:104CC000012E00D15B4223606B1C06E00378B342E7
:104CD0005BD1491E521C401C2B461678002EAFD1CA
:104CE00064E02A2A62D13A780378934204D0491EBC
:104CF000401C0029F8D100216B1C3A46EDE7039ACD
:104D0000131D03933E7812680023C45CB44233D071
:104D1000491E5B1C0029F8D13C46C7180021002A17
:104D20002ED12EE00297039A131D039312680023DD
:104D3000009E0778302F18D33A2F02D234462734FA
:104D40000BE0612F03D3672F344606D30DE03C46BA
:104D5000413C052C09D8344620341B011B19DB19B2
:104D6000491E401C0029E4D10021029C002A00D0E9
:104D700013606B1C2246B0E73C46C718002A00D0DF
:104D800009C26B1C22463846A7E700230EE0252EF9
:104D90000BD15178652908D103990A1D039209683E
:104DA000002900D008606B1C00E02B46184604B0B8
:104DB000F0BC02BC01B0084781B010B581B00C4610
:104DC000039303AB009310F033F9A04200D3601EAD
:104DD00001B010BC02BC01B0084770B50446002009
:104DE000002A1BD0002C19D0002B17D014600120F2
:104DF000022B13D32578002D10D0641C01208D4286
:104E000005D1651E00262E7085005451401C984225
:104E100004D2661C2578002D3446F0D170BDB0B5A3
:104E200004467821FBF7B8F9002805D1582120461F
:104E3000FBF7B2F9002828D04278002A23D0841C3E
:104E40000021084623460001D5B2302D0C4613D36D
:104E5000392D01D8303A0EE0412D0C460CD3462DA9
:104E600001D8373A07E01446613CE4B2062C01D37E
:104E7000002401E0573A1446E2B280185C1C1A780C
:104E8000002ADFD1B0BD0020B0BD2046FBF7C8F935
:104E9000B0BD70B504460026F043002C0DD00D4681
:104EA00000290AD0204610300121FEF740FCA968F5
:104EB00020342046FEF73BFC304670BD70B50446FA
:104EC0000026F043002C0DD00D4600290AD02046C4
:104ED00010300121FEF740FCA96820342046FEF77F
:104EE0003BFC304670BD70B50024002814D0054648
:104EF000064610363046FEF781FC01280CD02846C5
:104F00002030FEF77BFC012806D02C683046FEF7E7
:104F100066FC0C2141436418204670BDF0B583B097
:104F200000250295019500281FD00C46064607462D
:104F300010373846FEF76AFC002816D1304620307C
:104F400002AA01AB2146FEF71DFC00280DD13568F1
:104F50003846FEF746FC0C214143B068029A10180F
:104F600068506D186C600198A860284603B0F0BDC9
:104F700070B505460C2058430024904211D2121AF5
:104F8000461829606860AE60EA602846103019460D
:104F9000FEF729FCE96820352846FEF724FC204668
:104FA00070BDE443204670BD04217046084204D021
:104FB000EFF30983EFF3088203E0EFF30883EFF3E5
:104FC00009829BB004A8F0C044464D4656465F4651
:104FD00008A8F0C01846F0C86846F0C018690C90E0
:104FE000202018440D9058690E9098690F90D86948
:104FF0001090EFF310801190EFF314801290094994
:1050000008681390084908681490084908681590C2
:1050100007490868169017931892704619906846C9
:105020000DF0CCFE04ED00E00CED00E010ED00E032
:1050300014ED00E0F0B581B0002917D005461C4EF4
:1050400000910C462F783A0930461A490FF0DCFFE0
:105050000F223A40701C17490FF0D6FF641EB61C91
:105060006D1C002CEED10098410000E0002110489A
:105070000D22425401220A430A2383540E4EF06843
:10508000022812D137690D4CE0198D1C08492A46B7
:10509000FBF74AF87A193261B068214605F046F804
:1050A00000203061F078401CF07001B0F0BDC046C7
:1050B000C03E0202657B0100FCA8010275AD010241
:1050C000F0B581B0032600243046214609F0C0FE29
:1050D00004252846214609F0BBFE01273046394603
:1050E0003A4609F07BFE30462146324609F0D8FEAA
:1050F000284639463A4609F071FE022128462246E2
:1051000009F0CEFE01B0F0BDF0B58BB00A900325DA
:10511000002101220992284609F060FE0427384642
:1051200009F044FE0A24204607F03CFC384609F00A
:105130004DFE284609F042FE08900526304607F04D
:1051400031FC384609F032FE204607F02BFC384689
:1051500009F03CFE284609F031FE0790304607F082
:1051600021FC384609F022FE204607F01BFC384699
:1051700009F02CFE284609F021FE0690304607F083
:1051800011FC384609F012FE204607F00BFC3846A9
:1051900009F01CFE284609F011FE0590304607F084
:1051A00001FC384609F002FE204607F0FBFB3846BA
:1051B00009F00CFE284609F001FE0490304607F085
:1051C000F1FB384609F0F2FD204607F0EBFB3846CC
:1051D00009F0FCFD2846019509F0F0FD03903046EA
:1051E000029607F0DFFB384609F0E0FD204607F0A5
:1051F000D9FB384609F0EAFD284609F0DFFD0546EF
:10520000304607F0CFFB384609F0D0FD204607F0C6
:10521000C9FB384609F0DAFD019E304609F0CEFDA3
:105220000446029807F0BEFB384609F0BFFD304641
:1052300009990A4609F0D2FD0799481E81410A469C
:105240000899481E8141480080188000069A511E26
:105250008A4151004018059A511E8A4180188000E9
:10526000049A511E8A4151004018039A511E8A41E6
:1052700080188000691E8D4169004018611E8C41B4
:1052800006190A98002803D0032009F08FFD02E0D8
:10529000032009F09BFD0A24204607F083FB042528
:1052A000284609F093FD204607F07CFB284609F0CC
:1052B0007DFDF0B20BB0F0BDF0B589B008900324CD
:1052C000002120460A4609F089FD0427384609F0E6
:1052D0006DFD0626304607F057FB384609F076FD8F
:1052E000204609F06BFD07900525284607F04CFB8A
:1052F000384609F05BFD304607F046FB384609F0BA
:1053000065FD204609F05AFD0690284607F03CFB53
:10531000384609F04BFD304607F036FB384609F0B9
:1053200055FD204609F04AFD0590284607F02CFB64
:10533000384609F03BFD304607F026FB384609F0B9
:1053400045FD204609F03AFD0490284607F01CFB75
:10535000384609F02BFD304607F016FB384609F0B9
:1053600035FD204609F02AFD0390284607F00CFB86
:10537000384609F01BFD304607F006FB384609F0B9
:1053800025FD204609F01AFD0290284607F0FCFA98
:10539000384609F00BFD304607F0F6FA384609F0BA
:1053A00015FD204609F00AFD0190284607F0ECFAA9
:1053B000384609F0FBFC304607F0E6FA384609F0BB
:1053C00005FD204609F0FAFC0646284607F0DCFAFF
:1053D000384609F0EBFC0898821E501E82410121DC
:1053E000204609F0FBFC0799481E8141069A501E91
:1053F000824150004018059A511E8A4191000818B8
:10540000049A511E8A41D1000818039A511E8A41FC
:1054100011010818029A511E8A4151010818019A77
:10542000511E8A4191010143701E8641F0010843DB
:10543000C0B209B0F0BD70B50446032001210A4690
:1054400009F0CCFC042009F0B1FC60B2002803D4C0
:10545000032009F0ABFC02E0032009F0B7FC0A25A9
:10546000284607F09FFA0426304609F0AFFC28468C
:1054700007F098FA304609F099FC284607F092FAAE
:10548000600603D4032009F091FC02E0032009F038
:105490009DFC0A25284607F085FA0426304609F0C7
:1054A00095FC284607F07EFA304609F07FFC284636
:1054B00007F078FAA00603D4032009F077FC02E095
:1054C000032009F083FC0A25284607F06BFA04261E
:1054D000304609F07BFC284607F064FA304609F0B4
:1054E00065FC284607F05EFAE00603D4032009F0C5
:1054F0005DFC02E0032009F069FC0A25284607F05C
:1055000051FA0426304609F061FC284607F04AFAB1
:10551000304609F04BFC284607F044FA200703D434
:10552000032009F043FC02E0032009F04FFC0A25A8
:10553000284607F037FA0426304609F047FC28468B
:1055400007F030FA304609F031FC284607F02AFA15
:10555000600703D4032009F029FC02E0032009F0CE
:1055600035FC0A25284607F01DFA0426304609F0C6
:105570002DFC284607F016FA304609F017FC28469D
:1055800007F010FAA00703D4032009F00FFC02E093
:10559000032009F01BFC0A25284607F003FA04261D
:1055A000304609F013FC284607F0FCF9304609F0B4
:1055B000FDFB284607F0F6F9E00703D1032009F0C8
:1055C000F5FB02E0032009F001FC0A24204607F065
:1055D000E9F90425284609F0F9FB204607F0E2F92D
:1055E000284609F0E3FB204607F0DCF970BD70B5F2
:1055F0000446042009F0DAFB60B2002803D403203B
:1056000009F0D4FB02E0032009F0E0FB0A2528465C
:1056100007F0BAF90426304609F0D8FB284607F00F
:10562000B3F9304609F0C2FB284607F0ADF9600631
:1056300003D4032009F0BAFB02E0032009F0C6FB03
:105640000A25284607F0A0F90426304609F0BEFBDB
:10565000284607F099F9304609F0A8FB284607F0DC
:1056600093F9A00603D4032009F0A0FB02E0032075
:1056700009F0ACFB0A25284607F086F904263046D7
:1056800009F0A4FB284607F07FF9304609F08EFBAD
:10569000284607F079F9E00603D4032009F086FBD9
:1056A00002E0032009F092FB0A25284607F06CF976
:1056B0000426304609F08AFB284607F065F9304693
:1056C00009F074FB284607F05FF9200703D4032094
:1056D00009F06CFB02E0032009F078FB0A2528465C
:1056E00007F052F90426304609F070FB284607F00F
:1056F0004BF9304609F05AFB284607F045F9600798
:1057000003D4032009F052FB02E0032009F05EFB02
:105710000A25284607F038F90426304609F056FBDA
:10572000284607F031F9304609F040FB284607F0DB
:105730002BF9A00703D4032009F038FB02E0032073
:1057400009F044FB0A25284607F01EF904263046D6
:1057500009F03CFB284607F017F9304609F026FB14
:10576000284607F011F9E00703D1032009F01EFBDA
:1057700002E0032009F02AFB0A24204607F004F97E
:105780000425284609F022FB204607F0FDF82846AC
:1057900009F00CFB204607F0F7F870BDB0B5032404
:1057A000012120460A4609F019FB204609F00EFBAC
:1057B0000425284609F00AFB204609F0F7FA0A20DA
:1057C00007F0F0F8284609F0F1FAB0BD70B50324EF
:1057D000012120460A4609F001FB0425284609F06C
:1057E000E5FA204609F0E2FA0A26304607F0DAF830
:1057F000284609F0EBFA204609F0E8FA304607F0AF
:10580000D1F870BDF0B581B00326002501243046E3
:105810002946224609F0E2FA304609F0D7FA0F2667
:10582000304607F0BFF8042009F0D0FA304607F000
:10583000B9F8032009F0C2FA002820D0681CFA2D1C
:105840000546F6D3032528462146224609F0C6FA26
:105850000426304609F0AAFA284609F0A7FA0A27D2
:10586000384607F09FF8304609F0B0FA284609F0AC
:10587000ADFA384607F096F8204601B0F0BD042096
:1058800009F094FA0024204601B0F0BDF0B581B0D3
:1058900003260025012430462946224609F09EFAB7
:1058A000304609F093FA0626304607F06DF80420DA
:1058B00009F08CFA304607F067F8032009F07EFA09
:1058C000002820D0681CFA2D0546F6D30426304661
:1058D00009F06CFA0325284609F068FA0A273846C9
:1058E00007F052F8304609F071FA284609F06EFACE
:1058F000384607F049F828462146224609F06EFA54
:10590000204601B0F0BD032001210024224609F009
:1059100065FA042009F04AFA204601B0F0BD000003
:10592000F0B583B01C460092019106460325284637
:1059300009F04CFA0427384609F048FA284609F0DD
:1059400035FA0A20029007F01FF8384609F02EFABF
:10595000FE203040FFF74BFEFFF798FF5C4988615F
:105960000198FFF744FEFFF791FF5949C8612846A7
:1059700009F02CFA384609F029FA284609F016FAF7
:10598000029807F001F8384609F010FA01200643A2
:105990003046FFF72CFEFFF779FF4D490862002CD7
:1059A00038D0E0B2FFF788FC009D2870042009F091
:1059B000FDF9012C1DD06F1C032009F0F7F90A2610
:1059C000304606F0E1FF0425284609F0FFF930468D
:1059D00006F0DAFF284609F0E9F9641EE0B2FFF7A5
:1059E0006BFC3870284609F0E1F97F1CA0B2012851
:1059F000E2D1032009F0EAF90A24204606F0C4FFA8
:105A00000425284609F0E2F9204606F0BDFF2846A5
:105A100009F0CCF90424204609F0C8F903252846EA
:105A200009F0C4F90A26304606F0AEFF204609F018
:105A3000CDF9284609F0CAF9304606F0A5FF03B0B3
:105A4000F0BDC046F0B583B000AC0EC407460324D9
:105A5000204609F0BBF90425284609F0B7F920468D
:105A600009F0A4F90A26304606F08EFF284609F010
:105A70009DF9FE2007403846FFF7B9FDFFF706FF06
:105A8000134FB8600098FFF7B2FDFFF7FFFEF86014
:105A90000198FFF7ACFDFFF7F9FE38610298FFF7B8
:105AA000A6FDFFF7F3FE7861284609F07FF920464E
:105AB00009F07CF9304606F067FF284609F086F9C0
:105AC000204609F083F9304606F05EFF03B0F0BDD2
:105AD00084A8010270B504464D4E3070012020406C
:105AE000707003D1032009F061F902E0032009F08E
:105AF0006DF90825284609F069F9284609F056F994
:105B0000A007C00F707003D1032009F04FF902E025
:105B1000032009F05BF90825284609F057F92846C3
:105B200009F044F96007C00F707003D1032009F039
:105B30003DF902E0032009F049F90825284609F05B
:105B400045F9284609F032F92007C00F707003D1DB
:105B5000032009F02BF902E0032009F037F90825AA
:105B6000284609F033F9284609F020F9E006C00F6D
:105B7000707003D1032009F019F902E0032009F045
:105B800025F90825284609F021F9284609F00EF9DB
:105B9000A006C00F707003D1032009F007F902E0DE
:105BA000032009F013F90825284609F00FF92846C3
:105BB00009F0FCF86006C00F707003D1032009F0F3
:105BC000F5F802E0032009F001F90825284609F05C
:105BD000FDF8284609F0EAF8E009707060B2002884
:105BE00003D4032009F0E2F802E0032009F0EEF804
:105BF0000824204609F0EAF8204609F0D7F80724DF
:105C0000204609F0E3F8204609F0D0F870BDC04600
:105C100080A80102F0B581B00CF0BEF9B54D29782D
:105C2000002800D1BFE000290CD1B3480124047042
:105C30002C70B248002101700EF040F82046214639
:105C400002F0C4FAAE4F00247C737C84AD4D2C600E
:105C5000AD480460AD480460AD4E3460BC6220467F
:105C60000FF0A0F9FEF7B4FE796E401AA9498842F8
:105C70000FD3788C3C307884FEF7AAFE7866052036
:105C8000002102F0A3FA38464C300121A24A06F066
:105C9000CBF8B87B63280ED3797B00290BD17C84A9
:105CA000012179732246FF231902B32A08D91A0465
:105CB000622808D908E07A8CFF231902B32AF6D8A3
:105CC0000A46622800D80A463260FDF70FF800281D
:105CD00030D192480078012801D00EF031FE00F05A
:105CE00041F9FEF779FEFDF79BFC04F0ADFA562072
:105CF0008B49085A012801D104F012FBF87B0028D7
:105D000003D00020F87303F035F80CF077F9002881
:105D100008D0FEF75DFEF86305F058F8F87B002820
:105D20000DD110E07D20C00006F027FE0CF066F9D2
:105D300000282AD005F04AF8F87B002803D000207C
:105D4000F87303F017F8FCF7D1FF002806D033688A
:105D500000200146024603F069F80DE033686B4805
:105D6000026869480168286803F060F860206C499F
:105D7000095A012900D1A5E0387C002800D16DE73F
:105D80000CF00AF900282FD068E701253D70FEF7D6
:105D90001FFEF863634805705A4D05F017F8F87B4D
:105DA0000028CCD1CFE7012921D100242C705C48F8
:105DB000C483514804705148012101700DF066FF01
:105DC0000920214602F002FA0C20214602F0FEF9D9
:105DD0000F20214602F0FAF90820214602F0F6F9D8
:105DE000534806F0D1FD02E001207874414D04F0E3
:105DF000EDFF60214A48425A012A0AD1002242524C
:105E0000BFF34F8F484849490160BFF34F8F00BF30
:105E1000FDE70188474A914262D1C08800285FD0DF
:105E2000FEF7DAFD364CA07C01280ED13549002062
:105E30000860A07434490860344908603449086037
:105E400001460246034602F0F1FFA07B00280FD175
:105E5000A87800280CD0E07C002809D00120E07050
:105E6000FF2004302080FEF7B3FD20640020A870DE
:105E7000E078002824D023492F4808602249086090
:105E8000224908602249086001460246034602F0A2
:105E9000CDFFFEF79DFD216C401A042810D3092088
:105EA0000024214602F092F90C20214602F08EF9DE
:105EB0000F20214602F08AF90820214602F086F9D7
:105EC00001B0F0BD0021164A11520CF0FBFABFF3ED
:105ED0004F8F154815490160BFF34F8F00BFFDE795
:105EE000BFF34F8F104811490160BFF34F8F00BFC0
:105EF000FDE7C0461CA0010218A0010219A0010282
:105F000058AB0102F85B0202843D0202D83802025B
:105F1000743D02025902000001BD0000243D02024E
:105F200002C30102FDA801020CED00E00400FA0525
:105F300040420F00AA550000FFFFFF000248C06862
:105F4000811E484248417047FCA8010280B5FBF71A
:105F500093FA002801D00020C04380BD80B5FCF733
:105F600043FB80BD10B504480F2100242246FDF7F5
:105F7000D3FC204610BDC0462CAD0102B0B50724AD
:105F800000252046294608F063FF012120462A46C5
:105F900008F024FF022120462A4608F081FFB0BD08
:105FA000F0B581B0009003240127204639463A46D7
:105FB00008F014FF204608F009FF0425284608F0E1
:105FC00005FF204608F0F2FE0A26304606F0EAFCFD
:105FD000284608F0EBFE3220FFF72DFAFFF712FCFF
:105FE0000098C0B2FFF727FAFFF70CFC20463946AD
:105FF0003A4608F0F3FE204608F0E8FE284608F08E
:10600000E5FE204608F0D2FE304606F0CBFC2846DE
:1060100008F0CCFE3320FFF70EFAFFF7F3FB002069
:10602000FFF772F80090204639463A4608F0D6FE4F
:10603000284608F0BBFE204608F0B8FE304606F0C1
:10604000B1FC284608F0C2FE204608F0BFFE3046EC
:1060500006F0A8FC009801B0F0BDF0B583B0029145
:10606000019003240127204639463A4608F0B6FE3F
:10607000204608F0ABFE0426304608F0A7FE204676
:1060800008F094FE0A25284606F08CFC304608F0FD
:106090008DFE3220FFF7CFF9FFF7B4FB0198C0B2B5
:1060A000FFF7C9F9FFF7AEFB0298FFF7C4F9FFF756
:1060B000A9FB204639463A4608F090FE304608F0E3
:1060C00075FE204608F072FE284606F06BFC30464E
:1060D00008F07CFE204608F079FE284606F062FCB7
:1060E000284606F05FFC03B0F0BD000080B507480D
:1060F00001210170064802680A43026005480268EF
:10610000002A02D000200146904780BDDE380202FE
:106110001C100050E0380202F0B599B0F548017B40
:10612000C67A427B0E92F44C221F1368F34A12681F
:10613000069242780C9202790592C76A04931F4036
:1061400001200F907A0200D5BCE03A0200D5BFE0F2
:10615000FA0102D50F9802062260502508968A1986
:106160001826BB0102D50F984306236041230795EB
:1061700069430A96354655431426FC0210D50F98FC
:10618000040538463746DC4E3460DA4CA469B46402
:10619000D84CE4697464DA4C241D34603E460746EA
:1061A00090000B90D8040D90681809900E9B7343D3
:1061B0000F988203B902D04D22D50F98410529606E
:1061C000CC480E961646024681692965C169696503
:1061D00009990D9801430898000108180B99401877
:1061E000C018C849098892794A4380180A301C4669
:1061F00007F080F9234632460E9EC04988672A6020
:106200000F98C404380300D52C60F80302D50F980A
:10621000000428600F984104B80300D529603804B1
:1062200000D4E4E1039402910E9308920D980B9927
:106230000C180A980C9941430C910F98C0030B90CD
:1062400028600AF07DF9002801D007F035F90C9894
:10625000005B410B43D1099800190E99401805992C
:10626000090140180E90E74D287B079B4343E97ACC
:106270000A010D9C2243D21841188B00D2180A9BA8
:106280004B43D1186A7B564389190E9E2A79101800
:10629000DF4A12884243881816903068C000800D8B
:1062A00010A9C882002511957079C0077ED110A869
:1062B0000F998182069C00940020E8A2049B0DF0B7
:1062C000BFFB78E00F98820522603A0200D43FE7D6
:1062D0000F98C2052260FA0100D53BE73DE7072190
:1062E00049030840032149038842089A00D07EE10F
:1062F000069709F0B9FB0020169009901590C14C43
:10630000E07A217B08180A99414380000D9A1043D6
:106310004118627B0E9672438A186178A379079EB2
:106320007343D718FA683F26324063789A420C9735
:106330006ED105960A9A4A4380580F210A070240F7
:106340000398401EC04B1B68DB090340981810904F
:106350000F98C0020B90B868800767D42C46283C81
:106360000CF07EFA05462068000609D5C32084019A
:10637000786A400704D40CF073FA401BA042F7D9A6
:1063800005980002B96849080140B348036882686B
:10639000B868C40C20202040DB0700D095E0002323
:1063A00010221D461C460E9E0B9FB1E010A8858250
:1063B000B0681190069C701D924B1979E20707D1C5
:1063C000491C1971D97A1A798A4202D31D7100E0E9
:1063D000D970017842781202511882781204891813
:1063E00003229143017035715878401C5870D87A57
:1063F000197B08185978884200D85D70D879401EFA
:10640000D871596B002901D010A888477E4DEDE066
:1064100010A80B998182F8683040637800900020C2
:106420007CA20F990DF00CFB0E9E94E0388A874AEF
:10643000024010A8C2822022BA5C9307DB0F3C689E
:10644000C3720F9B1A4082726205D20C0D9B1A43D5
:106450001692FA68130E0372BB69FC697C4D2D68B5
:106460002D0C05745204920F427211931394654CD3
:10647000A07B002809980E9E0B9F5FD0754800688E
:10648000007A0328099859D00C98007D0840092803
:10649000099853D1C32084010CF0E2F905460C9809
:1064A000406A41070BD4594909680906890F06D18A
:1064B0000CF0D6F9401BA042F1D90C98406A410378
:1064C0000898884310A9888237E0D2070E9E0B9F58
:1064D00003D108230022154619E00C9B9A68029C00
:1064E000224211D19A68520C02249443002213468E
:1064F00015460DE0E83C020228A000503CA10050E7
:10650000FC1F0000E43C020204250022134614464E
:106510000843104318432843204310A98882384277
:106520000BD10C9B198A494A0A4010A9CA821968E2
:106530004905C90C0D9A11431691324C2921615C11
:10654000002908D03037B84205D010A908461130CC
:1065500012310BF0BFFBE77A2A48047BE519294882
:1065600000790E9027484078401C2946F9F7B2FD83
:1065700088000D9A10431890079961433801104321
:1065800040182049497B4E4380191C21694340181B
:106590000E9909191B4B1E4A12884A4380181790FE
:1065A000099A0C998A60987B002800D04A629879F1
:1065B000401C9871187B99798142069F00D39A718B
:1065C0005978491C5970D97A0818597888420E4D63
:1065D00000D85A70187A401E18722820185C0028BB
:1065E00004D0996B002901D010A88847089A174257
:1065F00002D00F98000328601C480449486019B075
:10660000F0BDC046E83C020228A000503CA100506A
:10661000E43C0202485720455420696478202564F0
:1066200020616E64204554206964782025642069C7
:106630006E2052582064657363206D69736D6174B8
:1066400063680D0A0000000038200040FF030000CE
:1066500094300040D4A60102604000404D414320E8
:106660004556542025782025780D0A00FFFFFF03AA
:10667000F0B5A5B01E460C9208910024239422A9DF
:106680000C8016A90C8024A909250D80598C0D9128
:10669000F9F720FD2A99012900D0DFE0318901298D
:1066A00000D0DBE0318C012900D0D7E00D99002922
:1066B00000D1D3E0224607962C990B912B99069195
:1066C00080B205900F9415A8058090000E900C994B
:1066D0000C582E460025204629461746FAF714F88E
:1066E0000028119636D12C200A977843089908186B
:1066F00017A90A4668C868C2E8C8E8C2E8C8E8C27C
:10670000079F119880B280000E5822AD019523A8F2
:10671000009020463946059A069B06F085F90F98A9
:10672000401C0F90288800282DD03B8A239913AC59
:10673000039416A8029014A8019015AE009617A80D
:1067400024AA06F033FD2588308811900120149E7C
:106750000A9A05E013A8058014952E4628463A4665
:106760000E9F51000B9B119C5C52591808830D849D
:10677000D81986600F981885521C0D9882426DD0EA
:1067800024A805889FE7099616A80025058014957A
:1067900024A80688239812902F46109503E06D1CBC
:1067A000A8B2B04213D8A8B2800017A90C5820464E
:1067B0001299F9F7B7FF0028F1D1002FEFD115A8F2
:1067C000058016A80127078014941094E7E715A800
:1067D0000288B01A012805D115A80680099F1497D0
:1067E000119628E010200799095E0129119221DBFA
:1067F000551CA8B20C18109F0E9B099403E06D1C49
:10680000A8B2844218DDAAB2B242F8D8800017AA12
:1068100010581090394634461E46F9F775FF334636
:106820002646099C0028EAD115A80580109F1497D8
:106830001195E4E7109F0E9B1C463E463846129980
:10684000F9F791FDF9F7F2FF0546052800D3052574
:1068500013A8058001200A9A274682E725B0F0BDDB
:10686000F0B58BB00243159A149C139E2BD00546AD
:1068700001A856C0129CD869196A09900A911E464F
:106880009F6B0123009309A807AA0146059308F00E
:106890002DFB716C3846F9F766FD0746E06A616BBF
:1068A000F9F761FD002D069613D004461198019961
:1068B000012924D10921081A0421069A515E88422F
:1068C00029D16425B1E000203080207010700BB019
:1068D000F0BDB08800226425002829D005926949BE
:1068E0003846F9F73BFF0028049C039E6FD16649A8
:1068F0003846F9F733FF00281DD05A2567E03C25BC
:10690000082800D191E05F492046F9F727FF0028C9
:1069100019D0502589E00A291DDB1D293BDC594986
:106920003846F9F71BFF0022002854D05A253AE0D8
:106930003346049C39E055493846F9F70FFF0028E3
:1069400021D0502543E050492046F9F707FF0028A1
:106950002ED0462569E03C25012866D049492046CD
:10696000F9F7FCFE0028D4D147492046F9F7F6FE96
:106970000028EED145492046F9F7F0FE002854D111
:10698000434920466EE042493846F9F7E7FE0028C1
:106990001CD128251BE03B493846F9F7DFFE0022D1
:1069A000002832D05025049C069B0299039E41E0AA
:1069B00036492046F9F7D2FE002836D13449204620
:1069C000F9F7CCFE00282FD114252EE037250299A7
:1069D000059A069B2EE005922B493846F9F7BEFE34
:1069E000002896D129493846F9F7B8FE0028B0D1D9
:1069F00027493846F9F7B2FE0028049C069B029905
:106A0000039E059A3BD11E2514E005921E49384687
:106A1000F9F7A4FE00289CD11C493846F9F79EFEE0
:106A200000281DD03C2500E02325049C069B0299EC
:106A3000039E059A25803270002008703078002867
:106A40000CD118681349F9F77BFE002806D120887D
:106A5000102803D30F3820800BB0F0BD0BB0F0BD71
:106A60000B493846F9F77AFE0028049C069B0299E8
:106A7000039E059A01D11425DCE72325DAE72D25AD
:106A8000D8E7C046CDCCCC3DCDCC4C3DCDCCCC3CDC
:106A90000AD7233C0000204070B588B00C4606465B
:106AA0004088002820D0F9F797FE059005A804A992
:106AB00001252A4608F084FC3088B188081AF9F7C5
:106AC00080FE0390049903A807AA2B4608F038FC1F
:106AD0005249079D2846F9F741FE002808D0BF20FB
:106AE0000006206008B070BD0020206008B070BDB6
:106AF0004B492846F9F716FE002804D03F2000062F
:106B0000206008B070BD47492846F9F727FE0028E5
:106B100001D0002010E000212846F9F71FFE0028D0
:106B200001D0022008E040492846F9F717FE002866
:106B300001D0042000E0062001957F21C9050291C3
:106B400080003A49091801A806AA022308F0ACFB04
:106B50000698206008B070BDF0B587B00C460546B9
:106B60004768002638463146F9F706FE002802D06D
:106B7000266007B0F0BD049704A803A90126324699
:106B800008F01EFCA8682968F9F7A8FB0290039991
:106B900002A806AA334608F0D3FB2049069D2846E2
:106BA000F9F7DCFD002804D0BF200606266007B0F8
:106BB000F0BD1B492846F9F7B5FD002804D03F2059
:106BC0000606266007B0F0BD16492846F9F7C6FD4F
:106BD000002801D0002010E000212846F9F7BEFD72
:106BE000002801D0022008E00F492846F9F7B6FD39
:106BF000002801D0042000E0062000957F21C9056F
:106C00000191800009490918684605AA022308F085
:106C10004BFB059E266007B0F0BDC046CDCC0C3FB7
:106C2000295C0FBFCDCC4C3ECDCC4CBEDCA60102C6
:106C3000F0B587B00C4606467F270088002801D0B3
:106C4000FD0503E0B08800282ED0334DF9F7C4FDD0
:106C500003907088F9F7C0FD049003A802A90126EB
:106C6000324608F0ADFB029904A806AA334608F0A4
:106C700067FB2A49069E3046F9F770FD002802D0CE
:106C80003F20010641E026493046F9F74BFD002838
:106C900002D0BF20010638E022493046F9F75EFDF8
:106CA000002805D0002024E00020206007B0F0BDBF
:106CB0001D493046F9F752FD002801D0022018E0A6
:106CC0001A493046F9F74AFD002801D0042010E0A7
:106CD00017493046F9F742FD002801D0062008E0A8
:106CE00014493046F9F73AFD002801D0082000E0A9
:106CF0000A200096F905019180000F49091868469D
:106D000005AA022308F0D0FA05992846F9F7EEFA09
:106D1000206007B0F0BDC046000080BF00003843CF
:106D20003333733F0000C84200007042000020422D
:106D30000000A0410000C040FCA60102F0B59DB0DB
:106D400015460B917F210391C9051C9102911B915E
:106D500019A900248C80199418941794598C0691C1
:106D6000198C0F91DE8B998B0791997805911F886B
:106D70002B21CA432799914201DB7F0015E0402275
:106D8000D243914211DC4922D243914202DB79087D
:106D9000CF190AE05322D2439142EEDA5D22D24368
:106DA000914201DBBF0000E0FF000A971396269E88
:106DB000597E00290BD0002132460F46D1709170C8
:106DC00051701170121D7F1C5C7EA742F6D30C938C
:106DD00011952599149122990D91159041088C4295
:106DE00011D2FD4A2346A00084583454270A451C7A
:106DF0007755250C871CF555240EC01C34545B1C9C
:106E00009CB2A142EFD823981090012009900090E5
:106E100030463146149A159F3B4608F075F80D9898
:106E200000060890400E139D00D186E06800049093
:106E3000002F3FD0002210461146144606E01C46A3
:106E40001146159F401C82B2BA420ED283B2AB42A9
:106E5000F8D09200149B9A5E0FB2BA42034600DC4F
:106E60002346BA42EBDC0A46E9E7002F25D0002290
:106E700010461146129206E012931146159F401CCF
:106E800082B2BA4214D283B2AB42F8D0A5B2AB42BE
:106E90000CD09200149B9A5E0FB2BA42034600DCFB
:106EA000129BBA42139DE7DC0A46E5E7139DE6E72D
:106EB000129903E00024214600E00021129110986D
:106EC0000183C4828582049FF057F9F77AFC792107
:106ED000C9050E91F9F70AFA1099C8610998074394
:106EE000F057F9F76EFC0E99F9F700FA109F386227
:106EF0002004C40B3057F9F764FC0E99F9F7F6F942
:106F00007862601C3056F9F75CFC0E9C2146F9F75C
:106F1000EDF9B86212980004C70BF057F9F751FC6D
:106F20002146F9F7E3F9109CE062781C3056F9F736
:106F300048FC0E99F9F7DAF92063119805800C984E
:106F4000407E410000278D4228463A46149E1ED3BB
:106F50000A9880B28AB29300F45E84420BDA491C2C
:106F60008AB2AA42F6D9002728463A4681B2691A5F
:106F7000012910D01BE0F018119B19800788080424
:106F80000FD0500040008019001F0288084681B2CF
:106F9000691A01290BD1A800301811990D800788B2
:106FA00026E00020024681B2691A0129F3D00A992D
:106FB00089B2079B4B43BB421AD306998A4217D822
:106FC0000599002914D0401C82B2891803E0401CA6
:106FD00082B291420CD983B2AB42F8D89200B35E30
:106FE000BCB2A342F3DDB218119B18801788EEE7FC
:106FF00012970B980580119800882B1A002B16DD2C
:1070000002210F9A1143032942D10E93411C421EC3
:1070100010B281420EDA0E98032824DB0C98808C83
:10702000012820D019A818A9FFF736FD1FE000207D
:1070300018902BE00026F443374608E0B8B2400031
:1070400019AD2B527F1C521C10B28142E3DB13B2EC
:10705000A3423346F2DD159B98423346EEDA8000B8
:10706000149B1B5AEAE719A818A9FFF7E1FD149E23
:10707000139D0F9A012A13D0032A11D0022A04D19A
:1070800011980088281A02280ADA0020179034E0A4
:10709000022A01D1022BB8DA00201890012AEBD184
:1070A000681C691E0FB2B84208DA0C98808C01285F
:1070B0001DD119A817A9FFF7BBFD1CE00022D3437F
:1070C000144608E0A5B26D0019AF7E53641C491C3C
:1070D0000FB2B842E9DB0DB29D421646F2DD159DB6
:1070E000AF421646EEDABD00149E765BEAE719A8B9
:1070F00017A9FFF7D1FC149E139D249F189C179984
:107100002046F9F7EBF80F99012900D8204638609E
:107110000D98002800D1CBE011990888109FB886FF
:107120000888281AB880129880B2F9F755FB79219F
:10713000CC052146F9F7DAF82146F9F7D7F8B86314
:10714000119F3888002849D081008919091F0988B2
:10715000129C0C191599884203D2800080198088EE
:10716000041915984300534916AA304608F0AAF8A6
:10717000169810994864F9F772FBA4B2A04201D1A5
:107180004D480FE0001BF9F727FB1C901CA81BA91A
:10719000012208F015F92046F9F71EFB01461B985D
:1071A000F9F7A4F8109908603988491B4A1C92B273
:1071B000032A02D20021159F17E009B20229159F68
:1071C00012DB3F210906F9F7C9FA002802990CD110
:1071D0000998810709E0C046402100400020129C28
:1071E00015998842B9D3BCE73449109801610898D1
:1071F000800E5DD0002F1CD0002211461446104690
:107200004B1B1DB2ED135B196B40139D1BB292001B
:10721000B25E53431818A418491C8AB2BA42EFD37D
:10722000F9F7DAFA06462046F9F7D6FA002C03D128
:1072300000E000260398C0051C901CA81BA901258E
:107240002A4608F0BDF81B9C20463146F9F74EF857
:10725000014610988160002F119422D00024274607
:10726000264613951291B8B2F9F7B6FA1299F9F7C2
:1072700035F80546A0001499085EF9F7A2FA014610
:107280001398C00785432846F9F730F80146304681
:10729000F8F7D3FF06467F1CBCB215988442E2D3B0
:1072A00000E0002611983146F9F720F81099C860DF
:1072B0001DB0F0BD00C101020000204100004040AF
:1072C000F0B58FB00692F74A09AF70CA70C770CA9E
:1072D00070C70328079320D88800F3A10858F649FF
:1072E000F8F7ABFF0446F549F8F7A7FF0D90F4490E
:1072F0002046F8F7A2FF0C90F2492046F8F79DFFD0
:107300000B90F1492046F8F798FF0A90EF49204684
:10731000F8F793FF0990EE4969E0042822D0062887
:1073200020D88800EBA10858EE49F8F786FF0446FC
:10733000ED49F8F782FF0D90EC492046F8F77DFF04
:107340000C90EB492046F8F778FF0B90E94920466E
:10735000F8F773FF0A90E8492046F8F76EFF0990A6
:10736000FD4944E00838022821D88800FBA10858CC
:10737000D149F8F762FF0446FC49F8F75EFF0D902B
:10738000FB492046F8F759FF0C90FF208105204665
:10739000F8F753FF0B90F7492046F8F74EFF0A9095
:1073A000CA492046F8F749FF0990FE491FE08800C6
:1073B000F1A10858F449F8F740FF0446F349F8F7FB
:1073C0003CFF0D90F2492046F8F737FF0C90F14949
:1073D0002046F8F732FF0B90EF492046F8F72DFFD3
:1073E0000A90EE492046F8F728FF0990EC490094EE
:1073F0002046F8F722FFEC4909680E90EB48046834
:10740000EB4801684808EB4F05463D400022002D3F
:1074100008922DD0CA01120E07D0280CE90D12D106
:107420004000E649085AE6490AE0C903090E0CD0B3
:10743000280AE90B10D14000E049085A8F21890041
:107440004018E4300DE0DC490AE081B27F2905D81C
:107450004800DA49085A04E0D94901E08F2189003F
:10746000401800B2F9F7ADF9D649F8F73FFF0246E8
:107470000292039507252606D34B1A68002A08981E
:1074800040D0791C8A420BD21102090E13D0110C84
:107490001F46D00D1FD14800C849085AC84907E007
:1074A0001F46110E002A13D44800C449085AC24985
:1074B0004018E4301FE011041F46090E0ED0110AD7
:1074C000D00B12D14800BD49085A8F218900EFE73F
:1074D000BE4808180FE0B84808180CE091B27F29A0
:1074E00006D84800B549085A05E0B548081802E032
:1074F0008F218900501800B2F9F763F9B149F8F704
:10750000F5FE3B460590159F2C40F50E5B69B04992
:107510001940089810D0DA02D20E34D0C80B3E21A0
:107520000140A648405AA6494018E43000B2F9F795
:1075300048F9A449F8F7DAFE0490149E6800A5A162
:10754000085EF9F73EF90146A00009AA1058F8F7BD
:1075500074FE0146B8B20128089F019102D1022CA5
:107560000AD9A74F052C24D1189808900C2D20D8A3
:107570000B2D16D3A44918E00027022C089718D029
:107580008120C70515E01A04120E00D1CAE0080ACE
:10759000C90B00D0CDE040008849085A8F218900EE
:1075A000C2E7092D00D2C7E096490898F8F745FED2
:1075B000089001200021B542034600D30B46052C5C
:1075C00000D308461799169A1A9C199D1843069BD2
:1075D000012B12D1079B402B22D1002840D03846E6
:1075E000F8F72BFE01460198F8F727FE01460098B0
:1075F000F8F774FE059A04998AE0079B402B1FD187
:10760000002838D03846F8F718FE01460198F8F7F8
:1076100014FE01460098F8F761FE059A049977E098
:10762000002833D03846F8F708FE01460198F8F7ED
:1076300004FE01460098F8F751FE059A049967E0A8
:1076400000285BD03846F8F7F8FD01460198F8F7B6
:10765000F4FD01460098F8F741FE059A049957E0B9
:1076600002981146F8F73AFE0399002900D16748BD
:10767000059A04994CE002981146F8F72FFE0399F9
:10768000002900D16148059A049941E00298114609
:10769000F8F724FE0399002900D15C48059A049963
:1076A00036E0C0469C660100000068C1000088C149
:1076B00066665EC1000084C1000084410000B441E0
:1076C00000004841000020400000F0C0000084C1DC
:1076D0000000F841333323C1000050C19A9929C1F9
:1076E0009A9949C19A9949413333CB4166667641AB
:1076F000CDCCAC40333393C09A9949C1029811461E
:10770000F8F7ECFD0399002900D14048059A049947
:1077100028601046F8F7E2FD0899F8F7DFFD2060D1
:107720000FB0F0BD99B27F2911D848002349085AFB
:10773000FCE623494018F9E6C12001060898F8F74D
:107740007CFD0890062D00D933E7002030E78F211B
:1077500089005818EAE6C0463333F341000058C1A7
:107760009A9961C19A9969C1000084C10000AC4135
:1077700000003841000008C1CDCC80C1CDCC88C10B
:1077800033338FC1333397C133339741CDCC8C41E1
:107790003333F3409A9919C0666646C1333397C1B3
:1077A000CDCCB4410000D4410C000040503000402A
:1077B00068400040FFFFFF007C080000806B010074
:1077C0005C050000919AF63C642000409C0B000090
:1077D000FFFF1F00FAFFFCFFFEFF00000200040095
:1077E000060008000A000C000E0010001200140031
:1077F000160018001A001C001E00200022002400A1
:10780000000080BF0000A0C0000040C00000DCC23B
:10781000F0B5FFB0ECB017460E460D900021E9918F
:10782000E891DC9199919891979196911491139187
:1078300012919AA8F49DF39CF29A002E00D1E6E1F1
:107840000B938030F09B1180099529602546DBACB5
:10785000218095AC21800C952980DA917F24E40564
:10786000B994B894B794B694B594B494B394B294CC
:10787000B194B094AF94AE94AD94AC94AB94AA94FC
:10788000A994A894A794A694A594A494A394A2942C
:10789000A194A0949F949E949D949C949B949A945C
:1078A000046644668466C466046744678467C46784
:1078B000046444648464C464046544658465C46584
:1078C000046244628462C462046344638463C46384
:1078D000046044608460C460046144618461C46184
:1078E000B0090B250B2800D3AE011095012B0B9D81
:1078F00000D070E12B89012B00D06CE1298C00298C
:107900000E9200D18BE16B8C002B00D1FAE1AA8C96
:107910003021695C002900D188E10892109F5F4303
:107920001196304639460F93F8F7D4FB0590F8F7D7
:1079300048FF01462046F8F716FD8321C905F8F7F0
:10794000D5FC064696A8021D119887420A9200D8D7
:1079500079E155A811909AA9069196AF15463A4635
:10796000059C234607F0A0FC15A80F9006992A460F
:10797000234607F099FC02230D93384631463A46D8
:1079800007F0DEFC012308930093E8AA1092384622
:10799000394607F0ABFAE898DD901198069D294624
:1079A0003A46234607F080FC0F9829460A9A234658
:1079B00007F07AFC384631463A460D9B07F0C0FC8A
:1079C000089B009338463946109A07F08FFAE898DA
:1079D000DE9011982C4629463A46059D2B4607F025
:1079E00063FC0F9821460A9A2C462B4607F05CFC54
:1079F000384631463A460D9B07F0A2FC089B00939F
:107A000038463946109A07F071FAE898DF901198D5
:107A1000069D29463A46234607F046FC0F9829461C
:107A20000A9A2346254607F03FFC384631463A4637
:107A30000D9B07F085FC089B009338463946109A49
:107A400007F054FAE898E0901198069C21463A46CF
:107A50002B4607F029FC0F9821460A9A2C462B4604
:107A600007F022FC384631463A460D9B07F068FC89
:107A7000089B009338463946109A07F037FAE89881
:107A8000E1901198069D29463A46234607F00CFCE2
:107A90000F9829460A9A2346254607F005FC3846E2
:107AA00031463A460D9B07F04BFC089B0093384645
:107AB0003946109A07F01AFAE898E2901198069C55
:107AC00021463A462B4607F0EFFB0F9821460A9ACB
:107AD0002B4607F0E9FB384631463A460D9B07F046
:107AE0002FFC089B009338463946109A07F0FEF9A0
:107AF000E898E390119821463A462B4607F0D4FBCC
:107B00000F9821460A9A2B462C4607F0CDFB3846A3
:107B100031463A460D9B07F013FC089B009338460C
:107B20003946109A07F0E2F9E898E4901198069D1A
:107B300029463A46234607F0B7FB0F9829460A9A8A
:107B40002546234607F0B0FB384631463A460D9BA2
:107B500007F0F6FB089B009338463946109A07F069
:107B6000C5F9E898E5901198069C21463A462B46BF
:107B700007F09AFB0F9821460A9A2B4607F094FBD0
:107B8000384631463A460D9B07F0DAFB089B0093D6
:107B900038463946109A07F0A9F9E898E690119806
:107BA00021463A462B4607F07FFB0F9821460A9A5A
:107BB0002B4607F079FB384631463A460D9B07F0D5
:107BC000BFFB089B009338463946109A07F08EF9A0
:107BD000E898E7907AE010880C9A10809991989133
:107BE000DA9E08460F46099DF59CF8F777FB28605A
:107BF000DC9827606060A6600C34DDA80EC80EC457
:107C00002EC82EC42EC82EC47FB06CB0F0BDFF208D
:107C100010800021296020807FB06CB0F0BD002270
:107C200001233021695C002900D076E6DDAA1ACF55
:107C30001AC23ACF3AC23ACF3AC20B213046F8F7CD
:107C400049FA054642E000200690059D0796089FE8
:107C50001190069801460D9C0F9A4A43D219109B29
:107C60005A43119BD218D200A35889002E4655AD15
:107C70006B503546121DA25815AB5A50401C01B22C
:107C80008E42E9DC55A89AAE96AC314622462B4688
:107C900007F00AFB15A831460A9A2B4607F004FBA9
:107CA000022320460799224607F04AFB012300934E
:107CB000E8AA2046214607F019F9119B9800DDA992
:107CC000E89A0A505B1C0B2B1846C1D1F19EDDA827
:107CD0009AA9DCAA0B2307F0E7FA09210E980F9165
:107CE00001800B98C168DC9C2046F8F7FFFA01463A
:107CF000A8B2E69F0F281BD808280DD30846F8F72E
:107D00009CFA14E0FF2010800021099A11600C9960
:107D100008807FB06CB0F0BD042803D381220846F0
:107D2000D10502E0412208461106F8F7DFFA0146C4
:107D30002B20C04386420D9704DB0846F8F77DFAF6
:107D4000014603E04020C043864244DD0E9A0C9C6D
:107D50000B98408A002811D00B98038A95A80390AD
:107D6000DBA80290DAA801900094DDA80D4605F08A
:107D70001DFA29462488DA9E099D68E011910F9822
:107D8000208000273D46109705E00E9804887F1C50
:107D9000B8B2A04211D8B8B28000DDA90C58204674
:107DA0001199F8F7BFFC0028EFD1002DEDD10C9808
:107DB000078001250F971094E7E7DBA805800F9A4D
:107DC00090B2201A012811D10C9804800D9FDA97E7
:107DD0003E46099D3AE04920C043864200DA8BE0E6
:107DE000FF2208469105F8F781FAA9E710200B99C0
:107DF0000E5E012E00DA90E0551CABB21846A1B21F
:107E0000AAB28A4217D805E00E990C88A1B2AAB28C
:107E10008A4210D88000DDA90C58204610991F46D0
:107E2000F8F772FC3B46002805D10C9805800B98AA
:107E3000068A0F95109430B2C1186D1CA8B2814209
:107E4000E2DC109EDA960F9C099D0D9F1199304639
:107E5000F8F789FAF8F7EAFC052800D3052095A978
:107E60000880A0B20E990988814218D9401C611E71
:107E70000CB2A04218DA12A898A9FEF76DFE0E986F
:107E80000188481C491E0CB2A04221DA12A899A907
:107E9000FEF762FE99999898099D0D9FA4E600212E
:107EA0009891999108469FE60022134608E09CB2FB
:107EB000A40012AF3D515B1C491C0CB2A042DADB9E
:107EC0008DB20A2D1546F2D8A400DDAD2D59EEE78E
:107ED0000022134608E09CB2A40012AF3D515B1C87
:107EE000491C0CB2A042D1DB8DB20A2D1546F2D846
:107EF000A400DDAD2D59EEE75320C043864200DBE0
:107F00001BE70E460B9881692046F8F7FDFB002819
:107F10000C9C08D10B98808B07E01446099D0D9F9F
:107F20001199109E93E70B98C08BF8F755FC01460A
:107F30003046F8F7DBF9119021E70000F0B58BB07F
:107F40001C4609930E46034600200A9040480088CC
:107F5000224F05970AA9049103940292109C019460
:107F6000012500950B21414389B230331C4A30462C
:107F7000FFF74EFC3868079078680890B86806905C
:107F800033480088334F009501940297324E3036C3
:107F90003249334A3346FEF76BFB0698F86207987E
:107FA000386308987863099800882E4905912E490E
:107FB00004912E4903910297019000962C4B28467C
:107FC00029462A46FEF74CFC432001060A98F8F79A
:107FD0008DF9F8F72BFC0BB0F0BDC046C8C001020C
:107FE00008520202F0B589B00F9F0E9C002815D0F0
:107FF0001098079016480088164E012500950191AB
:1080000002960893144B30331449154AFEF730FB9F
:10801000089BF76207983063746303E00D48476379
:10802000C462002518880F4905910F4904910F4932
:1080300003910849029101900748303000900121D6
:108040000B4B28460A46FEF70BFC09B0F0BDC046B4
:108050006CC70102CC46020230BA010280B90102AB
:10806000283D0202F8BD010268C7010208C70102EB
:1080700010C701022C487047364870474048704787
:108080001D487047800048490918C86B0022CA6320
:108090007047C046800044490918886C00228A64F1
:1080A0007047C04680B5404AD369002B01D0126AA0
:1080B0009847002080BDC04680003B490918002039
:1080C00088640122CA63704780003749091800207C
:1080D000C86301228A64704710B50024002809D0C3
:1080E000024609480121017003488021FCF764FE23
:1080F000204610BDE04310BDACC70102024908781C
:1081000000220A707047C046142F020200207047F8
:1081100080B5182905D803468A1E03481946F8F782
:1081200003F8002080BDC04670C70102B0B502460A
:108130000020022901D2C043B0BD8C1E0F2C07D8ED
:10814000044D284611462246F7F7EEFF0020285539
:10815000B0BDC0468CC70102B0B50246002002295E
:1081600001D2C043B0BD8C1E0F2C07D8044D284649
:1081700011462246F7F7D8FF00202855B0BDC0466B
:108180009CC701020849087800220A707047C0465F
:10819000B0B50446044DAA68002A02D0E96820461A
:1081A00090472C610020B0BD1CAA010280B5054893
:1081B0000268002001460CF0EBFD034948720120E3
:1081C000087280BD44A00102E0AA0102F0B581B0AE
:1081D000431E0F2B28D8082809D82420B24A145C43
:1081E00001259D4000290CD02C4314540EE025227B
:1081F000AD4B9C5C093801258540002904D02C43F7
:1082000003E0AC43145401E0AC439C542426A64F35
:10821000BC5D24377D784020022122462B46FDF7A5
:1082200011FCA14884557D7001B0F0BDF0B58DB052
:108230009D4C21462E310B914878BF2606404E704A
:108240002E20275C05460C9040200A9006210791BD
:108250003A463346FDF7F6FB67550B9846702146C4
:10826000243108914E780A9806434E702425675DA4
:108270000995022106913A463346FDF7E3FB67551F
:10828000089846700B994878DF2606404E700C9D82
:10829000625D05920A9F384607993346FDF7D2FB87
:1082A000059860550B9846700898467820210391F0
:1082B0000E434670099D625D38460699174633465F
:1082C000FDF7C0FB67550C99605CEF2707406754CA
:1082D000089D6E700B98407805900A9E304607996D
:1082E0003A46059BFDF7AEFB0C9827540999675C4D
:1082F00010200490074367540B98059941706D78DE
:10830000304606993A462B46FDF79CFB09982754C0
:108310000C99675CFE2002900740675408984570EE
:108320000B9E707805900A9D284607993A46059B52
:10833000FDF788FB0C9827540998275C01210191CF
:108340000F43275405987070089E73782846069945
:108350003A461D46FDF776FB099827540C99675C51
:1083600003980743675475700B9846780A98079DE1
:1083700029463A463346FDF765FB0C982754029888
:1083800006400B9846700A9829463A463346FDF750
:1083900059FB0C9827540B98467008984678019919
:1083A0000E434670099D675D0A9806993A46334622
:1083B000FDF748FB67550C99605C7F2707406754C1
:1083C000089846700B9846780A9D284607993A46C1
:1083D0003346FDF737FB0C9827540999605C8027DA
:1083E000074367540B984670089E73782846069991
:1083F0003A461D46FDF726FB099827540C99675C01
:108400000A980743675475700B994E78079D294663
:108410003A463346FDF716FB0C982754049806435A
:108420000B9846700A9829463A463346FDF70AFBF0
:108430000C982754F72535400B9E75700A980799BC
:108440003A462B46FDF7FEFA0C98275475700899AA
:108450004878082505434D700998265C0A9F3846E0
:10846000069932462B46FDF7EDFA099826540898EE
:1084700045700B994878042505434D700C98265C8F
:108480003846079932462B46FDF7DCFA0C982654FD
:108490000B9845703834002138462246069BFDF77C
:1084A0003FFA0DB0F0BDC04684A8010280B50A466F
:1084B00000210223FDF734FA80BD000080B5124888
:1084C00001681F220A40026003200840022812D1DE
:1084D0000E480268D30D02D0FF231B06D2180C4BA6
:1084E0001A600C4A12680C4B1A6080680B4A1080A4
:1084F000000C0B4A10801A488268002A02D0826859
:108500000020904780BDC046742000406440004079
:108510003C3D020278300040403D020294BA010224
:10852000C046020280B50D48016889070FD50521B4
:1085300001600B48C178002908D00021C170C168D2
:10854000002903D0C26841680020904780BD0548DB
:1085500005A10B4A0BA30AF017FAC0462C040040F1
:10856000C4A601027B8701005048595F54494D451C
:10857000525F49525148616E646C657200000000A0
:108580008D0A0000556E65787065637465642069B6
:108590006E746572727570740000000070B50446E8
:1085A000401E012814D80320084011D13F20400369
:1085B0000818050B281980280AD8164E3178012092
:1085C0004840294605F01CFE641E6D1C002CF5D1A8
:1085D00070BDC04680B50020014605F035FB00287F
:1085E00000D080BD0B480121017080BD70B51646DA
:1085F0000C460546FF22F7F7A9FD05483118054846
:108600000278012050402A46234605F0A1FC70BDA7
:1086100000E0070400C301020120000370470120AD
:108620004003704710B509F0DBFC002820D07D2402
:10863000E00004F0A2F909F0D3FC002820D0114991
:108640001148086011490860114908601149086023
:1086500001460246034600F0E9FBA00004F08DF954
:10866000834C0120E070812040002080403404E0F1
:10867000FCF7AEF97E4C60644834FCF7A9F9206041
:1086800010BDC046F85B0202FFFFFF00843D0202FE
:10869000D8380202743D0202F0B587B071487249C1
:1086A000016007F05BFE714F0A203884BD88704E70
:1086B0003583B87AF072B8897083B88AB083F98A42
:1086C000F1836C4A51831083BC8D148195807D2089
:1086D0000690C000F988F7F7FDFC30845420385A22
:1086E0005221795A09040A18E1204002824204D03A
:1086F0000321F165824204D105E00721F165824240
:1087000001D04B20C201788C02286DD2B88C02288F
:108710006FD20592388D0B2801D3012038850020B7
:10872000F8833220385C3073FF2018307880601E68
:1087300084416000306603264F4A304631462B465E
:108740000BF07EF97888C1B20091030A4B4A30469B
:1087500031460BF075F966203B5A6820385A6A2179
:10876000795A6C22BA5A6E243C5B00AD17C544A2FC
:10877000304631460BF064F9BB8C49A23046314695
:108780000BF05EF97B8C4BA2304631460BF058F96A
:108790003B8D4DA2304631460BF052F9FB8C50A276
:1087A000304631460BF04CF953A230463146059B1A
:1087B0000BF046F95620385A002821D0022825D03F
:1087C000012849D172203B5A7420385A7621795AAF
:1087D0007822BA5A7A243C5B00AD17C50320564A6A
:1087E00001460BF02DF937E001207884B88C02287F
:1087F0008FD30120B8840592388D0B288DD28EE757
:108800000320444A01460BF01BF925E00520C00176
:108810003B180324404A204621460BF011F915204D
:1088200040013B5A3D4A204621460BF009F93C489D
:108830003B183C4A204621460BF002F93A483B18C7
:108840003A4A204621460BF0FBF839483B18394A92
:10885000204621460BF0F4F80698800004F08DF8CD
:1088600007B0F0BD78B9010241B6000002C30102B1
:1088700058AB0102883E0202A97A0100717A010018
:10888000B7FECEF1C6F7B5D8D6B73A2025642E2567
:10889000642E25642E25643A25642E0D0A000000FE
:1088A000C9E8B1B8555742D7B4CCAC3A20257820A6
:1088B0002E0D0A00C9E8B1B8475053D7B4CCAC3A32
:1088C000202578202E0D0A00C9E8B1B8555742B9C5
:1088D000A4D7F7BCE4B8F43A202578202E0D0A007E
:1088E000C9E8B1B8475053B9A4D7F7BCE4B8F43AD3
:1088F000202578202E0D0A00B5B1C7B0475053B9D6
:10890000A4D7F7B2A8CCD8C2CA3A202564202E0D2D
:108910000A000000947A0100317B0100E37A010033
:10892000A20200001D7B0100C2020000F37A0100D8
:10893000E2020000077B0100B87A0100F0B583B0C5
:1089400030480068C16B0901890F01D003B0F0BD48
:10895000C16BC06B2C4D05404800400F08260296A5
:1089600086400227384603F0F3FE01907043C10BA6
:108970004A1B26485043F7F7C3FB044609F074FE30
:10898000032123A238461F4F009123460BF058F8CD
:10899000F88A002817D0019840012946F7F79AFB7A
:1089A00046431822324001200F2A014600D80021F8
:1089B00073095B181B4CA3420DD8194DED1A6D05B8
:1089C0000F2A0CD80CE038680021C160112003F098
:1089D000AFFE03B0F0BD5D1C6D050F2A00D95642F5
:1089E0002A0C029D2E4009018919A34202D8009841
:1089F000000400E04004081880183968086303B0D8
:108A0000F0BDC04654A70102FFFF1F0040420F0007
:108A100052434F33324B2070706D2025640D0A0095
:108A2000FF070000FE7F000070B52E494860172246
:108A30002D4B1EE01D68A5431D6000BF00BF00BF99
:108A400000BF00BF00BF00BF00BF00BF00BF00BF2E
:108A500000BF00BF00BF00BF00BF00BF00BF00BF1E
:108A600000BF00BF00BF00BF00BF00BF521E541CAC
:108A700036D20446D440012525400D701E6880245E
:108A800026431E6000BF00BF00BF00BF00BF00BF85
:108A900000BF00BF002DCDD000BF00BF00BF00BF92
:108AA00000BF00BF00BF00BF00BF00BF00BF00BFCE
:108AB00000BF00BF00BF00BF00BF00BF00BF00BFBE
:108AC00000BF00BF00BF00BF00BF00BF00BF00BFAE
:108AD00000BF00BF00BF00BF1D68A5431D60B3E716
:108AE00070BDC046C8A8010204200050B0B582B0D5
:108AF000154908688269D2070CD00122C2610D694C
:108B0000002D07D000686C46214609F01BFB0021B0
:108B10002046A84702B0B0BDB0B582B00A49086887
:108B2000026C92070ED5026C012313430364CD68D7
:108B3000002D07D000686C46214609F003FB002198
:108B40002046A84702B0B0BD54A7010206480168FC
:108B5000032291430160016801220A43026001F08F
:108B60004FFB09F0A7FDC0462800004080B50D4925
:108B70000868002810D5224802680423032A01D07F
:108B80001A4300E01A460A601E490A68002A02D009
:108B900041680020904780BD03A00CA19E2211A334
:108BA00009F0F2FE2C100140696E636C7564652F4C
:108BB000647269766572732F6D6B5F736C65657037
:108BC0005F74696D65722E6300000000534C45456B
:108BD000505F54494D45525F49525148616E646C33
:108BE00065720000556E6578706563746564207306
:108BF0006C65657020696E746572727570740000C2
:108C00000CA00102C846020270B50C46054640B2EF
:108C1000002803D40B2006F0C9F802E00B2006F070
:108C2000D5F80D26304606F0D1F8204603F0ACFE0C
:108C3000304606F0BBF8204603F0A6FE680603D4D3
:108C40000B2006F0B3F802E00B2006F0BFF80D266B
:108C5000304606F0BBF8204603F096FE304606F09C
:108C6000A5F8204603F090FEA80603D40B2006F0DA
:108C70009DF802E00B2006F0A9F80D26304606F01C
:108C8000A5F8204603F080FE304606F08FF8204617
:108C900003F07AFEE80603D40B2006F087F802E022
:108CA0000B2006F093F80D26304606F08FF820468C
:108CB00003F06AFE304606F079F8204603F064FEC1
:108CC000280703D40B2006F071F802E00B2006F011
:108CD0007DF80D26304606F079F8204603F054FE64
:108CE000304606F063F8204603F04EFE680703D4D2
:108CF0000B2006F05BF802E00B2006F067F80D266B
:108D0000304606F063F8204603F03EFE304606F09B
:108D10004DF8204603F038FEA80703D40B2006F0D8
:108D200045F802E00B2006F051F80D26304606F01B
:108D30004DF8204603F028FE304606F037F820466E
:108D400003F022FEE80703D10B2006F02FF802E023
:108D50000B2006F03BF80D25284606F037F8204694
:108D600003F012FE284606F021F8204603F00CFE20
:108D700070BD000010B51C4C2079411C2171792870
:108D80000DD3002121710520FFF720FA642003F0A4
:108D9000F4FD20464C300121144A03F045F8607977
:108DA000002812D1FDF7CAF8002804D0104800218D
:108DB0000170A17109E0A0791E2801D3002100E013
:108DC00001210B4A1170401CA071FBF741FE7F206E
:108DD000C105A06AF7F731FAA062FAF7C1FA642177
:108DE0004143E18210BDC04658AB010201BD000005
:108DF00048A30102B0B582B004460078002811D023
:108E0000094D01A908702868416A0029FCD101A90F
:108E10000122002003460BF0A5FB611C60780028AE
:108E20000C46EED102B0B0BDA0A70102F0B581B0F2
:108E30001C4615460E460746EFF3108072B6072013
:108E400005F0B4FFE120000100BF401EFCD1384610
:108E5000FFF7EAFD3046FFF7E7FD2846FFF7E4FDA0
:108E60002046FFF7E1FD62B601B0F0BDF0B581B07C
:108E70000C4606280ED0FBF7C7FC00280AD0FBF7EB
:108E8000C3FCDC4D4059002804D0FBF7BDFC415920
:108E9000D94888476068F7F7C3F9D84F7884A06845
:108EA000F7F7BEF9B884E068F7F7BAF90646F88430
:108EB0002069F7F7B5F9054638856069F7F7B0F925
:108EC00054217852010C5222B952B1B2002929D052
:108ED0001D4A914226D0A9B20A2923D8012422464C
:108EE0008A401A490A421DD0E1214902884203D032
:108EF0004B21C901884215D109F0E4FAFBF784FC43
:108F000000280AD0FBF780FCE34D4059002804D02C
:108F1000FBF77AFC4159BA48884760203C52002050
:108F200001B0F0BDFBF770FC0028F8D0FBF76CFC3B
:108F3000D94C00590028F2D0FBF766FC0159AE4825
:108F40008847002001B0F0BDFFFF00002A040000A8
:108F500010B5022804D14868FFF7BEF8002010BD04
:108F6000FBF752FC0028F9D0FBF74EFCCA4C005925
:108F70000028F3D0FBF748FC0159414888470020FE
:108F800010BDC04610B50220FFF796F8FBF73CFC79
:108F900000280AD0FBF738FCF44C0059002804D014
:108FA000FBF732FC0159F7488847002010BDC04646
:108FB000B0B50C4602280ED0FBF726FC00280AD0DC
:108FC000FBF722FCE94D4059002804D0FBF71CFCBC
:108FD0004159894888476068F7F722F9012816D077
:108FE0000446002827D10020F9F76EFFFBF70CFCA0
:108FF000002843D0FBF708FCEC4C005900283DD07A
:10900000FBF702FC0159EA4888470020B0BDFBF796
:10901000FBFB00280AD0FBF7F7FBF24C00590028B5
:1090200004D0FBF7F1FB0159E14888470120F9F72B
:109030004BFF0020B0BDFBF7E7FB022C11D100284D
:109040000AD0FBF7E1FBE74C0059002804D0FBF7FE
:10905000DBFB0159D64888470220F9F735FF00208D
:10906000B0BD00280AD0FBF7CFFBF44C0059002814
:1090700004D0FBF7C9FB0159014888470020B0BD67
:109080007A7B0100F0B581B04868F7F7C9F805466A
:109090007D20C1002846F7F71DF807460A24284618
:1090A0002146F7F717F8064620467043281A3F0373
:1090B000074364212846F7F70DF82146F7F70AF829
:1090C0000D023D4330462146F7F704F808012843D6
:1090D0004A4988800A49088009F0F4F9FBF794FBB3
:1090E00000280AD0FBF790FBEB4C0059002804D075
:1090F000FBF78AFB0159E9488847002001B0F0BD21
:1091000070AB0102B0B5012812DC0020C443FBF7AC
:109110007BFB00280AD0FBF777FB064D405900285F
:1091200004D0FBF771FB415903A088472046B0BD2E
:109130000020B0BD9405000064656275675F6F66CE
:109140006620666C61670D0A00000000B0B501285A
:1091500012DC0020C443FBF757FB00280AD0FBF7C2
:1091600053FB064D4059002804D0FBF74DFB4159F5
:1091700003A088472046B0BD0020B0BD9405000084
:1091800064656275675F6F6E20666C61670D0A00CB
:10919000B0B50C4602280ED0FBF736FB00280AD0EB
:1091A000FBF732FBE84D4059002804D0FBF72CFBBD
:1091B0004159114888476068F7F732F854210F4C3D
:1091C0006052000C5221605209F07CF9FBF71CFB45
:1091D00000280AD0FBF718FBDB4D4059002804D0CB
:1091E000FBF712FB4159CA488847602001212152F0
:1091F0000020B0BD94050000767B010002C301028F
:10920000717B010010B5FBF7FFFA00280BD0FBF7CC
:10921000FBFA214C0059002805D0FBF7F5FA02595A
:109220001EA024A19047FBF7EFFA00280DD0FBF712
:10923000EBFA194C0059002807D0FBF7E5FA04595E
:10924000FEF71AFF01461EA0A047FBF7DDFA002833
:109250000DD0FBF7D9FA104C0059002807D0FBF7C6
:10926000D3FA0459FEF706FF01461BA0A047FBF7FF
:10927000CBFA00280DD0FBF7C7FA074C005900289D
:1092800007D0FBF7C1FA0459FEF7F8FE014618A013
:10929000A047002010BDC0469405000056657273BB
:1092A000696F6E3A20202020202020202025730D79
:1092B0000A00000056323032313035313030300063
:1092C000494D45493A2020202020202020202020E0
:1092D0002025730D0A000000434349443A20202012
:1092E00020202020202020202025730D0A000000AF
:1092F000494D53493A2020202020202020202020A2
:109300002025730D0A00000080B503482321FBF7D8
:109310000FFA002080BDC04644710100B0B504467C
:10932000FBF772FA022C0FD1002400280AD0FBF7B9
:109330006BFA0E4D4059002804D0FBF765FA4159ED
:10934000EC4888472046B0BD0021CC430028F9D026
:10935000FBF75AFA054D40590028F3D0FBF754FAB1
:10936000415903A088472046B0BDC046940500007F
:1093700075736167653A206C6F6720737472696EEC
:10938000670D0A00717B010010B5FBF73DFA00285C
:109390000AD0FBF739FAD64C0059002804D0FBF765
:1093A00033FA0159D3488847002010BD94050000C6
:1093B000717B0100B0B5032801D10020B0BD0020B1
:1093C000C443FBF721FA00280AD0FBF71DFA054D2C
:1093D0004059002804D0FBF717FA415902A08847EA
:1093E0002046B0BD9405000075736167653A206C36
:1093F0006F675F7072696E74206173635B302D31CB
:109400005D20636E740D0A000020704770470000F5
:1094100010B50220FEF758FEFBF7F6F900280AD037
:10942000FBF7F2F9E04C0059002804D0FBF7ECF907
:109430000159DE488847002010BDC0469405000051
:1094400010B50020FEF738FEFBF7DEF900280AD041
:10945000FBF7DAF9D44C0059002804D0FBF7D4F913
:109460000159D2488847002010BDC04610B50020E1
:10947000FEF72AFEFBF7C8F900280AD0FBF7C4F96B
:10948000EC4C0059002804D0FBF7BEF90159EA481A
:109490008847002010BDC04694050000717B010084
:1094A000B0B50446FBF7B0F9022C0FD10024002818
:1094B0000AD0FBF7A9F90E4D4059002804D0FBF75C
:1094C000A3F94159DC4888472046B0BD0021CC4370
:1094D0000028F9D0FBF798F9054D40590028F3D042
:1094E000FBF792F9415903A088472046B0BDC0461A
:1094F0009405000075736167653A207274635F7349
:1095000065745F616C61726D207365630D0A0000A4
:10951000717B010070470000B0B5072801D1002021
:10952000B0BD0020C443FBF76FF900280AD0FBF759
:109530006BF9054D4059002804D0FBF765F94159F6
:1095400002A088472046B0BD94050000757361678E
:10955000653A207274635F73657420797979792034
:109560006D6D206464206868206D6D2073730D0A32
:1095700000000000BFF34F8F034804490160BFF3B0
:109580004F8F00BFFDE7C0460CED00E00400FA0578
:10959000B0B50C4603280ED0FBF736F900280AD0E8
:1095A000FBF732F9D74D4059002804D0FBF72CF9CE
:1095B00041591F4888476068F6F732FE0546A068A3
:1095C000F6F72EFE0146681E13281FD832291DDC2F
:1095D0007020CB4C25527D20C000F6F791FDE08035
:1095E00008F070FFFBF710F900280AD0FBF70CF920
:1095F000C44D4059002804D0FBF706F94159C24830
:1096000088476020012121520020B0BDFBF7FCF803
:1096100000280AD0FBF7F8F8EE4C0059002804D0D7
:10962000FBF7F2F80159024888470020B0BDC04658
:10963000767B0100F0B581B0052813DC0020C4431F
:10964000FBF7E2F800280AD0FBF7DEF8E14D4059BD
:10965000002804D0FBF7D8F84159DF488847204656
:1096600001B0F0BD0C460520C001D94F38184B6839
:1096700020254C4E294632460BF0AAFCA068FBF789
:10968000CEFB15214901785216483818E36829465F
:1096900032460BF09DFC144838182369294632469F
:1096A0000BF096FC114838186369294632460BF0D6
:1096B0008FFC08F007FFFBF7A7F800280AD0FBF79C
:1096C000A3F8E84C0059002804D0FBF79DF8015995
:1096D000E54888476020012139520024204601B026
:1096E000F0BDC046A2020000C2020000E20200007B
:1096F00094050000717B0100F0B581B0042813DCF3
:109700000020C443FBF780F800280AD0FBF77CF860
:10971000D44D4059002804D0FBF776F84159D3487E
:109720008847204601B0F0BD0C4601200090400261
:10973000CB4F38184B6820251A4E294632460BF07D
:1097400047FC112040013818A368294632460BF027
:109750003FFC092080013818E368294632460BF0A7
:1097600037FC1320400138182369294632460BF094
:109770002FFC08F0A7FEFBF747F800280AD0FBF7FC
:1097800043F8E04C0059002804D0FBF73DF801599C
:10979000DD4888476020009939520024204601B0F6
:1097A000F0BDC046DD83010094050000717B01001F
:1097B000F0B581B0012813DC0020C443FBF724F886
:1097C00000280AD0FBF720F8F24D4059002804D0B9
:1097D000FBF71AF84159F0488847204601B0F0BD20
:1097E0000C4648686946FBF7D3F956269C4DAF5B9B
:1097F0006068FBF714FBB84203D06068FBF70FFB0F
:10980000A85308F05FFEFAF7FFFF00280AD0FAF726
:10981000FBFFE04C0059002804D0FAF7F5FF01598E
:10982000DE4888476020012129520024204601B0EB
:10983000F0BDC04694050000717B0100F0B581B019
:10984000022813DC0020C443FAF7DEFF00280AD008
:10985000FAF7DAFFF24D4059002804D0FAF7D4FFA6
:109860004159F0488847204601B0F0BD0C46486891
:109870006D462946FBF78CF97220794E335A6A7887
:1098800029788B420FD17423F35A93420BD176235C
:10989000F35A6D46AD78AB4205D17823F35A6D4645
:1098A000ED78AB4209D07423F25231526846817888
:1098B0007622B152C078782170527A25775BA06801
:1098C000FBF7ADFAB84203D0A068FBF7A8FA7053D3
:1098D00008F0F8FDFAF798FF00280AD0FAF794FF8D
:1098E000F64C0059002804D0FAF78EFF0159F648CB
:1098F00088476020012131520024204601B0F0BD8C
:1099000002C3010294050000717B0100F0B581B033
:10991000022813DC0020C443FAF776FF00280AD09F
:10992000FAF772FFE54D4059002804D0FAF76CFFB2
:109930004159E4488847204601B0F0BD0C464868CC
:109940006D462946FBF724F96620454E335A6A785E
:1099500029788B420FD16823F35A93420BD16A23A3
:10996000F35A6D46AD78AB4205D16C23F35A6D4680
:10997000ED78AB4209D06823F252315268468178C3
:109980006A22B152C0786C2170526E25775BA06854
:10999000FBF745FAB84203D0A068FBF740FA7053D2
:1099A00008F090FD602001213152FAF72DFF0024CC
:1099B0000028C0D0FAF728FFC04D40590028BAD07F
:1099C000FAF722FF4159C0488847204601B0F0BD50
:1099D00002C30102940500007A7B0100F0B581B05A
:1099E000012813DC0020C443FAF70EFF00280AD038
:1099F000FAF70AFFB14D4059002804D0FAF704FFE6
:109A00004159B0488847204601B0F0BD0C4648682F
:109A10006946FBF7BDF85826114DAF5B6068FBF750
:109A2000FEF9B84203D06068FBF7F9F9A85308F0D3
:109A300049FDFAF7E9FE00280AD0FAF7E5FE9F4C47
:109A40000059002804D0FAF7DFFE01599E488847E4
:109A50006020012129520024204601B0F0BDC046FB
:109A600002C3010294050000717B01007A7B0100B2
:109A70000020704780B502A0F9F7D2FE80BDC04635
:109A80004576656E743A25750D0A0000B0B50C4632
:109A900002280ED0FAF7B8FE00280AD0FAF7B4FE72
:109AA000864D4059002804D0FAF7AEFE415984484B
:109AB00088476068F6F7B4FB00F00CF90446FAF743
:109AC000A3FE002C0ED000280AD0FAF79DFE7B4C96
:109AD0000059002804D0FAF797FE015979488847C1
:109AE0000020B0BD0028FBD0FAF78EFE734C005961
:109AF0000028F5D0FAF788FE0159734888470020FE
:109B0000B0BDC04694050000717B010070B50C46E5
:109B100004280ED0FAF778FE00280AD0FAF774FE6F
:109B2000664D4059002804D0FAF76EFE415964484A
:109B300088476068F6F774FB0546A668E068F6F7A4
:109B40006FFB82B22846314600F01CF90446FAF752
:109B50005BFE002C0ED000280AD0FAF755FE574CB9
:109B60000059002804D0FAF74FFE0159554888479C
:109B7000002070BD0028FBD0FAF746FE4F4C00597C
:109B80000028F5D0FAF740FE01594F4888470020D9
:109B900070BDC046940500007A7B0100717B010016
:109BA00010B582B00023019301A801211B4A00F0E7
:109BB0000DF90446FAF728FE002C0FD000280AD031
:109BC000FAF722FE164C0059002804D0FAF71CFEC2
:109BD000015914488847002002B010BD00280BD05E
:109BE000FAF712FE0E4C0059002805D0FAF70CFEC9
:109BF000025901990CA09047FAF706FE0028EAD016
:109C0000FAF702FE064C00590028E4D0FAF7FCFDF2
:109C100001592D488847002002B010BD759A0000F8
:109C2000940500007A7B0100536F636B49443A2529
:109C3000750D0A00B0B50C4603280ED0FAF7E4FD06
:109C400000280AD0FAF7E0FD1C4D4059002804D046
:109C5000FAF7DAFD41591A4888476068F6F7E0FAE2
:109C60000546A4682046F6F7A1FA02462846214692
:109C700000F05CFA0446FAF7C7FD002C0ED000286D
:109C80000AD0FAF7C1FD0D4C0059002804D0FAF7AC
:109C9000BBFD01590B4888470020B0BD0028FBD010
:109CA000FAF7B2FD054C00590028F5D0FAF7ACFDE3
:109CB0000159054888470020B0BDC0469405000002
:109CC000767B01007A7B0100717B010000207047E8
:109CD0007047000001460020022901D9C0437047A7
:109CE000BE4A4A43BE498B58022B02D3891805222B
:109CF0000A60704710B5E04C216806290FD8012092
:109D000002468A4058210A4209D020600020A06003
:109D10002369002B03D06269002002219847D548AF
:109D20002258062A11D801210B469340582213428B
:109D30000BD021502018002181600369002B04D032
:109D40000E48225801200221984748482258062AE6
:109D500011D801210B469340582213420BD02150B9
:109D60002018002181600369002B04D00448225888
:109D7000022001469847002010BDC046380D000063
:109D80005C1A0000F0B581B00024022803D9E44336
:109D9000204601B0F0BD17460B46094E4643094820
:109DA0008519284618302A2107A2FBF705F842201A
:109DB0002F52032003498851204601B0F0BDC04610
:109DC000240D00002CC8010225730000F0B585B0F9
:109DD000CD4D2C68002C0CD0CA4FCB4CE659002E30
:109DE0000CD0224FE659002E0DD00020C04305B004
:109DF000F0BD01AC0FC400272E4608E001AE0FC62F
:109E0000E619012703E001AE0FC6E6190227DD4C73
:109E100030462146FAF762FE022030607C43291961
:109E2000029D4D60CF600398086104984861084620
:109E30004430CC31012292021023FBF799F87D20A7
:109E40000201DF4800190A494118012D04D1B83038
:109E50000123F9F746FC03E074301023FBF788F880
:109E600001980760002005B0F0BDC046481A000008
:109E7000CC04000001460020022901D9C0437047EC
:109E8000D64A4A43D64988507047C046022806D869
:109E9000D2494143D24840180249401870474B20EC
:109EA00080007047A40C0000022802D94B208000DB
:109EB0007047CA494143CA48401865214901405882
:109EC0007047C046032801DB03487047C34941433C
:109ED000C348401818307047D77C0100022806DCC0
:109EE000BE494143BE4840184221405A70470020B5
:109EF0007047C046032801DB00207047B749414343
:109F0000B748401844307047022804DCB349414345
:109F1000B3484058704700207047C046022805DC0F
:109F2000AE494143AE484018406870470020704732
:109F3000B0B50024E14302280FD8A84A4243A84BF9
:109F40009D58042D09D0991801220A600B69002B35
:109F500005D04A690221984721460846B0BD2046EF
:109F6000B0BDC04610B50024022801D9E04310BDA1
:109F70009A4941439A4A0723535051180B69002BC1
:109F800003D04A69002421469847204610BDC046A8
:109F900010B50024022801D9E04310BD8F49414388
:109FA0008F4A0623535051180B69002B02D04A697F
:109FB00001219847204610BD10B50024022801D980
:109FC000E04310BD85494143854A51180B69002B78
:109FD00002D04A6903219847204610BD240D000095
:109FE0002CC80102F0B583B017460024E2430228D2
:109FF0001AD8002B18D00D467849414378484618A6
:10A0000070680128029312D1002F0AD0B8360024BC
:10A0100029193046F9F76DFB002825D1641CA742A9
:10A02000F6D1029807600022104603B0F0BD0192FD
:10A0300074363046FAF757FF002811D003464268BD
:10A04000BA4209D2196828461D46F6F76DF82B4624
:10A05000686802990860019430461946FAF719FFBA
:10A06000019A104603B0F0BD029804600022104629
:10A0700003B0F0BD240D00002CC80102F0B581B082
:10A0800004460020C343022C02D9184601B0F0BD9B
:10A0900015460E461B4A62431B498F1879680129F1
:10A0A00010D1002D28D01C460090B83738463146D4
:10A0B000F9F7F8FA002821D1761C6D1EF6D1009828
:10A0C00001B0F0BD0090743738462946FAF726FFF4
:10A0D00000280CD00446006831462A46F6F724F8DA
:10A0E00038462146FAF7EAFE009801B0F0BD07A015
:10A0F0002146F9F795FB009801B0F0BD204601B06C
:10A10000F0BDC046240D00002CC80102536F636BE4
:10A1100065745B25755D20526563762042756666C1
:10A1200065722046756C6C0D0A000000F0B583B0B6
:10A13000154607460022D043022F19D8002D17D00C
:10A1400000AB07C30F4878430F490E18443630461A
:10A150002946FAF7E3FE00280CD00446006801996E
:10A160002A46F5F7E1FF30462146FAF7A7FE0298A6
:10A1700003B0F0BD05A03946F9F752FB009803B0D3
:10A18000F0BDC046240D00002CC80102736F636B44
:10A1900065745B25645D2073656E6420627566205E
:10A1A00066756C6C0D0A000002460020022A04DC71
:10A1B0000A4B53430A4AD1507047C0437047C046C8
:10A1C0002CC80102022801D90020704703494143ED
:10A1D00003484018034940587047C046240D00000A
:10A1E0002CC801029C0C000080B504480168491C81
:10A1F00001600069002800D0804780BD345202020F
:10A20000014802490160704790A001020026B8038E
:10A2100010B53B480024C46008300221024A23469E
:10A22000FFF7D4FD204610BDB9A3000010B55A4871
:10A23000002404605F480121024A2346FFF7C6FD5F
:10A24000204610BD05AB0000F0B583B0FBF786FEDD
:10A25000012818D1FAF7BCFB294DE96802291CD066
:10A2600000290DD1FF210902264A11602978002911
:10A2700029D06969411A062902D300212970686131
:10A28000002003B0F0BD1E480021C160FF20000285
:10A290001C490860002003B0F0BDFF210904194AE1
:10A2A00011601949AA69821A3B2A03D86A780B7887
:10A2B0001343E5D0A86100206870087000F084FCAA
:10A2C000002003B0F0BD0126EE6066200F4F3B5A20
:10A2D0006820385A6A21795A6C22BA5A00AC07C4ED
:10A2E000B1020B4C0BA22046FAF766FD6E203A5ADB
:10A2F000A8682146FFF746FD2E70002003B0F0BD90
:10A30000FCA80102D838020259AB010202C30102C3
:10A310009026020225752E25752E25752E25750091
:10A32000B0B584B0FBF71AFE012824D1FAF750FB30
:10A3300019490A68022A24D0002A19D1012008608C
:10A340007221174D6B5A7421695A7622AA5A7824C1
:10A350002C5B00AF16C78102124C13A22046FAF7FD
:10A360002BFD7A202A5A134800682146FFF70AFD80
:10A37000002004B0B0BD084800210160002004B0F6
:10A38000B0BD4A68821A054B9A42F1D300220A6096
:10A390004860002004B0B0BD28A9010210270000C9
:10A3A00002C30102902A020225752E25752E2575FD
:10A3B0002E257500B4A60102F0B5FFB08EB00329BA
:10A3C0002CD8C0467944097949008F4401091219F3
:10A3D000F248C168012921D10021C16001701DE04E
:10A3E000EE48C168012919D10221C1607FB00EB0C9
:10A3F000F0BDEA480021C16001707FB00EB0F0BD31
:10A4000000250295E54880680127BE02721EE44CD3
:10A4100002AB2146FFF7E6FD002802D07FB00EB068
:10A42000F0BD0197029FE555DEA108222046F5F711
:10A43000D2FE002800D184E0D948DDA10822F5F73A
:10A44000CAFE002800D1CBE0D548DCA10822F5F7F0
:10A45000C2FE002800D115E1D148DBA10922F5F7A1
:10A46000BAFE002800D11CE1CD48DAA10A22F5F796
:10A47000B2FE0028D2D0CA48D9A10922F5F7ABFE16
:10A48000002800D13AE1C648D8A10922F5F7A3FE79
:10A49000002800D158E1C248D7A10A252A46F5F77D
:10A4A0009AFE002800D1E5E1BD48D6A11022F5F7BB
:10A4B00092FE002800D139E2B948D7A10C22F5F765
:10A4C0008AFE002800D183E2B548D7A11022F5F713
:10A4D00082FE002800D19BE2B148D8A11122F5F7F5
:10A4E0007AFE00289AD1AE482C2181AA0C23FAF7D3
:10A4F00074FC044603A8D649C822F5F715FE002CC3
:10A500008CD08298FAF718FBD2498988884285D185
:10A5100003ACA022A2710320A080CF480390E01DCD
:10A52000CC49F5F701FEA01CA521F8F7C3FBA72134
:10A530006054000A2146A731487098488068A922D3
:10A54000FCE097482C2181AA0C23FAF746FC052849
:10A5500000D263E78298FAF7EFFABE4EB1888842DC
:10A5600000D05BE78398FAF75AFC7021725A904248
:10A5700001D07052019D849803AC2146FAF708FB84
:10A580006620335A627821788B42844F0FD168233A
:10A59000F35A93420BD16A23F35A03ACA478A34233
:10A5A00005D16C23F35A03ACE478A3420CD06823A2
:10A5B000F252315203A881786A22B152C0786C21DC
:10A5C00070520020F86001256E24375B8598FAF7F9
:10A5D00026FCB84200D085E0002D00D086E01DE7C3
:10A5E0006F482C2181AA0C23FAF7F7FB042800D22C
:10A5F00014E78298FAF7A0FA96498988884200D031
:10A600000CE703A89549018080A80570EFF310803E
:10A6100072B62846294603F017FB60490871000608
:10A6200026D1019F3E0300258D4C28462146324607
:10A6300003F064FA103403AA02232846214603F0EB
:10A640005FFF884C28462146324603F057FA80AA1D
:10A650002846214626463B4603F052FF839C20466F
:10A66000F5F7A4FD711C431C2846224603F048FF61
:10A6700062B6BFF34F8F7C487C490160BFF34F8FB8
:10A6800000BFFDE746482C2181AA0C23FAF7A5FB61
:10A69000032800D2C2E68298FAF74EFA7FB00EB0D5
:10A6A000F0BD3F482C2181AA0C23FAF796FB032822
:10A6B00000D2B3E68298FAF73FFA664CA188884246
:10A6C00000D0ABE683986AA1F5F777FD002800D0AB
:10A6D000A4E60A200121FDF779FD3046E03802F0BA
:10A6E0004CF921E08598FAF79AFB305307F0EAFE1F
:10A6F0006020012131527FB00EB0F0BD03A8009060
:10A70000F048EE4A81AB3946FAF784FA022800D0C5
:10A7100084E6829881990D54EB4CA5888198FAF7CC
:10A720000BFAA84200D079E6A388E64CF44A20460A
:10A730003146FAF741FB0246E14880682146FFF7BF
:10A74000F5FC7FB00EB0F0BDDE482C2181AA0C23B1
:10A75000FAF743FB04468298FAF7EEF9022C00D28E
:10A760005CE6D94DA988884200D057E68398FAF76D
:10A7700056FB04468498FAF752FBA1B2102900D187
:10A780004CE64A0A01D14900685207F09BFE60205E
:10A79000019929527FB00EB0F0BDC046FCA801025D
:10A7A0009026020224636F6E6669672C0000000029
:10A7B000247570646174652C000000002467657462
:10A7C0006C6F672C0000000024636F6E74726F6CF6
:10A7D0002C0000002475736572646174612C0000A4
:10A7E00024736574746F6E652C00000024736574A7
:10A7F000706172612C000000247265616470617286
:10A80000612C000024646F776E6C6F61645F61750A
:10A8100064696F2C0000000024706C61795F6175C1
:10A8200064696F2C00000000247365745F677073A7
:10A83000757762706172612C00000000247265619E
:10A84000645F677073757762706172612C000000DD
:10A85000C866010002C3010255AA03A5CCCCFFFFC4
:10A8600000D0020400A007040CED00E00400FA058B
:10A870005454530093482C2181AA0C23FAF7ADFAC3
:10A8800004468298FAF758F98F4FB988884200D069
:10A89000C4E5022C00D2C1E58398FAF7C0FA064657
:10A8A0008498FAF7BCFA019090480390904804907D
:10A8B00090480590BA8803A80B308FA10AF0A4FB3A
:10A8C0000446019881B20A2900D329460B34002995
:10A8D0000FD03D46B0B20F1840002A5AA0B203A9CB
:10A8E000081886A10AF090FB2418761CB0B28742A3
:10A8F000F2D8A0B203A965220A54601C80B26E226D
:10A900000A54A01C80B264220A54E01C80B20D22BA
:10A910000A54201D80B20A220A5469488068621DC8
:10A9200092B2FFF703FC7FB00EB0F0BD65482C215A
:10A9300081AA0C23FAF751FA032800D26EE5829817
:10A94000FAF7FAF860498988884200D066E503A8DA
:10A950006149018080A8019F0770EFF3108072B6F3
:10A960000020014603F070F955490871000625D111
:10A970003E030025594C28462146324603F0BEF8D6
:10A98000103403AA02232846214603F0B9FD3C46B1
:10A99000534F28463946324603F0B0F880AA28467D
:10A9A0003946234603F0ACFD839C2046F5F7FEFBB9
:10A9B000791C431C2846224603F0A2FD62B6BFF371
:10A9C0004F8F484848490160BFF34F8F00BFFDE7F4
:10A9D0003C482C2181AA0C23FAF7FFF9032800D266
:10A9E0001CE58298FAF7A8F837498988884200D090
:10A9F00014E50A200121FDF7E9FB642001F0BDFF09
:10AA00008398F5F70DFC00F0C0FF7FB00EB0F0BDED
:10AA10002C482C2181AA0C23FAF7DFF92B4903AA31
:10AA200018C918C238C938C2062800D2F6E482987C
:10AA3000FAF782F8244CA188884200D0EEE483988B
:10AA4000FAF7EDF960848498FAF7E9F9A08485981B
:10AA5000FAF7E5F9E0848698FAF7E1F92085879816
:10AA6000FAF7DDF954216052010C5222A152E18C17
:10AA7000002902D0164A914208D11148806803A9E2
:10AA80000A22FFF753FB7FB00EB0F0BD218D0A29DB
:10AA9000F3D8019A8A400F490A42EED0E1214902D7
:10AAA000884203D04B21C9018842E6D107F00AFD54
:10AAB0006020019921527FB00EB0F0BD547B01009F
:10AAC000FCA801029026020202C30102B466010042
:10AAD000FFFF00002A040000CCCCFFFF00D00204DE
:10AAE00000A007040CED00E00400FA052472657074
:10AAF0006C79706172612C0025782C0025642C0023
:10AB0000417B010010B582B0032925D87944097929
:10AB100049008F44010911161F48016801291BD102
:10AB20000021016002B010BD1B480168012913D14A
:10AB30000221016002B010BD17480021016002B07F
:10AB400010BD00200190114800681149114A01AB65
:10AB5000FFF748FA002801D002B010BD019CF9F7B8
:10AB600037FF0D494860002C0AD001200849002316
:10AB7000224609F0F7FC002802D008A0F8F750FEA2
:10AB80000CA02146F8F74CFE02B010BDB4A601029D
:10AB9000902A0202FF03000028A9010252544B2010
:10ABA000446174612053656E64204572726F720D4A
:10ABB0000A0000002575422052544B204461746104
:10ABC0002053656E740D0A00F0B58FB0464DE868ED
:10ABD000022800D086E05620444F385A002600282C
:10ABE0002ED0022856D00128324675D1B8880E9052
:10ABF0003F4800780D907C88FDF73CFA0C9072215C
:10AC0000785A0B907422B85A7623FB5A7821795AD5
:10AC10007A22BA5A374F3F7808910992E1B2220A54
:10AC20000D9C0094019202910C99039104970B9949
:10AC3000059106900793012081022F4841A247E029
:10AC4000B8880E902A4800780D907C88FDF712FA9B
:10AC50000C907221785A0B907422B85A7623FB5AC2
:10AC60007821795A7A22BA5A224F3F78089109926C
:10AC7000E1B2220A0D9C0094019202910C99039179
:10AC800004970B99059106900793012081021A48B9
:10AC90001AA21DE0214838180D90B8880E9014486B
:10ACA00000780C907C88FDF7E5F9124909780522B7
:10ACB000D201BA18E3B2240A0C9F009701940293C0
:10ACC00003AB07C30D980690012081020A4814A225
:10ACD0000E9BFAF771F8024606480670A868064906
:10ACE000FFF724FA0FB0F0BDFCA8010202C3010275
:10ACF00066AB010258AB010290260202245854426E
:10AD00002C25582C2530327525252C25642E2564BC
:10AD10002C25732C25642C312E2C3100A20200002E
:10AD2000245854422C25582C2530327525252C25A5
:10AD3000642E25642C25732C25642C322573202544
:10AD4000732C3100245854422C25582C2530327550
:10AD500025252C25642E25642C25732C25642C3365
:10AD60003A25642E25642E25642E25643A25642E0A
:10AD70002C31000080B582B00E4908680022C26004
:10AD80000192CA68002A02D0016801A8904702B067
:10AD900080BDC04680B582B0064908690022C26005
:10ADA00001220192CA69002A02D0016801A89047D5
:10ADB00002B080BD20A3010280B5002009F08CF80C
:10ADC00080BD80B5012009F087F880BDF0B581B065
:10ADD00003F074FF184DE860A978002901D001B094
:10ADE000F0BD29790029FAD10121297100281ED04E
:10ADF0008F02381AA968814219D03E46A868C8490E
:10AE0000095C0024204600F097FBF7F7B5FFA8681F
:10AE1000401CA860A868791E884200DDAC60E96823
:10AE2000A868022E03D3791A761E8842E6D1002044
:10AE3000287101B0F0BDC046E4A80102F0B587B0AA
:10AE40000346134DE86802281FD112488088124932
:10AE50000978EA88114C2488114E3678114F3F78D2
:10AE600000900191029203940496059701208102BB
:10AE70000D4C0EA22046F9F79FFF0246A868214616
:10AE8000FFF754F9A878401CA87007B0F0BDC04681
:10AE9000FCA8010202C3010266AB01026EAB010213
:10AEA000ACAB010260AB01029026020225732C2597
:10AEB000582C253032782C25782C25642C25642CB0
:10AEC0002564250D0A000000F0B583B0F9F780FD78
:10AED000794CE16B88423FD005F0B0F91F4908601A
:10AEE000F9F776FDE063A1780020002924D0744EA4
:10AEF000724D04E0491EAD1C761C00291BD0747EE7
:10AF0000671C7776132CF5D82A88029282B25300F8
:10AF100001900298694CE0526848C31801986C8E01
:10AF20005C863378664CA354A2183223F45CD45464
:10AF30005776401CDEE7604CA070208B421C2283B9
:10AF40000748818A92B28A4201D9491C2183008D27
:10AF5000012801D100F006F803B0F0BDACAB01024E
:10AF600002C30102F0B58BB0534CA378022B4ED331
:10AF7000581E01900020514932310A46044602937E
:10AF8000049106E0039C641CA0B201998142029BDB
:10AF900038DD0394C043181809900128F2DB00271C
:10AFA0003C4604E0641CA7B20998B842EADD7E0082
:10AFB0001546905F7B1C5900555E0A90A842F1DD52
:10AFC0000595154690190890501807903C48C25CAA
:10AFD0000692C25DC254069AC2553848825B0692F8
:10AFE000425A8253364A3232D55CD65DD654D55554
:10AFF000049A069B43520898059901800A9907987C
:10B000000180CFE70E2B2C4C01D90E23A3702D4DC0
:10B010001220A870AA206870552028702A4800883D
:10B020002871618BA971294A12782A7205220A9225
:10B030005A430F320992EA70000A6871481C608313
:10B04000080AE871224800782249097889010143F9
:10B0500069722148008801784078687329732B74DD
:10B060000020E873A873284611305F00134E314664
:10B070003A461C46F5F758F8781911303236314601
:10B080003A46F5F751F8A000401911300C49224614
:10B09000F5F74AF8A81C0999F7F70CFE06498978D4
:10B0A0000A9A51434A19030A93745074133128467B
:10B0B000F9F7C0FF0BB0F0BDE0AA010234AC010209
:10B0C000C4AB0102645A020270AB010266AB01021A
:10B0D00058AB0102F45B02026EAB010270B50E25A3
:10B0E00000242846214603F0B3FE0D20214603F03C
:10B0F000AFFE0124204608F0F7FD0426284631461D
:10B1000003F0A6FE0920314603F0A2FE204601F01E
:10B11000FBF8A2020249034B204609F0E3F870BD98
:10B12000E43802021D45010080B5012810D800292D
:10B130000ED07C224243B1488018C268012A07D849
:10B140002030F8F7D6FA002801D00020C04380BD97
:10B150000020C04380BDC046F0B589B00022D54371
:10B16000012800D981E00C4600297ED0216A0723FE
:10B17000944DA9420EDC984DA9421ADD974A91429E
:10B180002FDC4B22D501A9423ED0120291424BD175
:10B19000042246E08C4A914217DD8C4A91422ADC17
:10B1A000E1221203914231D08A4A91423CD10C22D1
:10B1B00037E04B252E01B14233D06A01914227D0AE
:10B1C000AA01914230D102222BE0E1225502A9428C
:10B1D00020D09502A9421FD0D202914224D1092247
:10B1E0001FE04B225202914218D0E12212029142FA
:10B1F0001AD1062215E0E1225203914210D0744A7E
:10B20000914211D10D220CE003220AE00A2208E04B
:10B21000012206E0072204E0082202E0052200E005
:10B220000B22D1006E4A53587C214143C94A5050E9
:10B2300056182068B0606068F060A1683161E2680B
:10B240007261012508950025079506950595032748
:10B250000497039502950193012809D000280CD189
:10B26000203601233046F8F73CFA284609B0F0BDF5
:10B27000304620300123F8F734FA206970636069A2
:10B28000B063E069B067A069F063706801A908F075
:10B2900055FF2068012806D8304640302346103339
:10B2A0000ECBF9F765FE60680128DED1301D7036DF
:10B2B00000680122034B314609F014F8284609B012
:10B2C000F0BDC04635450100B0B588B00C467C21C4
:10B2D0004143A0484518686808F006FD281D07216D
:10B2E000384A94420EDC3C4A94421ADD3B4A94426E
:10B2F0002FDC4B22D3019C423ED0120294424DD10E
:10B30000042148E0304A944217DD304A94422ADC56
:10B31000E1221203944231D02E4A94423ED10C21B4
:10B3200039E04B2213019C422AD053019C4229D080
:10B330009201944232D102212DE0E12253029C423B
:10B3400022D093029C4221D0D202944226D10921DC
:10B3500021E04B22520294421AD0E122120294427E
:10B360001CD1062117E0E1225203944212D0184A60
:10B37000944213D10D210EE003210CE00A210AE0D2
:10B38000002108E0012106E0072104E0082102E095
:10B39000052100E00B21C900114A515800240494F2
:10B3A00003220392029401940091059406940121D2
:10B3B000090207910068694608F0C0FE204608B0FF
:10B3C000B0BDC046FFC10100FF0F0E00FF1F1C00F3
:10B3D00080841E0040420F007F250000FF95000082
:10B3E000BC670100B0B50C467C214843594A15188A
:10B3F0002846F9F773FB6C600020B0BD98EF01029E
:10B40000F0B583B00024E743012800D98EE00E4652
:10B41000002900D18AE01546002A00D186E07C216F
:10B4200041434C4841188868022832D001283AD05C
:10B4300000282BD1EFF31080C00702D1EFF310806A
:10B4400072B602910846403001902946F9F766FD30
:10B45000002863D0014601980F46F9F72FFD3868A0
:10B4600031462A46F4F760FE0198F9F73CFDEFF308
:10B470001081C90703D1EFF3108172B662B6029949
:10B480004D6806C82B4B284609F06CF8204603B0DF
:10B49000F0BD4868002431462A46234609F062F888
:10B4A000204603B0F0BDEFF31080C00702D1EFF3E8
:10B4B000108072B602910846403001902946F9F793
:10B4C0002DFD00281ED0014601980F46F9F7F6FC25
:10B4D000386831462A46F4F727FE0198F9F703FD4C
:10B4E000EFF31081C90703D1EFF3108172B662B692
:10B4F00002994D6806C80F4B284609F033F82046DC
:10B5000003B0F0BDEFF31080C0070FD1EFF3108050
:10B5100072B662B63C46204603B0F0BDEFF3108031
:10B52000C00703D1EFF3108072B662B63C462046E6
:10B5300003B0F0BD3548010080B582B001AA11709A
:10B540007C2141430348401820301146F8F7AAF8FF
:10B5500002B080BD98EF0102B0B582B0602833D050
:10B56000622843D0642854D101A82F490180EFF309
:10B57000108072B600242046214602F065FB2B4D58
:10B58000002805D1012002030020294602F0B6FA66
:10B59000103501AA02232046294602F0B1FF62B607
:10B5A00023A0FDF727FC64201B490C5206F08AFFFC
:10B5B0001A4801F0E9F9BFF34F8F194819490160A2
:10B5C000BFF34F8F00BFFDE76020134900220A52EE
:10B5D00006F078FF114801F0D7F9BFF34F8F1048FC
:10B5E00010490160BFF34F8F00BFFDE762200A4999
:10B5F00000220A520A8006F065FF084801F0C4F9EB
:10B60000BFF34F8F064807490160BFF34F8F00BF5C
:10B61000FDE702B0B0BDC04602C30102A086010032
:10B620000CED00E00400FA05AAAA000000D0020414
:10B63000BDF8C8EBC9FDBCB6C4A3CABD0D0A000065
:10B64000F0B581B08A490A78002A23D0874EF28B60
:10B65000002A1FD1874FBA68082A23D8930001A473
:10B66000E3589F4689B60000A5B60000A5B60000C5
:10B67000B5B60000E1B60000EBB60000F5B600007C
:10B68000C3B60000FFB60000552854D10120B860B1
:10B6900001B0F0BD4978002900D1CDE0F7F768FD91
:10B6A00001B0F0BDAA2839D1012A37D10220B860F3
:10B6B00001B0F0BD0421B9600021B970787001B00B
:10B6C000F0BD39797A181073481C3871C0B2797896
:10B6D000491F814200D0AFE00820B86001B0F0BD42
:10B6E0000522BA60887001B0F0BD0621B960B8705B
:10B6F00001B0F0BD0721B960387001B0F0BD7A78B3
:10B70000062A009223D3541F00252B467A19127B58
:10B710009A1893B26D1CA542F8DB19E0C31E59427A
:10B72000594103280AD1022A08D10120F8700320C8
:10B73000B86001B0F0BDC01E414241417879002996
:10B7400022D0002820D101207871032127E0002396
:10B750001818009A821888781118BD7849193C7811
:10B760000919FA78002A00D0C91CC9B2FF2958D19A
:10B7700001282CD0022854D11E2D5FD1FFF7AEFC3A
:10B780000120F08301B0F0BD421E531E9A410123F7
:10B7900059400A4309D10220787103210120002376
:10B7A000024608F0DFFE01B0F0BD801E421E90414F
:10B7B00001433DD100242046F7F786FB03210120F9
:10B7C0000246234608F0CEFE7C7101B0F0BD2A4A45
:10B7D0009471032010719070AA2050705520107041
:10B7E00068085071651DD570400031181646D01D8F
:10B7F0002246F4F799FC301DE11CEAB2D21C037812
:10B8000092B2D218401C491EF9D1A019D143C1717E
:10B81000090A01720934012000233146224608F04A
:10B82000A1FE0020B870B8603871787001B0F0BD2A
:10B830000020B870B860787001B0F0BD701939465A
:10B840000C312246F4F770FC387B012802D12846DF
:10B85000FFF782FE06F036FEBFF34F8F0748084918
:10B860000160BFF34F8F00BFFDE7C04602C3010276
:10B8700018A0010270AA010275B501020CED00E0EA
:10B880000400FA05B0B506F0B9FB002804D0F9F7BA
:10B890009FF80A49C86307E07D20C00001F06DF8F9
:10B8A00006F0ACFB002800D0B0BD044C012525708B
:10B8B000F9F78EF8E06302480570B0BD58AB01029D
:10B8C000FDA8010210B582B009F042FA144C60796B
:10B8D00009F03AF813498A88684682800A884988BC
:10B8E00009048918009104F001FE6079052804D04C
:10B8F00002220D49092805D003E001220A4909283E
:10B9000000D0891849792079621D09F0E1F8607B3F
:10B9100006F0DCF90548064903F0E4FE02B010BD6C
:10B9200044A001029067010098BA0102513C010055
:10B93000E123010080B582B0002001900448C26874
:10B94000002A02D001A80021904702B080BDC04665
:10B9500030A80102B0B508240125204629462A4610
:10B9600003F03CFA0D2029462A4603F037FA0B2053
:10B9700029462A4603F032FA0C2000210A4603F039
:10B980002DFA204603F022FAB0BD70B504460D2012
:10B9900003F00CFA0825284603F008FA052000F009
:10B9A000ECFFF02064263146FDF72EF920463146A3
:10B9B000FDF72AF9284603F009FA70BDF0B583B007
:10B9C00000242046FCF706FEFCF729FE274EB06057
:10B9D000FCF722FE7060264F0BE001A8C18880882A
:10B9E000084319D101A8408824180834B06884425B
:10B9F00035D201AD082128462246FCF7F7FD2888FC
:10BA00000028EAD0B8422AD001AD0421284600F02F
:10BA100059FFA9888842E5D03460B06884420CD2CE
:10BA200001AD022128462246FCF7E0FD2888B842F5
:10BA300003D0A41CB0688442F2D370682118491E58
:10BA40004042084030600DD00024254601202946A0
:10BA5000FCF7A4FD03CE4D19083E8542F6D33460B1
:10BA600003B0F0BD0024346003B0F0BD88A901022A
:10BA7000FFFF0000F0B585B01F4604920646C817C8
:10BA80000C1844400A2C039114D301250A212046A6
:10BA9000F4F720FB6D1C632C0446F7D804998D4203
:10BAA00000D329460A9C002F09D00398002808D407
:10BAB000002207E0012504998D42F2D2F2E700222C
:10BAC00005E00122042323409B081343FA1A0223B2
:10BAD000234004980028029412D1002B10D0F4685F
:10BAE000002C62D40398002825D40298400734D54E
:10BAF0007068B5686F1C87422FD830682B2423E00C
:10BB0000E407ECD1002A0AD1E9E73768202038554C
:10BB1000B560F068441CF460521E002CDFD49142E2
:10BB2000DDD27768B468651CBD42EED9F468521E58
:10BB3000002CF4D5D3E7404203907068B5686F1CC1
:10BB400087420AD830682D244455B760F068441CF9
:10BB5000F4600025ED43A84227DB002B1CD0012018
:10BB6000029B1840049B184316D1002A03D113E00E
:10BB7000521E002C0ED491420CD27068B3685D1C2A
:10BB80008542F5D830683024C454B560F068441C50
:10BB9000F460EDE7002C08D40092029801900A228C
:10BBA00030460399049B00F003F805B0F0BD000097
:10BBB000F0B587B01F4615460290012406919142C8
:10BBC000009407D3012406982946F4F783FA641CED
:10BBD000A842F9D20D980C9ABC42039700D3039463
:10BBE00000990140002A009109D00029029C25D12A
:10BBF0002021800705D40846002F11D004E0029CC4
:10BC00001CE03020002F0BD0084609E02368585470
:10BC1000A260E168491CE1603246721E00290DD421
:10BC2000039991420AD216466368A1684A1C9A4257
:10BC3000ECD9E1683246721E0029F1D5E06800288F
:10BC400059D40590012401E07F1E6C43022FFBD2E2
:10BC5000069821461646F4F73DFA3246A842F4D239
:10BC6000029880680490069F019506973846214601
:10BC7000F4F730FA049D691C029F7A68914206D954
:10BC8000069F059A019D0592002A0ED516E01B4AD3
:10BC9000125C3B685A55B960FA68521CFA6004910C
:10BCA000069F019D0592002A08D460433F1A204652
:10BCB0002946F4F70FFAAC420446D6D20098002881
:10BCC000029C059B049D16D0002E14D0701C01E030
:10BCD000002B10D4401E039981420CD2691C62686B
:10BCE0009142F5D8226820235355A160E268531C85
:10BCF000E3600D46ECE707B0F0BDC046986A01006E
:10BD0000F0B583B002900191002924D00025194C90
:10BD10002E460BE01A480818410F4018C008C0B260
:10BD2000A073761CB1B2019B994216D2029800888A
:10BD30004B27390100B200F025F840007901401886
:10BD4000A08401B20C4881422846E9DB0B488142BD
:10BD5000E0DD6420E4E70748807B642802D90548D9
:10BD60006421817303480121C1740520FCF72EFA78
:10BD700003B0F0BD58AB0102E40C000068100000F5
:10BD80001CF3FFFF074A904201DD054A801800B20C
:10BD90004143C817400D0818C00A00B27047C0469A
:10BDA00000F0FFFFFF07000010B50078012819D14F
:10BDB000AC480269012A04D1614A13680124A343F3
:10BDC0001360032905D080214161C269002A05D191
:10BDD00007E001214161C269002A02D0018980691E
:10BDE000904710BDFF222E32024803A107A306F0A0
:10BDF000CBFDC046647701006164635F646D615F81
:10BE000063616C6C6261636B00000000556E657865
:10BE100070656374656420646D61206368616E6E33
:10BE2000656C0D0A00000000F0B58DB00D460124D0
:10BE3000EFF31081214002D1EFF3108372B6894EE7
:10BE400073690F2B06DD102B37D0402B2FD0802BA2
:10BE50002DD005E0002B2AD0012B01D110237361D6
:10BE6000B5813581B061F261002900D162B63179C6
:10BE7000002929D00294304C05A90A460495039064
:10BE8000E8CCE8C2E8CCE8C2029C204600F02EFED6
:10BE90002A4800902A4D294608312046039A049BDF
:10BEA00000F09CFE2C60002420460DB0F0BD00295F
:10BEB000FAD162B620460DB0F0BD02240029F3D1BC
:10BEC00062B620460DB0F0BD3178002907D01C487D
:10BED000072181610460002420460DB0F0BD326965
:10BEE000B3891749002B15D0B5693089012A02D0D2
:10BEF000002A03D003E09FB2874200D10C604F6854
:10BF0000FF07FCD08F6880C55B1E1F04EED10023A5
:10BF1000B381B561012A02D10A68A2430A60746143
:10BF2000F2690024002ABFD0B36931898800181A49
:10BF3000904720460DB0F0BDD86A0100A9BD0000B1
:10BF400008D00140F0B581B0002856D00446424EDA
:10BF5000F068800754D41325284600F0F1FB2846EA
:10BF600006F0E2F827686168012538462840CA07CC
:10BF7000920F1018227C1207120E8018627C120792
:10BF8000120D8018A27C1207120C8018627D130714
:10BF90001B0AC01812091206801830607D200602A4
:10BFA0000029304600D12D48E3681A0A7D2A1A4636
:10BFB00029D22B4EB3422AD200292BD0002A29465F
:10BFC000254E00D01146F4F785F8401E80B270600F
:10BFD00024480761E27C0270237D0371224F3E6892
:10BFE0006902A468012C1BD02C0226433E60002B62
:10BFF0001ED00121184A116329E0012001B0F0BDD3
:10C00000022001B0F0BD3246154EB342D4D33346C0
:10C010000029D3D11A46002A29460F4ED2D1D2E7A1
:10C020003F242401A6437618F0363E60002BE0D171
:10C03000002A0CD0FF2212020C4B1C6894430122F0
:10C04000D203A2181A60304A1160304A11600121EF
:10C050004161002001B0F0BD00D001400026B803CE
:10C0600080841E0048A801022C06004008E400E07D
:10C0700070B5002801D0012070BD0C461625284659
:10C0800000F05EFB284606F04FF8002C05D01B4858
:10C09000183014222146F4F747F828211748415C4C
:10C0A000002915D04168002916D403220B4693437A
:10C0B000144A9C588D07ED0EFF26AE40B4439C50A9
:10C0C0001F220A40012191400F4A11600F4A11605E
:10C0D00001210161002070BD8A07D20EFF23934029
:10C0E0000F220A40083A03218A43054954589C43C9
:10C0F000545001210161002070BDC04694A001028E
:10C100001CED00E000E400E080E200E000E100E07F
:10C110005A21014A5052704730BA010280B50029B5
:10C1200000D080BD02A007A10B4A0CA306F02CFC96
:10C13000696E636C7564652F6D61696E2F6D6169E1
:10C140006E2E63006170705F7764745F63616C6C06
:10C150006261636B000000008D03000057445420AF
:10C1600054494D454F5554A3ACB3CCD0F2B8B4CEDE
:10C17000BB00000070B55621EB48B42242525C214E
:10C1800000234352414AC287838739244487404968
:10C19000C18683863F4D45863F4D05863325C5853F
:10C1A00083854485C18483847A2444840384C3833F
:10C1B0000383C3820382394C44608360C360836518
:10C1C00003463E33364C250CDD829C82160C5E8283
:10C1D0001A826422DA8157229A8167225A815E226A
:10C1E0001A81DD809C805E80090C018701853D21DC
:10C1F000490441834182090C8183818270BDC0461C
:10C2000070B55621C848B42242525C2100234352E3
:10C210001E4AC2878387392444871D49C186838685
:10C220001C4D45861C4D05863325C5858385448573
:10C23000C18483847A2444840384C3830383C382B4
:10C240000382164C44608360C360836503463E33BB
:10C25000134C250CDD829C82160C5E821A826422AD
:10C26000DA8157229A8167225A815E221A81DD8003
:10C270009C805E80090C018701853D214904418332
:10C280004182090C8183818270BDC0466C006300CD
:10C2900024002F00C7FF0000B7FF00004C3C3C3CCF
:10C2A0006200640070B5A1484C21016001252C0298
:10C2B000601C00F0C5F9322000F066FB00F07CF94C
:10C2C000284600F083F9284600F092F800F06EF955
:10C2D0000C4800F0B5F900263046314600F0C0FAAF
:10C2E0002846314600F0BCFA204600F0A9F90220A9
:10C2F00000F0A6F94834204606F058FA06F0B6FADF
:10C3000070BDC0460102000010B50446072107F0C9
:10C31000F5F93248446010BD10B5044607F0EEF957
:10C320002E48446010BDC04670B50520042529463E
:10C3300002F08EFD06242046294602F089FD0126E2
:10C340003046294602F084FD0E20294602F080FD89
:10C3500011200025294602F07BFD2846314602F0D7
:10C3600077FD022128462A4602F09AFD092021463F
:10C3700002F06EFD0A20214602F06AFD70BD80B514
:10C38000072002F013FD80BDB0B5104800681049C9
:10C390000860012007F0D2FEF6F7B2F80D48FFF76B
:10C3A000D1FD0D48002101600C4D2A6811200321A8
:10C3B00002F08CFC0724204602F008FD06F056FA35
:10C3C0006868214607F09AF9B0BDC046B4AB0102D7
:10C3D00080A701022CA00102ECA80102F4A801022E
:10C3E00002480168012291430160704758000040F3
:10C3F00002490A6802408242FBD170470460004053
:10C40000B0B5494D28688107484C0ED528797F2161
:10C41000084022688A431018206023680B400220DD
:10C420000321434A07F00CFB286880040ED55E20E8
:10C43000285C7F21084062688A4310186060636846
:10C440000B40022003213B4A07F0FAFA172000F0C4
:10C4500077F93948016802220A4301218A430260C0
:10C4600036483749016037480021C17181791F255D
:10C4700029408171817A427C837C1B029A18C37C9B
:10C480001B04D218037D1B06D2182F4B9A4218D1D9
:10C49000427B837B1B029A18C37B1B04D218037C4C
:10C4A0001B06D218294B9A420BD1C27A037B491E34
:10C4B000122906D819028918254A914201D1202152
:10C4C00001720178CA0602D11022114301701C3C8E
:10C4D00020682021884320601E481F490160416870
:10C4E0000029FCD503F026FF0446022003211BA2ED
:10C4F000234607F0A5FA0A20C441032C05D80220E0
:10C5000003211DA207F09CFAFEE71848C1680F221C
:10C510009143C1600168164A0A4002601920000177
:10C52000144948600D60B0BD98BA0102480000404F
:10C53000AC77010096770100040200400C06004031
:10C54000AF6B100A6B0001404D383650312E323639
:10C550000734000000600040FE1C008043686970E2
:10C560002049443A20253038780D0A00C860004040
:10C57000FEFFC3FF0C0400404F6C642063686970C9
:10C58000206D6F64656C206973206E6F7420737505
:10C5900070706F72746564206279207468697320AA
:10C5A00053444B2121210D0A0000000080B51720C3
:10C5B00000F0BEF8002080BD10B51724204600F022
:10C5C000BFF8204605F0B0FD002010BD0121C907CD
:10C5D00001430148016070470060004070B5382099
:10C5E000144C265C204638304578A80604D4B007A1
:10C5F00013D4280718D570BD0F48002101600F48DB
:10C600000178002904D101210170002006F066F8AC
:10C610006078401C6070B007EBD5FCF703F8A07899
:10C62000401CA0702807E6D4FFF72CF9E078401CE6
:10C63000E07070BD84A8010280AB0102D6A00102A7
:10C6400010B5C1B2000AC2B202290CD0012913D020
:10C65000002930D1911E7F4802291BD20121032AD3
:10C660002AD0490429E07B484168002A1FD00246AD
:10C67000203A1143416010BD76480168D31E022B59
:10C6800010D3012A29D0002A41D1012292079143D7
:10C69000016010BD002A16D10121490702688A43B2
:10C6A000026010BD0123042A1FD05A041EE001229B
:10C6B00092079143416010BD0904194A7F32C36A51
:10C6C00013405918C16217498A699207FCD50121A4
:10C6D000490702680A43026010BD05221207914310
:10C6E0000246203A0A43026010BD1A04836A0C4CC9
:10C6F0001C40A21882620B4A131F00241C600A4BC4
:10C700000A4C1C600D235B0214681C431460054A2C
:10C7100093695B06FCD5052212071143016010BD29
:10C7200080FFFCFF1402004004010040FF0F0000E6
:10C7300001218140474802688A4302607047C04631
:10C7400001218140434802680A4302607047C046A5
:10C7500010B5052811D8C0467844007940008744B8
:10C76000020E192434393B490A680868C0003CD5D8
:10C770003A4820390A425DD03BE0002010BD3549DF
:10C780000A680868C00035D534480B46203B1A4279
:10C7900037D134E02F490A680868C00036D52F48E1
:10C7A0000B46203B1A424CD135E02A494C68012007
:10C7B000C0030A680B46203B1C421AD00C68E400F8
:10C7C0003BD5264C1A423CD03AE022480068012072
:10C7D000C00310BD1F490A680868C0001ED51F4865
:10C7E0000B46203B1A4220D11DE01B4820390A424B
:10C7F00020D010BD18480B46203B1A4201D1012021
:10C80000C00349688900890FC84010BD12480B4613
:10C81000203B1A4215D10120C00312E00E480B46FE
:10C82000203B1A4201D10120C00349680903890F46
:10C83000C84010BD0120C00310BD074C1A4200D0F3
:10C8400020464A689200920FD04049680901890F3A
:10C85000C84010BD20000040006CDC020026B80378
:10C8600004282CD8164AC0467844007940008744F2
:10C87000020A121A21000320000713688343880765
:10C88000800818181AE0032080061368834388077D
:10C890000009181812E003208004136883438807F6
:10C8A000000B18180AE0FF200002136883430802F7
:10C8B000181803E01068FF23984340181060704771
:10C8C00024000040B0B5002200290CD0074B0478AA
:10C8D00095B22D0A65406C001C5B12026240491E35
:10C8E000401C0029F3D190B2B0BDC0469868010049
:10C8F000002841D000BF00BF00BF00BF00BF00BF85
:10C9000000BF00BF00BF00BF00BF00BF00BF00BF2F
:10C9100000BF00BF00BF00BF00BF00BF00BF00BF1F
:10C9200000BF00BF00BF00BF00BF00BF00BF00BF0F
:10C9300000BF00BF00BF00BF00BF00BF00BF00BFFF
:10C9400000BF00BF00BF00BF00BF00BF00BF00BFEF
:10C9500000BF00BF00BF00BF00BF00BF00BF00BFDF
:10C9600000BF00BF00BF00BF00BF00BF00BF00BFCF
:10C9700000BF00BF401EBDD1704780B57D21C900FA
:10C980004843FFF7B5FF80BD00280AD030B4072523
:10C990002C02CD256419604340091238001FFDD8D0
:10C9A00030BC704700283ED000BF00BF00BF00BFB2
:10C9B00000BF00BF00BF00BF00BF00BF00BF00BF7F
:10C9C00000BF00BF00BF00BF00BF00BF00BF00BF6F
:10C9D00000BF00BF00BF00BF00BF00BF00BF00BF5F
:10C9E00000BF00BF00BF00BF00BF00BF00BF00BF4F
:10C9F00000BF00BF00BF00BF00BF00BF00BF00BF3F
:10CA000000BF00BF00BF00BF00BF00BF00BF00BF2E
:10CA100000BF00BF00BF00BF00BF00BF00BF00BF1E
:10CA200000BF401EC0D17047F0B583B01F46164608
:10CA30000D460146E8680291F3F758FC04460F2EB4
:10CA400011D8082E04D320462146F3F7F6FB09E05F
:10CA5000042E02D38120C10501E0412001062046B9
:10CA6000F3F744FC04460999089E2B20C0438742F3
:10CA700005DB20460F462146F3F7DFFB0DE03F20A4
:10CA8000C04387420BDA4920C04387420CDBFF20BA
:10CA90000F4681052046F3F729FC39460446688A8B
:10CAA0000880346003B0F0BD01915320C043874239
:10CAB00006DB20462146F3F7C0FB0446688A10E0F7
:10CAC000A8690299F3F73CFE002801D1A88B00E089
:10CAD000E88BF3F781FE01462046F3F707FC044696
:10CAE000002001990880346003B0F0BDF0B581B03A
:10CAF00005460120072D66D80C46002963D04E4F0D
:10CB000038680169C90736D105263046FFF718FE97
:10CB1000304605F009FB03CF03690122134303618B
:10CB2000002918D403200B46834329481E58880740
:10CB3000C00EFF278740BE43402787403743244825
:10CB40001F501F2008408240224802602248026095
:10CB5000394800680FE08A07D20EFF2696400F235F
:10CB60000B40083B03218B4318495F58B7434026CD
:10CB700096403E435E506901401801210902421867
:10CB8000E369DB069B0CA569ED00EDB2EB18536081
:10CB900062685207520B23685B075B099A18A36807
:10CBA0005B079B0CD218E3685B075B0DD218236907
:10CBB0005B01DBB2D21863699B07DB0ED2188023BE
:10CBC00013434350002001B0F0BDC0461CED00E00F
:10CBD00000E400E080E200E000E100E0F0B581B0B8
:10CBE000002A23D005460835134C2668F668EE4027
:10CBF000F50702D0022001B0F0BD069D8600A619FF
:10CC0000B560400124682018009301231D024619D5
:10CC100077680724A7437760F16032610099B160BB
:10CC2000415919434151002001B0F0BD03A00AA1B0
:10CC300074220DA305F0A8FED8A20102696E636CF0
:10CC40007564652F647269766572732F6D6B5F64AE
:10CC50006D612E6300000000646D615F7472616E2F
:10CC60007366657200000000496E76616C6964202D
:10CC70007472616E7366657220647374206164649B
:10CC800072000000F0B58BB017460C4609AA0021CF
:10CC900091800991CD430890002800D1FCE0002646
:10CCA000062109AA304605F009FE062800DAF3E05D
:10CCB0000697059409A9C878000402918988090497
:10CCC00009BA0D182846F3F78FFD0746EC0D744B93
:10CCD000049107963246F3F785FB06460D46002C75
:10CCE00000D13E46002C00D1049D089C2068F3F73B
:10CCF0008FFD02460B4630462946F3F78DFC05466C
:10CD00000E460A20205EF3F76FFD02460B4604959F
:10CD1000284603963146F3F717FC05460F460820D0
:10CD2000205EF3F74EFD3F210906F3F7DFFAF3F734
:10CD3000CFFD02460B4628463946F3F753FB069AC9
:10CD400003C2029A907851780902081811780904F0
:10CD500044182046F3F748FD06460F46E40D079AAF
:10CD60004F4BF3F73FFB0D46002C00D130460690A9
:10CD7000002C00D13D46089948680E46F3F748FD5F
:10CD800002460B4606982946F3F746FC04460690F1
:10CD90000D461C20305E3746F3F726FD02460B4653
:10CDA000204629462E46F3F7CFFB04460D461820B1
:10CDB000385EF3F719FD02460B4620462946F3F785
:10CDC00011FB02460B46069C204631460096F3F7BF
:10CDD000BBFB02900D463869F3F706FD02460B4691
:10CDE00002982946F3F7FEFA02460B4620463146E2
:10CDF000F3F7AAFB04460D46F868F3F7F5FC024684
:10CE00000B4620462946F3F7EDFA04460E46142059
:10CE1000385EF3F7E9FC02460B46049F3846039D53
:10CE20002946F3F791FB22463346F3F7DBFA0290EB
:10CE30000191069E3046009C21463A462B46F3F768
:10CE400083FB054604911A20089F385EF3F7CCFC5B
:10CE500002460B4630462146F3F776FB04460E4663
:10CE60001620385EF3F7C0FC02460B4620463146DA
:10CE7000F3F7B8FA02460B4628460499F3F764FB29
:10CE8000029A019BF3F7AEFA01229207054BF3F7E2
:10CE90005BFB059A03C2079D28460BB0F0BDC04658
:10CEA000000070C1E17A843FF0B587B004460120EC
:10CEB000C043461C002C68D00D46002965D0019067
:10CEC0002046383000270090078029680D208847C9
:10CED000002859D4102858D1E563E968002902D008
:10CEE00028208847E56B02AA1782059704970397C5
:10CEF00002976B68102012219847122848D1049895
:10CF000040BAA08202A8418949BAE18241780A095F
:10CF100003781B019B180F221203DD0A00D09B1817
:10CF2000238183780907090DC918CB0A00D0891815
:10CF3000618101790901C2781203511842791309FC
:10CF4000CB183E49DD0C00D05B18E360C3791207B3
:10CF5000120BD21883791B02D218D30C00D05218AE
:10CF60002261059949BA2183C08940BA6083069835
:10CF700040BAA083E06B016828208847002859D474
:10CF800080210840606306E0019E304607B0F0BD96
:10CF900006460028F9D4E06B82680E26A5213046AB
:10CFA0009047E06B82680F25962128469047E06BFA
:10CFB0008268622002219047E06B82680027304639
:10CFC00039469047E06B8268284639469047E06BC7
:10CFD0008268656BE9B20720904700282AD4E06B8D
:10CFE00082680620072631469047002822D4009800
:10CFF000007804210143E06B8268092090470028F3
:10D0000018D46762A762E76226636563FF20400366
:10D010000B49491C21606060E06B82680820314642
:10D02000904700283046019EAFD420623E463046ED
:10D0300007B0F0BD019E304607B0F0BD0000F0FF24
:10D04000FFFF070000015849085840687047C04674
:10D05000F0B581B005460120012D4CD80C460029C1
:10D0600049D0002D03D0012D04D10F2000E00E2067
:10D07000FFF766FBA668012E04D0002E4FD1E08991
:10D0800000284CD12901294843580020D860F507D1
:10D09000AD0F27686668B607360F76192569EA0767
:10D0A000920EB618022F04D0012F03D1012216438D
:10D0B00000E040361D4F9E60E2681A6079188D606E
:10D0C0006269CA604968002917D403220B4693435A
:10D0D000184A9C588D07ED0EFF26AE40B4438026BB
:10D0E000AE4026439E501F220A4001219140124A21
:10D0F0001160124A116001B0F0BD8A07D20EFF2400
:10D1000094400F230B40083B03218B4308495D5893
:10D11000A543802494402C435C5001B0F0BD08A08E
:10D120000FA1492212A305F02FFCC04620A3010243
:10D130001CED00E000E400E080E200E000E100E03F
:10D14000696E636C7564652F647269766572732F9E
:10D150006D6B5F6475616C5F74696D65722E6300E1
:10D160006475616C5F74696D65725F6F70656E0088
:10D17000636F6E66696720697320696E76616C699A
:10D18000640000000001084A105801608168802294
:10D190000A4382607047C04600010349085881680D
:10D1A000802291438160704720A30102F0B58DB0C9
:10D1B000019315460E460A901298002408900480A8
:10D1C000149F3C8013980990046015980490048083
:10D1D000FF2081053046F3F789F802903046039628
:10D1E0003146F3F72AF82B463D4606902746079529
:10D1F0000B9311E011801888800028580999086065
:10D200000120079D28800520049908807F1CBCB25E
:10D210001888844200D9A0E028880028F6D1A00010
:10D220000A9D2E5830460699F3F77CFA002817D04D
:10D2300030460399F3F776FA00280B9B079DE5D15A
:10D24000089A1780099D2E601888011B012934D186
:10D250001080198889000A9A51582960059035E094
:10D26000089A1780099806600B9B1988081B0128EB
:10D27000C0D00C96019825187E1CB0B28542BFD351
:10D2800089B2B2B28A420ED880000A990C58204660
:10D290000C99F3F739FA0B9B002804D10998046024
:10D2A000089806800C94761CB0B28542A8D31988E1
:10D2B00089B2B2B28A42E7D9F5E70C9601996218B1
:10D2C0007D1CA9B216468A4205972CD2059884B2D5
:10D2D000A5000A9E7259002C104609D0A819001FFB
:10D2E000016810460C92F2F7A8FF0C9A062C07D89A
:10D2F0000446A81941681046F2F79FFF0C9020469B
:10D30000079D0299F3F71CFA00280B9B07D10C9894
:10D310000299F3F707FA0B9B002800D076E701206B
:10D320002880032070E780B2AAB282420FD888001A
:10D330000A990C5820460C99F3F7E6F90B9B002844
:10D3400005D1099804600898058005950C946D1C1A
:10D35000A9B28E42BAD31888E5E70DB0F0BD00003F
:10D36000F0B585B001273904494D686804918843B8
:10D3700068602868474901432960390746480160C9
:10D380004648039101600024204600F0BDFD44485A
:10D39000017849B2002902D480220A4302706869E8
:10D3A0000290A86901903F4803683F4E7360C368CC
:10D3B00033603346143B1B68F3603346103B1B68F5
:10D3C000336133460C3B1B6873613346083B1B6873
:10D3D000B361331F1B68F3616C62FB052C460C3C88
:10D3E00020689843206078046A6882436A6030BF8E
:10D3F0006A6802436A602068184320602B4C0298D8
:10D400000440002901D426480170072068620020EA
:10D4100000F08CFD264803990160BFF34F8FBFF3E6
:10D420006F8F1D48016070681E4908603068C860D1
:10D43000002C08D08C622046019A104008632046D8
:10D440009043C862CC611B4801688906FCD50A2458
:10D450002046FFF799FAF80229688143296020469F
:10D46000FFF792FA38032968814329602046FFF7C5
:10D470008BFA2868B8432860284614380068C00230
:10D48000FAD5686804990843686005B0F0BDC046E5
:10D490002C000040011C000080E200E000E100E000
:10D4A00067000140042000501C010040FFFF030002
:10D4B00080E100E02C0200400A490A680A48024064
:10D4C0000A60FD214900094A1268515C002908D010
:10D4D00007490A6C02400A64012000060A68824378
:10D4E0000A60704700040040FFFFFF7FD4A60102DE
:10D4F0002000004000207047F0B583B00D46044680
:10D500007C26464350488719F869396AF2F7E2FDEC
:10D51000A84200D892E0019502940121EFF3108017
:10D52000084002D1EFF3108272B63C4610343B69DA
:10D530000025062B0CD80A469A40D3065B0F06D16D
:10D5400061231A4275D00D46002803D003E002255E
:10D55000002800D162B6002D02D0284603B0F0BDED
:10D5600000943C462034384880591021C1613E4621
:10D57000143605F075F905463868C069C00605D54A
:10D5800005F06EF9401B31888842F5D90621029DCD
:10D59000284600F02FFF206801994143B869091817
:10D5A00038688160172179563C461734002909D51F
:10D5B000C16920220A43C2610121F9668905026816
:10D5C0000A4302600521284600F014FF207840B28B
:10D5D00000250028C1D42B4800687D24E100F2F723
:10D5E00079FD61014143029800F0D6FE05F038F95B
:10D5F00004463868C069C00705D005F031F9001B42
:10D6000031888842F5D905F02BF904463868C1699C
:10D61000890706D505F024F9001B31888842F5D921
:10D6200038680121009A116053498161284603B08E
:10D63000F0BD0321216000288CD08CE7034804A1B1
:10D64000084A09A305F0A0F94CA30102DC77010008
:10D65000666C6173685F626C6F636B5F6572617348
:10D66000650000005D020000626C6F636B206964FE
:10D6700078206973206F7665722072616E67650D20
:10D680000A00000048520202F0B583B002907C21EB
:10D690004143934A5418E56EEAB2511E02291FD243
:10D6A00029040126090E18D001960092022100F0EB
:10D6B000A1FE2746143705F0D3F806462068C16955
:10D6C000890606D405F0CCF8801B39888842F5D944
:10D6D0002068007DC007019E08D0304603B0F0BD31
:10D6E000032A36D100922804000E36D020466C3032
:10D6F0002D0C0021019101602746143705F0B0F888
:10D7000006462068C069C00705D005F0A9F8801B4F
:10D7100039888842F5D905F0A3F806462068C16922
:10D72000890706D505F09CF8801B39888842F5D911
:10D73000206811498161E9B20120002911D0032933
:10D740000099019E00D006202061226F002A0ED190
:10D75000C3E70026304603B0F0BD0126304603B0D3
:10D76000F0BD0099019E2061226F002AB5D002A869
:10D770009047304603B0F0BD000093EB70B5002831
:10D7800001D0012070BD7825CD4E705D00280ED0EF
:10D7900000240921204600F02DFE0F20FFF7F4F8A9
:10D7A0001520FEF7C5FF74553461204670BD042076
:10D7B00070BDC046F0B581B00C460078484EF168A7
:10D7C00081422CD1032C54D1706EB16E884261D944
:10D7D00000240621204600F00DFE3068F16D8160C6
:10D7E0002046214600F006FE354660352CCDF06817
:10D7F0003168B48C414F00975B1BA34200D81C4694
:10D80000A3081431FFF7EAF9B06E0019B066306E64
:10D8100000193066F06D0019F06501B0F0BDB16817
:10D82000814255D1032C45D1F08CF16D0918F16579
:10D83000316E09183166B16E0818B066716E81429A
:10D8400038D900240621204600F0D4FD3068F16D5F
:10D8500081600121204600F0CDFD316EB068F38C6F
:10D860003268264C009414329B08FFF7B7F901B0D8
:10D87000F0BD30681021C16104F0F2FF0546306848
:10D88000C069C00616D504F0EBFF401BB18A884280
:10D89000F5D90FE030681021C16104F0E1FF0546C1
:10D8A0003068C069C00605D504F0DAFF401BB18AB4
:10D8B0008842F5D90120C107326813688B43136091
:10D8C000F16E22040A4300021043F06601B0F0BD7D
:10D8D0004D200201034804A1844B05F055F8C046D1
:10D8E0004CA30102DC770100666C6173685F646DB4
:10D8F000615F63616C6C6261636B0000B5D70000AF
:10D90000F0B581B000786E4DAA68824200D0D0E0B8
:10D9100001263002032942D16A6DAA66AB6DAC6A5A
:10D92000A418EB652C66AB6C5B1CAB646B6E93420E
:10D9300035D95E30FFF728F8686CA96C02293AD314
:10D94000814238D1E88C696D08186865002006218D
:10D9500000F050FD2868E96D81602F6D04F080FFB4
:10D9600004462868C069C00705D004F079FF001B91
:10D97000A98A8842F5D904F073FF04462A68D06961
:10D98000800706D504F06CFF001BA98A8842F5D9F0
:10D990002A687420285C012841D0F10440E0F20795
:10D9A0002B681C6894431C60EA6E09041143014310
:10D9B000E96601B0F0BD0229FBD38142F9D2E88CBF
:10D9C000696D09186965A96D0818A8650020062108
:10D9D00000F010FD2868E96D8160EF8C04F040FFD5
:10D9E00004462868C069C00705D004F039FF001B51
:10D9F000A98A8842F5D904F033FF04462A68D06921
:10DA0000800706D504F02CFF001BA98A8842F5D9AF
:10DA10002A687420285C012822D0F10421E0310515
:10DA2000334B3B405918012802D01920400601E031
:10DA30000720C00608182F4940185060002F0DD04D
:10DA400004F00EFF04462A68D069800706D404F06B
:10DA500007FF001BA98A8842F5D92A682B6D1FE0B1
:10DA60003105234B3B40C918012802D0192040063C
:10DA700001E00720C00608181E4940185060002F1A
:10DA80000DD004F0EDFE04462A68D069800706D464
:10DA900004F0E6FE001BA98A8842F5D92A68EB8CBF
:10DAA000296EA868144C00941432FFF797F801B05F
:10DAB000F0BD044804A10C4A0C4B04F065FFC046BD
:10DAC0004CA30102DC770100666C6173685F646DD2
:10DAD000615F77726974655F6E62797465735F63A5
:10DAE000616C6C6261636B0072040000C3770100BB
:10DAF000FF3F00000080800001D90000F0B587B032
:10DB000004460126880E14D01546002A11D00F466F
:10DB10008120C004401B88420BD37C206043F04925
:10DB200008180590818C38460691F2F7D3FA00293F
:10DB300002D0304607B0F0BD28460699F2F7CAFA7F
:10DB40000029F6D1059880693E1A30460699F2F709
:10DB5000C1FA0746039670190190069E3146F2F706
:10DB6000B9FA0546C01B04900598006A0290314638
:10DB7000F2F7B0FA049981420FD20026BD42D8D9FB
:10DB80002046394600F03CFB2046FFF77DFD00288B
:10DB9000FAD17F1CAF42F3D3CBE700900398029DEC
:10DBA0002946F2F797FA0646284670430399081A61
:10DBB000019800D0761C2946009D7543F2F78AFA39
:10DBC0000590029941430198401A03900699F2F793
:10DBD00081FA0490AF420BD22046394600F010FB88
:10DBE0002046FFF751FD0028FAD17F1CAF42F3D346
:10DBF00005988642069D009F0CD220463146FFF7CD
:10DC00007BFC2046FFF740FD0028FAD1761C0598E2
:10DC10008642F2D30398A84203D20026304607B0CA
:10DC2000F0BD059847430025E919204600F0E8FAC1
:10DC30002046FFF729FD0028FAD16D1C0026049824
:10DC40008542F1D375E7C046F0B585B0002803D012
:10DC50000124204605B0F0BD7822A14FB85C002811
:10DC600003D00024204605B0F0BD0492002905D061
:10DC7000384614300CC90CC01CC91CC00020F86602
:10DC800015242046FEF75CFD204604F04DFA386866
:10DC90001021C16104F0E4FD04463868C169C90679
:10DCA00007D504F0DDFD001BB98A8842F5D9386834
:10DCB00000E0B98ABA7D1207120B5218F97DCB0722
:10DCC000DB08D2188B07DB0F5B05D218CB06DB0F06
:10DCD000DB05D2184B07DB0FDB06D2188B06DB0FF8
:10DCE0005B07D2180907C90F890711430160002497
:10DCF0000A21204600F07EFB3220FEF745FE082177
:10DD0000204600F077FB04F0ABFD05463868C1699A
:10DD1000890606D404F0A4FD401BB98A8842F5D9CF
:10DD20003868017D0A46C23A5342534174257B55F7
:10DD30000904027D12025118007D0B1802200326EF
:10DD400068A2314605F07CFE785D0128039619D162
:10DD5000F87D029000260621304600F04BFB07219B
:10DD6000304600F047FB012102988143785D01288D
:10DD700047D138688901017506757521795C0129DB
:10DD800038D048E00020032100F034FB04F068FDA7
:10DD900006463868C169890606D404F061FD801B17
:10DDA000B98A8842F5D93868007D46080122F87D95
:10DDB000014631431640C90701D0304036D00295A4
:10DDC000002506212846019200F014FB072100954A
:10DDD000284600F00FFB019846400298385C012865
:10DDE00013D13868B1010175009901757521795C0D
:10DDF000012910D114307621795C4A424A41510000
:10DE000008E038680675490003E038680099017534
:10DE1000710014300170374800687D21C900F2F7A5
:10DE200059F928214143002000F0B6FA7720385CE8
:10DE3000012803D102200021FEF712FD04F010FD9D
:10DE400006463868C069C00705D004F009FD801B8C
:10DE5000B98A8842F5D904F003FD06463868C169DD
:10DE6000890706D504F0FCFC801BB98A8842F5D9E5
:10DE70003868E249816117203856002829D578682A
:10DE8000002816D40146039A91431C4A8B588507F3
:10DE9000ED0EFF26AE40B3438026AE401E438E50AB
:10DEA0001F2101400120884015490860154908607C
:10DEB0000FE08107C90EFF228A400F230340083B71
:10DEC000039883430C481D58954380228A402A4377
:10DED0001A500120049978543861204605B0F0BDED
:10DEE0004CA301026A656465635F69642025780D4F
:10DEF0000A000000485202021CED00E000E400E0CD
:10DF000080E200E000E100E080B57C214143A648CA
:10DF100042187823D25C002A05D04058024941605B
:10DF20000F20FEF731FD80BD008020B980B57C2137
:10DF300041439D4842187823D25C002A05D04058BE
:10DF4000024941601E20FEF71FFD80BD008020AB0E
:10DF5000F0B593B07C270A9047439348C6199807B9
:10DF600004D0F07D4024044000D017E10125880E44
:10DF70002ED0002B2CD08120C004C01A884227D379
:10DF800009920122EFF31084144002D1EFF31080C4
:10DF900072B6304610300590306900250628089189
:10DFA000069310D8079414468440E106490F04D123
:10DFB00061210C4203D0154604E0022502E0022153
:10DFC000059B1960079C002C00D162B6002D02D081
:10DFD000284613B0F0BD344617347348C059102199
:10DFE0000491C1613746143704F03AFC05463068A5
:10DFF000C069C00605D504F033FC401B398888424F
:10E00000F5D92078400665D40297B78C069C204647
:10E010003946F2F75FF8079039464143601A03909A
:10E0200035462435A74200D894E0039800281CD038
:10E0300006210A9C204600F0DDF92888079948430C
:10E04000089940183168886000272046039C3946AB
:10E0500000F0D0F9079B099A28885843C019316805
:10E06000097D11547F1CA742F6D330680499C16121
:10E0700004F0F6FB0446029D3068C069C00605D571
:10E0800004F0EEFB001B29888842F5D904F0E8FB78
:10E0900004463068C069C00705D004F0E1FB001BEE
:10E0A00029888842F5D904F0DBFB04463068C16951
:10E0B000890706D504F0D4FB001B29888842F5D9CE
:10E0C00030680121059A1160B24981610025284616
:10E0D00013B0F0BD03200025089FF765099931664C
:10E0E00006997166B566F0660120C00731680A6856
:10E0F00002430A6006210A9C204600F07BF9306842
:10E1000087602046294600F075F93A4F0BAA0A921B
:10E110001BCF1BC21BCF1BC2B48CF0680A99FEF741
:10E12000E5FCF0683168344A0092069A944200D3C4
:10E130001446A3081431099AFEF750FDB06E001979
:10E14000B066306E00193066F06D0019F065284633
:10E1500013B0F0BD002404E0641C0798844200D38F
:10E1600063E706210A9800F045F92888604308997A
:10E1700040183168886000270A98394600F03AF95B
:10E1800028880028099AE7D0604310183168097D73
:10E19000C1557F1C28888742F6D3DDE7034804A1D8
:10E1A000064A07A304F0F0FB4CA30102DC77010050
:10E1B000666C6173685F726561640000C60300008D
:10E1C00054686520444D412072656164206C656E21
:10E1D0006774682073686F756C642062652074686A
:10E1E00065206D756C7469706C65206F6620340DE8
:10E1F0000A000000386B0100B5D70000000093EB67
:10E20000F0B583B00D4604467C2646435148871935
:10E21000F869B98CF1F75EFFA84200D894E0019547
:10E2200002940121EFF31080084002D1EFF3108235
:10E2300072B63C4610343B690025062B0CD80A46C2
:10E240009A40D3065B0F06D161231A4277D00D4660
:10E25000002803D003E00225002800D162B6002D7B
:10E2600002D0284603B0F0BD00943C46243439481F
:10E2700080591021C1613E46143604F0F1FA05467A
:10E280003868C069C00605D504F0EAFA401B318839
:10E290008842F5D90621029D284600F0ABF8208877
:10E2A00001994143B8690918386881601721795686
:10E2B0003C461734002909D5C16920220A43C261AE
:10E2C0000121F966890502680A4302600421284693
:10E2D00000F090F8207840B22C4600250028C0D4E9
:10E2E0002B4800687D21C900F1F7F4FE20492D314B
:10E2F0004143204600F050F804F0B2FA0446386872
:10E30000C069C00705D004F0ABFA001B3188884211
:10E31000F5D904F0A5FA04463868C169890706D51D
:10E3200004F09EFA001B31888842F5D93868012133
:10E33000009A116017498161284603B0F0BD03219E
:10E34000216000288AD08AE7034804A1084A09A36B
:10E3500004F01AFB4CA30102DC770100666C6173C8
:10E36000685F736563746F725F65726173650000E7
:10E370002B020000736563746F72206964782069F2
:10E3800073206F7665722072616E67650D0A0000FA
:10E3900048520202000093EBF0B583B001917C2259
:10E3A0000290424353498C182546143504F058FA1C
:10E3B00006460221029800F01DF804F051FA0746C3
:10E3C0002068C169890606D404F04AFAC01B29886E
:10E3D0008842F5D92068007DC00708D06420FEF788
:10E3E000D3FA04F03DFA801B01998842E1D903B0C9
:10E3F000F0BDC046F0B585B0049104467C20604372
:10E400003C490F183D46143504F02AFA0646386890
:10E41000C069C00705D004F023FA801B2988884210
:10E42000F5D904F01DFA06463868C069800705D59D
:10E4300004F016FA801B29888842F5D91421049B20
:10E440005943DC2060432C4A101803900291401875
:10E45000018A8268C47C7426BE5D012E0DD10191B3
:10E46000012B02990CD0012B0DD07526BE5D012E1B
:10E470000ED0019E072B0ED10EE00E4602990BE046
:10E480000222012BF1D138247526BE5D012EF0D178
:10E490000326072B00D0019E184B33402406920719
:10E4A000D20A1219D218039B5958C907490C52189D
:10E4B0004168CB071B0CD218837C5B075B0BD2181F
:10E4C000C0684007000A10183A685060002E0ED04D
:10E4D00001290CD104F0C4F904463868C0698007EA
:10E4E00005D404F0BDF9001B29888842F5D905B090
:10E4F000F0BDC0464CA30102806C0100FF3F00004C
:10E50000F0B59DB00D460126890E2FD0002B2DD0E1
:10E5100011928121C9041093C91AA94226D301215D
:10E52000EFF310840C4002D1EFF3108272B67C221C
:10E530000F904243E74814928718384610303B69E1
:10E540000026062B0DD80A469A40D3065B0F07D14A
:10E5500061231A4200D16FE30E46002C03D003E082
:10E560000226002C00D162B6002E02D030461DB02B
:10E57000F0BD0290BD650021139179651098401E91
:10E5800012904019B964B9690D916E1A1199B96266
:10E59000FD6238637E63F98C0E913046F1F79AFD87
:10E5A0000446B863129830180E9E3146F1F792FD7A
:10E5B000109B011B4A1CF86339647A64139A002982
:10E5C000194608D0704359190D9BC91A0A1A744389
:10E5D000581B80190119384648300E90384644308F
:10E5E0000D90384640300B9038462630059038461E
:10E5F00058301390384654301290F9643A651498A4
:10E60000B44908581021C161384614301490384676
:10E61000503004903D464C3504F022F904463868E9
:10E62000C069C00606D504F01BF9001B14990988BF
:10E630008842F4D9F87D40060C9500D574E2012398
:10E640000E9803600D98016800290F9800D1CDE263
:10E650003A4674320A92DA0407921A05099219228C
:10E66000520606920722D206089216E09A480068DF
:10E670007D21C900F1F72EFD109941430F9C2046E2
:10E68000FFF78AFE20460C9D0E9A11684B1C136002
:10E690000D9909688B4200D9A8E20B9A1268012AE9
:10E6A00055D0002A00D0A8E02E6812990C68139962
:10E6B0000D6806211091FFF79DFE3868856011985E
:10E6C000051904F0CDF804463868C069C00706D0C3
:10E6D00004F0C6F8001B149909888842F4D904F0A4
:10E6E000BFF804463868C169890707D504F0B8F84F
:10E6F000001B149909888842F4D938680A990A7865
:10E70000012A089900D00699012A099A00D0079A8F
:10E710003346724C234013430B4371490B43436010
:10E72000002EA3D004F09CF804463868C069800726
:10E7300006D404F095F8001B149909888842F4D98E
:10E740003868297801756D1C761EFAD18EE7012B89
:10E7500000D0C7E02E6812990C6813990D68062145
:10E760001091FFF747FE386885601198051904F08D
:10E7700077F804463868C069C00706D004F070F81E
:10E78000001B149909888842F4D904F069F80446FA
:10E790003868C169890707D504F062F8001B14992D
:10E7A00009888842F4D938680A990A78012A0899B0
:10E7B00000D00699012A099A00D0079A3346474C9F
:10E7C000234013430B4346490B434360002E69D05B
:10E7D00004F046F804463868C069800706D404F09F
:10E7E0003FF8001B149909888842F4D938682978C1
:10E7F00001756D1C761EFAD154E0012B00D0C9E0E2
:10E800002E6812990C6813990D6806211091FFF774
:10E81000F1FD386885601198051904F021F8044667
:10E820003868C069C00706D004F01AF8001B1499B4
:10E8300009888842F4D904F013F804463868C1699D
:10E84000890707D504F00CF8001B14990988884241
:10E85000F4D938680A990A78012A089900D00699EB
:10E86000012A099A00D0079A33461C4C23401343CF
:10E870000B431B490B434360002E13D003F0F0FF02
:10E8800004463868C069800706D403F0E9FF001B1E
:10E89000149909888842F4D93868297801756D1C63
:10E8A000761EFAD10C4800687D21C900F1F712FCF0
:10E8B000109941430F9C2046FFF76EFD20460C9DAA
:10E8C0002A68139B196889181960129B196889189E
:10E8D0001960D9E64CA3010248520202FF3F000032
:10E8E000008080008B4200D0CEE604990E68129919
:10E8F0000C6813990D6806211091FFF77BFD3868AD
:10E9000085601198051903F0ABFF04463868C069AB
:10E91000C00706D003F0A4FF001B149909888842A1
:10E92000F4D903F09DFF04463868C169890707D50B
:10E9300003F096FF001B149909888842F4D93868BF
:10E940000A990A78012A089900D00699012A099A99
:10E9500000D0079A3346D44C234013430B43D3498A
:10E960000B434360002E00D180E603F079FF04469C
:10E970003868C069800706D403F072FF001B149941
:10E9800009888842F4D93868297801756D1C761E8B
:10E99000FAD16BE6129A1268119CA618139A1568A0
:10E9A0008B425FD104990C6806210391FFF722FD89
:10E9B0003868856003F054FF05463868C069C007B1
:10E9C00006D003F04DFF401B149909888842F4D902
:10E9D00003F046FF10900C9D3868C169890708D57F
:10E9E00003F03EFF1099401A149909888842F3D920
:10E9F00038680A990A78012A089900D00699109176
:10EA0000012A099A00D0079A2346A7490B401343CD
:10EA100010990B43A5490B434360002C14D003F01D
:10EA20001FFF10903868C069800707D403F018FFF3
:10EA30001099401A149909888842F3D938683178B6
:10EA40000175761C641EFAD19A4800687D21C900C0
:10EA5000F1F740FB039941430F9C2046FFF79CFCD4
:10EA6000204611E605990C8806210391FFF7C2FCA8
:10EA70003868856003F0F4FE05463868C069C00751
:10EA800006D003F0EDFE401B149909888842F4D9A2
:10EA900003F0E6FE10900C9D3868C169890708D51F
:10EAA00003F0DEFE1099401A149909888842F3D9C0
:10EAB00038680A990A78012A089900D006991091B5
:10EAC000012A099A00D0079A234677490B4013433D
:10EAD00010990B4375490B434360002C14D003F08D
:10EAE000BFFE10903868C069800707D403F0B8FEF5
:10EAF0001099401A149909888842F3D938683178F6
:10EB00000175761C641EFAD16A4800687D21C9002F
:10EB1000F1F7E0FA039941430F9C2046FFF73CFCD4
:10EB2000204605990A88CCE65E4815A90A4678C8A9
:10EB300078C278C878C20125E8073A6813680343A9
:10EB40001360B868FDF7D2FF02200026139C2168ED
:10EB5000BA6AF9653A6610997966BE66F8660C98E5
:10EB60000068129A1168091811600E9B19684A1CF6
:10EB70001A60226810182060002900D0F6E4109571
:10EB80003846603013903C465C343846083012906A
:10EB900006210F98FFF72EFC3868216881600C98D9
:10EBA0000068119003F05CFE04463868C069C00735
:10EBB00006D003F055FE001B149909888842F4D949
:10EBC00003F04EFE0446109D3A68D069800707D5D1
:10EBD00003F046FE001B149909888842F4D93A686C
:10EBE0007420385C01282DD0E9042CE003F038FEB5
:10EBF00004463868C069C00706D003F031FE001B28
:10EC0000149909888842F4D903F02AFE044638682A
:10EC1000C169890707D503F023FE001B14990988F1
:10EC20008842F4D938680121029A11602249816131
:10EC3000002630461DB0F0BD04210160002C00D13B
:10EC400091E491E42905119C174B234059180128A0
:10EC50000C9D02D01920400601E00720C0060818CC
:10EC6000124940185060002C0ED003F0F9FD044604
:10EC70003A68D069800707D403F0F2FD001B1499AD
:10EC800009888842F4D93A682B6813980168129869
:10EC90000068074C00941432FDF7A0FF30461DB009
:10ECA000F0BDC046F86A0100FF3F00000080800010
:10ECB00001D9000048520202000093EB3920C00045
:10ECC0000149096808587047D8A20102F0B5032924
:10ECD00020D8C0467944097949008F4401080F15AE
:10ECE000012181404F4B1B685963D96212E0012119
:10ECF00081404C4B1B681963D9620BE001218140B4
:10ED0000484B1B68596304E001218140454B1B6857
:10ED10001963996283004349CB18DA608A68002A34
:10ED200029D14A68002A16D4032314469C43174B62
:10ED3000E5589607F60EFF27B740BD438027B7403A
:10ED40002F43E7501F23134001229A40104B1A60B3
:10ED5000104B1A600FE09307DB0EFF259D400F2438
:10ED60001440083C03229443074AA658AE4380252A
:10ED70009D403543A55001228240086802628868A0
:10ED800010438860F0BDC0461CED00E000E400E0E8
:10ED900080E200E000E100E010B501242046FDF72C
:10EDA000CFFC204603F0C0F9002010BD01218140B6
:10EDB0001C48006842688A434260704719490968E4
:10EDC0000968C140012008407047C04601218140C8
:10EDD0001448006842680A4342607047012907D01E
:10EDE000002910D1012181400F4802680A430FE039
:10EDF000012181400B4800684368002A0DD00B4375
:10EE000043600161704701218140074802688A43DD
:10EE1000026004480068416170478B4343600161B0
:10EE20007047C046DCA301020801004010B5054848
:10EE300004680548006860430449F1F761F9201A45
:10EE400010BDC04674000040C446020240420F009C
:10EE5000124A072809D880000F23834081401940B7
:10EE6000106898430843106070470F280AD8800044
:10EE700020380F238340814019405068984308434D
:10EE800050607047800040380F2383408140194014
:10EE900090689843084390607047C0463400004033
:10EEA000F0B54307DC0E0726A640C3089D000E4BB5
:10EEB000EF187D68B5433E1D002908D0356001225A
:10EEC000824001290CD1186810431860F0BD01215F
:10EED0008140186888431860A24015433560F0BD32
:10EEE000186890431860F0BD0C01004010B582B066
:10EEF00014460A46014604980093019008202346D0
:10EF000000F092F802B010BDB0B584B014460A46C5
:10EF10000146089802250095019302900720234698
:10EF200000F052F904B0B0BD70B500285BD0314993
:10EF30000A783149002A03D14A68012313434B6000
:10EF4000428803881B049A180B46183B1A60828873
:10EF500083891B049B180C460C3C23600B46083B22
:10EF600084681C60446903232340057CAD00EB18D2
:10EF70008569AD072D0D5B19457C2D035B19C569AE
:10EF8000AE07B60A9B19867CB6059B190E1F336027
:10EF9000036A122B04D107240C60541EA2410AE01C
:10EFA000032C05D1012D03D807220A60012202E0BB
:10EFB00006220A600122114C002525700F246401ED
:10EFC0002034C57C6D0225401B069B0BD218C379EB
:10EFD0001B07DB0ED21880790007C00D10184019EE
:10EFE0001439086070BD064806A1862209A303F003
:10EFF000CBFCC046DC38020218100050DE3802029A
:10F00000388601006C73705F656E67696E655F724C
:10F01000756E0000506172616D6574657220697370
:10F02000206E756C6C000000F0B58BB0109E34043F
:10F030003ED00D46D64C2140012701977F06B942AC
:10F040003CD111462140B9423FD11C40BC4243D182
:10F05000119902AC0027E781E7806680278027822C
:10F06000A774E1749908A181A908A1800A90099761
:10F0700008970797900880B204902046FFF754FF46
:10F08000AA480078002801D00BB0F0BDAB48016859
:10F09000C90708D10168C90705D10168C90702D1AC
:10F0A0000168C907F3D07F48019901700BB0F0BD2A
:10F0B000B8480D49AF22C14B03F066FC0095B54836
:10F0C0000949B022754B03F05FFC0092B148064934
:10F0D000B122724B03F058FC0093AE480249B222B1
:10F0E0006E4B03F051FCC0460E860100F0B58DB0AA
:10F0F0000392139E340446D00A46A54C21400125B4
:10F1000002956F06B94244D103992140B94247D1D3
:10F110001C40BC424CD11499129D04ACE1742949A5
:10F1200021820027E781E780668027809908A181F6
:10F130009108A1800B95012D01D16121CF43A774C6
:10F140000C9002200A9009900398800880B20690E3
:10F150002046FFF7E9FE75480078002801D00DB081
:10F16000F0BD76480168C90708D10168C90705D113
:10F170000168C90702D10168C907F3D0494802995B
:10F1800001700DB0F0BD83480D49FB228B4B03F09D
:10F19000FBFB00927F480A49FC22404B03F0F4FB42
:10F1A000039800907B480649FD223C4B03F0ECFBA2
:10F1B000009378480249FE22384B03F0E5FBC04635
:10F1C0001B8601008E8E0000F0B58BB0119E3404BA
:10F1D00047D00D466E4C2140012701977F06B9426A
:10F1E00045D111462140B94248D11C40BC424CD1C6
:10F1F0001299109F02ACE174294921820021E1811A
:10F20000E180668021809908A181A908A1800997E1
:10F21000012F01D0712100E06121C943A1740A903E
:10F22000032008900790900880B204902046FFF7D2
:10F230007BFE3E480078002801D00BB0F0BD3F486F
:10F240000168C90708D10168C90705D10168C90764
:10F2500002D10168C907F3D01248019901700BB0BF
:10F26000F0BD4C480C49D522544B03F08DFB009562
:10F2700048480949D622094B03F086FB00924548CD
:10F280000549D722054B03F07FFB00934148024913
:10F29000D822024B03F078FB2A8601005886010031
:10F2A00086860000DE38020210B582B014460A4697
:10F2B000014600200093019004202346FFF7B4FE8E
:10F2C00002B010BD10B584B014460A4601460020B5
:10F2D00000900193029004202346FFF707FF04B03B
:10F2E00010BD000070B50D46064604242046FDF70B
:10F2F00027FA204602F018FF0B4805600B480670FD
:10F30000002E0ED00A48016880220A437F218A43DA
:10F3100002600120000307490860074908600748A8
:10F320000460002070BDC046E0380202DC380202F2
:10F330000CE400E080E200E000E100E01C1000507E
:10F34000B0B582B0144602461148204001256D0632
:10F35000A8420DD1180413D0174801600020009373
:10F360000190062011462346FFF75EFE02B0B0BDB5
:10F370000094FF228C320748074908A303F004FBDE
:10F38000FF208C30421C034803490C4B03F0FCFA6D
:10F390000300FCFF388601000086010044737420DE
:10F3A0006164647265737320257820697320696EC7
:10F3B00076616C69640000000810005076860100D8
:10F3C00080B582B00B4601460020009201900320D8
:10F3D0000A46FFF729FE02B080BD0000002801D0D8
:10F3E000042100E00221C14A5172411E884180017E
:10F3F00003490A6840239A43101808607047C046C2
:10F4000050A00050F0B583B002912E49CD7A0E7B0A
:10F41000771987424FD9089901911825454341260C
:10F42000F604BF00BE19745B34490C4057033C1905
:10F430009B07D90C6418324B1B681B7A74537519DF
:10F440006C880326B60326409B079B0C9B193F2420
:10F4500004401819029CA3061B0DC0186880012ADD
:10F46000184E13D8707B14224243307B5023434301
:10F4700024011B199A18F37AC0181C234343D0188F
:10F4800080081E4A104007430F432F800198686090
:10F4900002F0E0F8A860E8681A4908403030E860F7
:10F4A000286908402721715C4018286101F044F860
:10F4B000686103B0F0BDFF228832034803A108A3AE
:10F4C00003F062FAE83C0202C78601006D61635FE7
:10F4D00063735F636F6E7374727563740000000012
:10F4E000435320696E646578206973206F76657276
:10F4F0002072616E67650D0A00000000FF070000C2
:10F50000D4A601020000F0FF2820E94900220A5495
:10F510007047C046F0B581B0009314460D460746CB
:10F5200006263046FDF70CF9304602F0FDFD262197
:10F530001D48475400210170417081710171817033
:10F540004171C170C17102224272C16201634163A3
:10F55000816304734273C572009A561C134A168065
:10F5600001724120C00401214903F0F7F6FD50204B
:10F5700060432901081861198A00801818224A433B
:10F580008018B2B24A438018094940180949884294
:10F5900004D200F0ADF8002001B0F0BD064807A18C
:10F5A0009A2209A303F0F0F9E83C0202E43C0202CB
:10F5B0002800080201200802C78601006D61635F10
:10F5C000696E697400000000454D206F76657266B3
:10F5D0006C6F770D0A000000F0B583B002912A49E4
:10F5E0004B7B834248D9CB7A0C7BE31818245C43CD
:10F5F0009B00E3184124E4041A19142401900546E1
:10F6000065430026565100925519EE882E4F0B4641
:10F610007A1C32402D4E3688497A711A2C4E0E4093
:10F62000B618EE803740997BEF80AA88294F1740A3
:10F630004A424A4191007918274A8918A980274FE0
:10F640000F402D1D029801280AD125490E4009219D
:10F65000C902711869800121C9037918298000E065
:10F660002F800198444300980019074A918C4182E9
:10F67000118C018203B0F0BD3520C200034804A103
:10F6800009A303F081F9C046E83C0202C7860100E5
:10F690006D61635F6C696E6B5F646573635F636FFD
:10F6A0006E737472756374004C696E6B206465735D
:10F6B0006320696E646578206973206F76657220B7
:10F6C00072616E67650D0A00FFFBFFFFE43C0202FA
:10F6D000FF03000003D0FFFFE80F0000EF1F000052
:10F6E000FF830000D34A506391637047E83C0202F5
:10F6F000F0B581B04348CC21016003214160CD4980
:10F700000A7BD304404C1B19CC7AA218541E1C430C
:10F710001823534392009A184B7B14255D435219CA
:10F720009201224301246306134343610022826253
:10F73000C262026342638263C26342650267334B03
:10F740001A605A609A60324B1A601A619A61DC61E1
:10F75000304C1C62304C251D1D6325460C3D5D63FD
:10F760002546283D9D632D4EDE631C645C642C4D54
:10F770002F461C379F642746143FDF64103C1C65EE
:10F78000284C5C65284C9C650C369E67274CA5630D
:10F790004035E563DA651A665A669A66DA661A676C
:10F7A000234DDD6702258561224DC561C325AD036B
:10F7B000CD620A63D2435A601F4A1368FF25AB43E8
:10F7C00026254D5DAD072D0EEB1813601B4A102347
:10F7D00013601B4A1360272260238B5419498160F0
:10F7E000C160016121607D21090101664166164900
:10F7F000C164164941641649016400F08DFE01B0F0
:10F80000F0BDC04604A000500000F8FF94A00050D6
:10F8100034A10050FF185A0030040040041000408A
:10F820001C2000405430004060400040B8A100500F
:10F8300014001400FF3F3FFF04E400E080E200E01A
:10F8400000E100E0DC05DC053F0270020133D00777
:10F85000D007D00770B5182002F066FC192002F01E
:10F8600063FC0624204602F05FFC2046FCF768FF9C
:10F87000D34C002525706570A5712571A570657143
:10F88000E570607B14214143207B50224243E37AA0
:10F890001E0192195118C0181C2242438918412098
:10F8A000C004F0F75AFCE5712572FFF721FF70BD27
:10F8B000E83C0202F0B58BB0079208910146C04FB8
:10F8C000B8780991FFF788FE78793A7B79790691C3
:10F8D000824200D89FE0FB7A9A1818235343920083
:10F8E0004124E10404915218D2187B7B14214B432C
:10F8F000D21850246043155801230A93DB022E4688
:10F900009E4316504E4B2B4005937D7B03914D43F8
:10F910003E7B7443F97A0B011B195B1971181C2487
:10F92000029461435918A74B1B88069C5C43091934
:10F93000C904490D059BC918115010180799416059
:10F9400038787979089A00920322099BFFF75AFDCB
:10F95000F87A397B09183878814263D98300099392
:10F96000049AD45C0894F7212140D154D1184D78E1
:10F970008E7836027619CB781B04F31807900A9814
:10F9800086051E43330CCB70FB7A387BBC784D70F8
:10F990009E4D3540039E6643C018029B4343981911
:10F9A00040029B4B03405C19200A8870200CC870F1
:10F9B000F023089D2B401B1D3D7B0895FE7A099D79
:10F9C0005355C8700620079A50438019089A80182A
:10F9D00048701F22D20222400243100A88707879B0
:10F9E000401C7871387B7979814201D3002179718B
:10F9F0003978491C3970F97A08183978884201D861
:10FA00000020387028200A993954387A401C3872FE
:10FA1000387A0BB0F0BDA7204200D1480649074B09
:10FA200002F0B2FFA72042007A32CD487249734BF0
:10FA300002F0AAFFE83C0202E7860100908601007E
:10FA400000F0FFFF0320000605490A6882430A60B0
:10FA50000A6802430A600348012101607047C046FA
:10FA60001C0000401CA0005080B50120FDF794FB55
:10FA700080BD0000F0B587B006930646504C607A12
:10FA8000504B1B88181A0C9DA84200DC89E00F46D9
:10FA90000592012E06D156480021C1620169554ADE
:10FAA00089180160A0783146FFF796FDE078E1788B
:10FAB000069A2B4600F0AEF82078E17800970022F5
:10FAC00006923346FFF79EFCE07A217B08182178E6
:10FAD00088426ED94120C20404918800815C039160
:10FAE000F7250D40029285544549455C4549465CE1
:10FAF000360276194449475C3F04F6190127BF05D1
:10FB000037433E0C4654E67A217BA3783C4A855421
:10FB10003E4D3D4014275F4389191C234B43D9199F
:10FB200049023B4B0B405D19290A364BC1542E0C40
:10FB300035494654F02703990F400599002900D113
:10FB40003F1D217BE37A029A87542F4A865406226E
:10FB5000049E7243D2185118294A81541F22D2029E
:10FB600015400D43290A274A8154E078401CE07073
:10FB7000E07AE178814201D30699E1702178491C4D
:10FB80002170217B08182178884201D806982070BE
:10FB9000E079401CE071A07A401CA072E07907B0C7
:10FBA000F0BD3920C2001632074808A109A302F0AF
:10FBB000EBFE3920C20004480F49104B02F0E4FE6E
:10FBC000E83C0202E43C0202C78601006D61635F0B
:10FBD000747800004D4143205458206C656E2069B4
:10FBE00073206F7665722072616E67650D0A000082
:10FBF0000804004090D00300FD860100AE8601009D
:10FC0000010008020200080203000802FF07C0FF0B
:10FC100000F83F00F0B589B00893019204914F4D70
:10FC2000EF7A874200D891E0297B502632464A433A
:10FC30004124E3040693D218CC19A10051181822CC
:10FC4000059254430A19697B1423079359435318A7
:10FC500002900001195804460390504A0A40A97ABC
:10FC6000C902511808988205D2088A181A514C49BD
:10FC700011402A7B00965643384CE57A2C010698B1
:10FC80002418A719354E5419A5007D190598444329
:10FC90002819747B079D6C430519049FD2194148AC
:10FCA000048854432A19089CD204520D51181D4649
:10FCB0000398195000F04AFC0146707A00190204BA
:10FCC0003E460CD080B2C000002900D1801E029FA9
:10FCD000A5214900F0F7FEF91F21014001E00021B4
:10FCE000029F38012818427983791B029A18C37938
:10FCF0001B04D2182C4B1340437109045918090CEA
:10FD0000C171002C20D0154835460646007B009B6B
:10FD10004343F17A0A01069F3A43D21841188B00F7
:10FD2000D218059B4B43D118727B079B5343C918CC
:10FD300040191C4A1288424388180199884203D00E
:10FD400001992246F0F7F0F909B0F0BDFF225C32CC
:10FD5000034804A109A302F017FEC046E83C0202D2
:10FD6000C78601006D61635F74785F646573635F6C
:10FD7000636F6E737472756374000000545820448E
:10FD800045534320696E646578206973206F7665FA
:10FD9000722072616E67650D0A000000FF0700E0C7
:10FDA00000F8FFFFE43C0202EFFFE0000168044AB4
:10FDB00011604168516081689160C068D06070478F
:10FDC00080A0005082B062B6FCF76CFA05260025D0
:10FDD00030462946FFF73CF8062738462946FFF704
:10FDE00037F80124304621462A46FEF7F7FF384609
:10FDF00021462A46FEF7F2FF0A202946FFF728F897
:10FE000009202946FFF724F8204603F06DFF284615
:10FE100003F06AFFFCF788FAFEF7BEFFF5F750F92A
:10FE2000F2F78CFDF2F7ECFEF8F700FA0721204616
:10FE3000FCF772FA02F0F8F802F0F0F88348016873
:10FE400083480068890308D4032109070840210773
:10FE5000884202D0FCF78EF906E0FBF7AFFDFCF715
:10FE6000CFF90020FDF78AFCFCF7CAFA00252846E6
:10FE700005F004F8F8F710FC012420462946FBF7AA
:10FE8000B1FA28462146FBF7ADFAF2F739FFF6F74B
:10FE90005DF8FAF7BDF956206E4E0190305A0128F0
:10FEA00001D1FAF7C3F96C4F391D0025284605F03A
:10FEB00019F8F6F763F80A202146F8F787F9FBF7F7
:10FEC00049FD38461030FCF73DF8A2026349644B07
:10FED000204604F007FA01F043FEFBF7F3FC308DF7
:10FEE000002804D0B08C002801D0F8F75FF902F0A8
:10FEF00053F800281AD1FF2001040702594A3B4653
:10FF0000F8F794FF7D2080000090FCF736FD38461E
:10FF100054493A460B46F8F789FF0098FCF72DFD47
:10FF20000020014602460346F8F780FF4A48057064
:10FF3000F5834D4805704D48047003F0A7FE204638
:10FF40002946F8F743F9B08C002801D1F2F7C4FE36
:10FF5000474A2046214602F05BFBA00302F088FBE3
:10FF600005200021F8F732F92146424C20464C305A
:10FF7000414A0F46FBF758FF404800F079FAF3F783
:10FF8000EFF964214143E18202E0A0652772256315
:10FF900004F0D6FCF5F7E6FFF4F71EFDF3F740FB9F
:10FFA000FAF752F90025284604F0FCFF0198305A70
:10FFB000012801D1FAF7B4F9E07B002802D0E573FB
:10FFC000F8F7D8FE708FF0F707FC0146A06AF0F74B
:10FFD0009BFB002810D1F08F01280DD11E484078DE
:10FFE000002809D0A5621C484570A77041208000F8
:10FFF0002080F4F7EDFCA063A07800280BD0F4F784
:020000040001F9
:10000000E7FCA16B401A042805D31120002101F060
:100010002DFE00F035F8F5F7FDFD606DA16D88420D
:100020000CD1206B0028B3D1216DE06A411A1E2942
:10003000AED32065022020722763A9E7A065216B5B
:100040000129A2D1E16A216561639EE718000040A1
:100050003000014002C301021CA00102E438020288
:100060001D450100FFFFFF0018A0010219A00102B9
:100070000D25010058AB010201BD00005D04010027
:10008000B0B503F0DBF8EFF310800124C00719D1FD
:10009000EFF3108072B6092000252946F8F796F88C
:1000A0000F202946F8F792F80C202946F8F78EF829
:1000B00002F0FAFA204601F003FD284602F00EFB9A
:1000C00062B6B0BD092000252946F8F77FF80F2059
:1000D0002946F8F77BF80C202946F8F777F802F064
:1000E000E3FA204601F0ECFC284602F0F7FAB0BD36
:1000F000F0B581B0009003240127204639463A46E6
:10010000FEF76CFE2046FEF761FE04252846FEF74A
:100110005DFE2046FEF74AFE0A263046FCF742FC0A
:100120002846FEF743FE4E20F5F785F9F5F76AFB02
:100130000098C0B2F5F77FF9F5F764FB2046394621
:100140003A46FEF74BFE2046FEF740FE2846FEF7F5
:100150003DFE2046FEF72AFE3046FCF723FC2846EB
:10016000FEF724FE4F20F5F766F9F5F74BFB00206C
:10017000F4F7CAFF0090204639463A46FEF72EFEB5
:100180002846FEF713FE2046FEF710FE3046FCF729
:1001900009FC2846FEF71AFE2046FEF717FE3046F9
:1001A000FCF700FC009801B0F0BDF0B583B00291FF
:1001B000019003240127204639463A46FEF70EFEF9
:1001C0002046FEF703FE04263046FEF7FFFD2046DC
:1001D000FEF7ECFD0A252846FCF7E4FB3046FEF767
:1001E000E5FD4E20F5F727F9F5F70CFB0198C0B2B5
:1001F000F5F721F9F5F706FB0298F5F71CF9F5F785
:1002000001FB204639463A46FEF7E8FD3046FEF748
:10021000CDFD2046FEF7CAFD2846FCF7C3FB30465D
:10022000FEF7D4FD2046FEF7D1FD2846FCF7BAFBC9
:100230002846FCF7B7FB03B0F0BD000010B50D2059
:10024000FFF756FF04460E20FFF752FF2102081861
:10025000400802498860888010BDC046D0A80102CD
:10026000B0B5002424212046FFF79FFF2E48FCF75D
:1002700099FB0F202146FFF798FF10200521FFF77B
:1002800094FF11200421FFF790FF7F248321204653
:10029000FFF78BFF69212046FFF787FFBD2120462E
:1002A000FFF783FF21480078262807D18C242046B9
:1002B000FFF71EFF00212046FFF777FF27200024CD
:1002C0002146FFF772FF19200421FFF76EFF162069
:1002D0008721FFF76AFF5B48142101872820FFF779
:1002E00064FF0A20FCF75EFB11252846FFF700FF9C
:1002F00028462146FFF759FF0D48FCF753FB2F20F6
:100300000121FFF752FF30206221FFF74EFF31201D
:100310004621FFF74AFF32200146FFF746FF332010
:10032000A221FFF742FFB0BD204E000030A4010221
:10033000A0860100014800687047C0460C000040DC
:1003400081B080B581B0039303AB009302F0F2FF5C
:1003500001B080BC02BC01B008470000F0B581B01C
:10036000002630463146FDF76FFC0125AC023449CA
:10037000344F30463A462346FDF7EAFD3988324885
:1003800081425AD064217E5262217E5260217E5287
:1003900056217E527A212D4A7A5278212A227A5287
:1003A0007622E223BB5274222123BB52722279238C
:1003B000BB526E22264BBB526C220D23BB526A22CB
:1003C000D223BB526823FA5266222723BB5244220F
:1003D000BE52FD87BD877987022139874321F9867F
:1003E000BE83FD811B49B9817E810A2139811A4969
:1003F000B9803880FE837D20C000F88070203D5297
:1004000050203E523D85FD84BD847D84EFF31080F5
:1004100072B630463146FDF717FC00280CD12A038E
:1004200000263046064D2946FDF768FB054A304652
:1004300029462346FEF764F862B601B0F0BDC04617
:1004400000E0020402C30102AA5500004F2300008D
:10045000581B0000E1FF00003412000080B540206E
:100460000249F8F723F8FCF7B9F880BDBCA80102EF
:1004700070B50C4E306011240025204629462A46CE
:10048000FEF7ACFC032220462946FEF709FD326840
:1004900002212046FEF71AFC2046294601F0E6FB21
:1004A00070BDC046F4A801020020704710B50024BA
:1004B000002809D0002905D003464A000348194600
:1004C000EFF732FE204610BDE04310BD40A301020D
:1004D000014600200A2901DAC0437047014A118011
:1004E0007047C046C8A301020020704780B501884C
:1004F000064A11808178064A1170C178054A117048
:100500000079FBF705FE002080BDC046BEA60102B3
:10051000C0A60102383D02020448054901601521C8
:1005200009044160034981607047C0469C30004027
:100530004100080034000700074800684069704720
:10054000FD20400004490968085C704702480068C3
:100550006221405C7047C046D4A601020A491A22B3
:100560000A600A4948704878FF210902084A13685E
:100570008B43800380B2C0181060064820210160C0
:10058000054801600020704770200040C4A60102A9
:1005900004E400E080E200E000E100E0F0B5A9B092
:1005A00016460F460546C648002B024600D01A469E
:1005B0003921CC003D21C900511811918242189275
:1005C00006D001204202BE491898EFF7ADFD189AF7
:1005D0006120111913910E21119C0A91A170002F15
:1005E0000D9501D00A2100E00921592317938300BA
:1005F000E17078427841139908703078109010704B
:10060000F17AE17471785170B7789770F178D170A0
:100610003579157174795471B1799171F179D1711C
:10062000317A1172717A5172B17A91727E1EF0B282
:1006300000210328169106D870B28000A1A210589C
:100640006A00805A1690179882001898C018149063
:10065000F81E022804D3012E084604D89D4800E065
:100660009D48031918781290189DA81817902846CD
:10067000303015902C4656346D2080002950974A12
:10068000974B149E33627262B362F2623176F182EA
:10069000139B597009229A70281841608160C160CB
:1006A0000161109880008F490858F0F711F9012F67
:1006B00010900F9104D0022F05D17F217E2004E0FD
:1006C0007C217B2001E05B215A20159DA9842070AC
:1006D00003200C90A080012666701F200B90A8823A
:1006E0001820A8740A46083A179BDA76169B129AC5
:1006F000D2184A439100189A9163B702791E8B422F
:100700000E9109D97848608034206884774828821F
:1007100077481399088339E07F2B10DD802B18D0A0
:1007200031028B421BD071028B4227D16E4961800E
:1007300068846F4813990883CF20C00025E0202BE0
:1007400017D0402B1AD1684860800420688469481B
:100750001BE06548608006206884674815E06248B1
:10076000608010206884624813990883C520C00007
:100770000BE0624860800220688404E00420688402
:10078000812040006080FF2002302882104600F067
:1007900005FF1298102806D0402808D10820149987
:1007A000C876072000E004201799887002E01798A7
:1007B0000C9981701898169A8078C11E02290CD362
:1007C000022811D001280CD12672BA4200D9002685
:1007D0006672BA4213D8F44812E00D200002119953
:1007E00008800120800201E00C9800022081BA42BA
:1007F00001D8EE4800E0FA20179988600EE0FA2050
:1008000017998860139800780028119901D0E8485A
:100810004880E848139A1083E7480880A88CEFF7CF
:10082000F7FF0026E54B3246EFF78EFE02460B46F9
:10083000E3493046EFF7F0FEE24B3246EFF784FE35
:10084000F0F722F80746E080DF493046109A0F9B08
:10085000EFF7E2FEDD4B3246EFF776FEF0F714F8E5
:1008600078434042800B608116990E98814208D9E6
:100870000C20149FB872D648179988831220189AB2
:100880000EE0480A189A149F01D00D2003E0080AD0
:1008900000D1DBE20A98B872CE48179988831220FB
:1008A000F872D078052844D878440079400087440D
:1008B0000227402C3339C848B881C8482FE0C046C9
:1008C000D8A00102A86A0100A86A0100B86A010064
:1008D000B86A0100966701009D670100307500004D
:1008E000102700005868010005020000FF06000004
:1008F000040800000A04000036040000030200009F
:10090000B748F881B748388013E0B748F881B7484E
:100910003882B74838600CE0B448B881B5481799B8
:10092000C88306E0B4487882B448B8800B980006C3
:100930009064AE483881A748F880B14802882A847C
:10094000B0480078E874B0480078119F7875387D19
:10095000139000285ED0AD490A681023DA413A604E
:100960000A794B79CF8867801B029A186A840A7AC1
:100970004B7A8F7AC87A0D7B65701B029A183B04FC
:10098000D21800061018179FF860487B8A7BCB7B33
:100990003B77120210186081087C7877487C149AA3
:1009A0009072887CD072C87C159B1874087D58742E
:1009B000487D11909874C87D0A7E120212181A841C
:1009C000887DD87418464B7EC375887ECD7E2D02F7
:1009D0002818B880087F4D7F2D022818F880887F5E
:1009E000B877C87FF8772020085C149D28732120F1
:1009F000085C68732A20085C2A314D782D0228187B
:100A00008D782D044019C978090640181899886412
:100A1000119801E0EB7DA87C7D498B700A808000F5
:100A20001F38C882C883139800281FD02222774815
:100A3000825C034622335B781B029A180A842422C4
:100A4000825C034624335B781B029A18CA842622F0
:100A5000825C034626335B781B029A188A8328221D
:100A6000825C283040780002801888846948032519
:100A700069A2294602F0E4FF189F387814907B7829
:100A8000B8780F90FA78B8791390F8791190387A8D
:100A90001090787AB97A0890099100930F98019094
:100AA000029216980390129804901398059011984A
:100AB000069010980790FAA2F8482946149B02F075
:100AC000BFFF3D46643580212846EFF746FBB878E6
:100AD000C11E02290ED3012800D18FE1022800D0C7
:100AE000ABE11691149078787F225043F749401873
:100AF000F74907E01691149078785B225043F1494A
:100B00004018F14941182846EFF70EFB0D9D189843
:100B1000C6870E34324602E0641C0F2A0ADA2178B6
:100B20000029F9D0491C8907C90F91400E43C68797
:100B3000521CF1E71699022907D31499491E01297D
:100B400000D97DE14279D24901E04279CF49891843
:100B50000C78002D00D177E1C1790E91032900D9DD
:100B60004AE14279062A00D979E1492189004118F0
:100B70001191E43010900E98401E129019A800199F
:100B80000F9000231392149403E01898290600D1C3
:100B90005AE1052A5AD8C0467A441279520097443D
:100BA000455C728598ABC04688130000E2040000E3
:100BB0000C080000060A0000040F000000001041AD
:100BC00030C1BD41000070400000F0400000D04145
:100BD000120C0000140B000012120000140E000092
:100BE0000E160000130D0000121600000E12000079
:100BF000140B0E0A12080000101600000E0B000065
:100C0000BEA60102C0A60102383D0202443D020216
:100C10002CA7010201080000436173652070617216
:100C2000616D65746572733A200D0A001693DFB228
:100C3000002F04D019A801223946EFF787FA002CBB
:100C400000D191E019A8C019BB498AE0E8B2022896
:100C500067D00027022867D06BE00E98022872D177
:100C6000E8B2022800D103461693DFB2002F04D069
:100C700019A801223946EFF769FA002C74D019A897
:100C8000C019ACA16DE0E8B2022800D1042316938C
:100C9000DFB2002F04D019A801223946EFF756FA27
:100CA000002C61D019A8C0199FA15AE0E8B202280F
:100CB00000D106231693DFB2002F04D019A8012219
:100CC0003946EFF743FA002C4ED019A8C01992A16B
:100CD00047E0E8B2022800D10C231693DFB2002FC0
:100CE00004D019A801223946EFF730FA002C3BD086
:100CF00019A8C019874934E0E8B2811E4A424A4126
:100D00009700022804D119A801223946EFF71EFAEC
:100D1000002C16D019A8C0197CA12246EFF704FABE
:100D20000FE00627022804D119A801223946EFF75F
:100D30000DFA002C05D019A8C01980492246EFF7FA
:100D4000F3F9169710E01693DFB2002F04D019A81C
:100D500001223946EFF7FAF9002C05D019A8C0197D
:100D600073492246EFF7E0F93C193F2C05D80F985C
:100D7000C0194021091BEFF7F0F9129802281898C2
:100D800001D2002002E0C078411E88411599087008
:100D9000611E2E46E8B202280CD1179A517019A98B
:100DA000119AB8C9B8C2B8C9B8C2B8C9B8C2B8C926
:100DB000B8C20DE0179A117019A9109AB8C9B8C233
:100DC000B8C9B8C2B8C9B8C2B8C9B8C2C10709D190
:100DD00080073546149C139A169B00D4D5E6022052
:100DE0008543D2E6FE20354605401898149C139A98
:100DF000169B290628D0CCE637A231E01691149034
:100E000078780B994143334808181F386F21C9433C
:100E10000D9D7A180378D427D3554378D827D35516
:100E20008378DC27D355002900D170E6C378E0270A
:100E3000D3551031001D189FEBE70120404A10E008
:100E40000024002D00D087E629B0F0BD80290ED304
:100E50000F20B872104817998883102020E525A22A
:100E60000120014602F0ECFD189829B0F0BD1020D9
:100E7000402904D3B8720849179B998310E5B872CA
:100E800004481799888314200AE5C0469D6701002D
:100E900096670100150F0000140B00000108000008
:100EA00025642025642025642025642025642025D0
:100EB0006420256420256420256420256420256481
:100EC0000D0A0000B29001001DF7FFFFCA87010064
:100ED00089FBFFFFBA8F01007472785F6D6F6465E4
:100EE00020706172616D65746572206572726F72D7
:100EF0000D0A00004E73666420706172616D657446
:100F00006572206572726F720D0A0000FFFFFFFFAD
:100F100001FF0000586B0100FFFFFFFFFF0101FF11
:100F2000FF01FF01FFFF01FFFFFFFF01FFFF01FFC7
:100F30005C720100FFFF01FF786B0100C86A0100CD
:100F400039870100002800D101481D490860704719
:100F5000D8A0010210B5002801D0044601E01848CD
:100F60000468204600F006FC204600F021F80B48FB
:100F700041780B4A1A23136041704078FF2109021F
:100F8000084A13688B438007000CC018106006489D
:100F9000202101600548016010BDC046C4A60102C1
:100FA0007020004004E400E080E200E000E100E0A6
:100FB000F0B586B0002805D10148006802E0C046BF
:100FC000D4A601023121C900049141188A791F2356
:100FD0001A40CD79ED06AD0DAA180D7AED066D0C0F
:100FE00052194D7AED062D0B52198D7AED06ED0949
:100FF0005219CD7AED06AD0852194D7CED07521904
:10100000BD4C22600A7B1A404E7BF606B60DB21824
:101010008E7BF606760C9219CE7BF606360B92196D
:101020000E79F606F60992194E79F606B608921967
:1010300062604A6AB14D2A40A2608A6A2A40E26030
:101040002D22D20087183A7E1A4003937E7EF60640
:10105000B60DB218BE7EF606760C9219FE7EF60626
:10106000360B92193E7FF606F60992197E7FF60638
:10107000B60892190E7CF60792192261BA7F1A40BF
:101080000597FE7FF606B60DB218049BC35CDB061F
:101090005B0CD2184B78DB061B0BD2188B78DB0667
:1010A000DB09D218CB78DB069B08D2186261CA69CB
:1010B0002A40A2610A6A2A40E2618A7C01252A400C
:1010C000CB7CDB079B0F9A180B7DDB075B0FD218DD
:1010D0004B7D9B07DB0ED2188B7DDB079B0ED21856
:1010E000CB7D1B079B0D9A180B7E1B079B0CD21800
:1010F0004B7E5B06DB0A13438A7E520612091A43B3
:10110000CB7E5B075B0813432362CA6A62620A6B89
:10111000A2624A6BE2628A6B22633922D200835C4C
:101120001E462E4066635E425E41B304AE04744FB9
:101130003C68B443E3183B6083185A782A409C7893
:101140002407E40EA2188C8F6401A2186D4C144081
:10115000C98FC905490A0919DA78D207120A89180C
:101160001A791207120989185A79D207D2088918F0
:10117000FB4EB1639968F163997904952940DA7956
:10118000D207920F51181A7B5207D20E89185A7B38
:10119000D206920D51189A7B5207D20C8918DA7B2D
:1011A000D206920B89181A7CD206520A89185A7CE8
:1011B000520792090A43997CC906490851183164BB
:1011C000D97C039A11401A7DD206920D51185A7D8E
:1011D000D206520C89189A7DD206120B8918DA7D34
:1011E000D206D20989187164197E0F2421405A7ED3
:1011F000120151189A7E12038918DA7E1207120A18
:1012000051181A7F1207120989185A7F1207891874
:10121000B164997F01942140DA7F1207120E5118B0
:101220003D22D200835C5B075B0D591884186278FD
:101230001207520C8918A278D206120B8918E2788C
:10124000D206D2098918F164217907220A4061790E
:10125000C9008918A2795206920B5118E2799207B7
:10126000120B8918227AD2078A18BF490A60627A5B
:10127000A37A1B029A18E37A1B04D2184A60E28907
:10128000BA4B13400394228AD2049209D2188A607E
:1012900003463033598CB64A114002939A8CD205DA
:1012A000D20A51185622825C12068918B14D296063
:1012B000014656314A788C782402A2188C8864053D
:1012C0006409A218CC78240712196A60CA880C7ABB
:1012D000A407A40BA2184C7A6407E40A1219AA60A6
:1012E0004989E960492189004118FF226632821844
:1012F00000921035002207E000300040FFFFFF00A1
:1013000004040040FF3F000084186427E65D0327C3
:101310003E406523E35C9B071B0F9B196626A65D79
:10132000B607B60EF3186726A65DB601F318DBB252
:101330006826A65DB607B60DF3186926A65DB60742
:10134000360DF3186A26A65DB607B60CF3186B26A1
:10135000A65DB607360CF3186C26A65DB607B60B6D
:10136000F3186D26A65DB607360BF3186E26A65D3C
:10137000B607B60AF3186F26A65DB607360AF31845
:101380007026A65DB607B609F3187126A65DB607E6
:101390003609F3187226A65DB607B608F318732649
:1013A000A45DA407E31808C51032802AACD1019AC5
:1013B000D243704EB4180B783B404D78AD072D0FDB
:1013C000EB188D78AD07AD0EEB18CD78AD01EB18AD
:1013D000DBB20D79AD07AD0DEB184D79AD072D0DD5
:1013E000EB188D79AD07AD0CEB18CD79AD072D0C51
:1013F000EB180D7AAD07AD0BEB184D7AAD072D0B41
:10140000EB188D7AAD07AD0AEB18CD7AAD072D0A32
:10141000EB180D7BAD07AD09EB184D7BAD072D0922
:10142000EB188D7BAD07AD08EB18CD7BAD07EB1846
:10143000A3641031121DBDD1009B19785A78520750
:10144000520D51189A78D207120D8918B164059B74
:101450001968F164D97D5A6812025118316599688A
:10146000454A0A40998A490589187165D9683D4CF1
:101470002140B16519692140F165029E3178049DD2
:10148000294082785207120F5118C2799207920EA2
:101490008918427A9207920D5118827A9207120D9A
:1014A0008918C27AD207920C89189A7DD207520CF9
:1014B000891872789207D20B8918B2781207D20A6B
:1014C0008918F2781207D2098A182C490A60327CEE
:1014D000737C1B071B0D9A18B37C9B069B0BD218C1
:1014E000F37C1B079B0AD218337DDB065B09D218FD
:1014F000737DDB071B09D2184A60B27D2A40C38F77
:101500005B009A188A60826CCA60C26C22400A61D1
:10151000F27D7F231340328C5204520AD2184A6162
:1015200002698A614269CA6182690A62C2694A6261
:10153000026A8A62426ACA62826A0A63C26A4A6349
:10154000039A927CD201121D0A64027A3A40CA655B
:10155000808F074A10400866002006B0F0BDC046E4
:1015600000300040FFFFFF009C300040FF1F0000E4
:10157000FF03000000400040FFFF1F00002000406C
:1015800004480068806B80080349096849004018D6
:1015900009307047D4A601021004004010B52D2177
:1015A000C9004118027A032A04D10079002807D023
:1015B000082006E08378DA1E022A05D2032412E00E
:1015C000142088601C203DE0012B02D1C8228A60D3
:1015D00012E00479042C01D3462404E0032C01D149
:1015E000322400E014248C605B1E022B04D3022AF8
:1015F00010D24279154B01E04279154B9B181B78AC
:10160000402B04D0102B06D11423442405E02A23B8
:101610003E2402E04279342348244B800C80022A85
:1016200006D0062A08D0052A08D118224C2301E04A
:10163000142250230B8000E01C224A80C07804282A
:1016400003D1142048806420088010BD9D670100EC
:1016500096670100424800687047C04610B53F4A8F
:10166000107091703E49002813D050680861042022
:1016700048619078FF2212023A4B1C689443800321
:1016800080B20019186001204007054A1060364AF0
:10169000106000200860354901220A6010BDC04674
:1016A00080E200E03148002101602D4801680268B5
:1016B0008A420BD0016802688A4207D0016802683A
:1016C0008A4203D0016802688A42EFD17047C0465F
:1016D000F0B581B021480178214D002911D08178E1
:1016E000FF2212021F4B1C689443890389B2091917
:1016F0001960012149071C4A1160406828610420D3
:1017000068610127EFF310803840009002D1EFF3B9
:10171000108072B6154807602E682868B04208D15C
:101720002868B04205D12868B04202D12868B0428A
:10173000F3D0FDF77BFB0446EFF74EF80C49EEF7CC
:10174000D5FDEFF78CF83018B843286000980028D2
:1017500000D162B6204601B0F0BDC046C4A6010269
:10176000180400401CE400E000E100E070000040CC
:1017700080096E45F0B591B0002801D1C0480068DD
:101780008778F91E022913D3012F21D0022F3CD1D3
:101790001021CA4344782146193991423DD8009717
:1017A0000125B94A28462946234602F049F953E162
:1017B0000821CA43447821462139914218D800971C
:1017C0000125B14A28462946234602F039F943E16A
:1017D0000821CA43447821460939914234D80097F8
:1017E0000125A94A28462946234602F029F933E172
:1017F000032F3CD0042F43D1C3780125042B00D004
:101800002DE106462A02042343E00125A6A228462C
:1018100029463B4602F014F91EE1C3780125052B49
:101820000AD806462A02284698401B21084230D191
:101830000021052B08462ED002200090914A284610
:10184000294602F0FDF807E10646C3780021022B85
:101850001ED3032B1CD0042B08460A461BD001259F
:101860000095884A2846294602F0EAF8F4E0C37851
:101870000125032B00D0FAE006462A02032308E0E4
:10188000012583A2284629463B4602F0D9F8E3E029
:101890000A46012148020F91592189007518FD213E
:1018A000490071180291314662313F05D219641E18
:1018B0001F2727405C013C19144304433279520727
:1018C000D20C22432B789B065B0BD218B379DB0733
:1018D0001B0B13436D4D2B60F279032310931A40B9
:1018E000737A9B079B0E9A18B37A5B07DB0D9A18E5
:1018F000F37ADB079B0DD218337BDB075B0DD21825
:10190000737B1B075B0CD218AA603269EA607269AC
:101910002A61B2696A61F269AA61326AEA61726A2D
:101920002A62B26A6A620F980870F06AA8623F2061
:10193000C4432C353046E4300F903046E5300E90ED
:101940003046E6300D903046E7300C903046E830B7
:101950000B903046E9300A903046EA300990304624
:10196000EB3008903046EC3007903046ED30069072
:101970003046EE3005903046EF3004903046F0307F
:1019800003903746F1373046F230F3360F990A1993
:101990004021525C109B1A400E9B1B195B5C9B07FD
:1019A0001B0F9A180D9B1B195B5C9B079B0E9A18CB
:1019B0000C9B1B195B5C9B019A18D2B20B9B1B19E9
:1019C0005B5C9B079B0D9A180A9B1B195B5C9B0732
:1019D0001B0D9A18099B1B195B5C9B079B0C9A18A3
:1019E000089B1B195B5C9B071B0C9A18079B1B1918
:1019F0005B5C9B079B0B9A18069B1B195B5C9B0708
:101A00001B0B9A18059B1B195B5C9B079B0A9A187A
:101A1000049B1B195B5C9B071B0A9A18039B1B19F1
:101A20005B5C9B079B099A183B195B5C9B071B0936
:101A30009A1803195B5C9B079B089A183319595C29
:101A40008907891802C51034A0D1029800780421B2
:101A500001430E48C1630025284611B0F0BD0420A3
:101A60000090084A2846294601F0EAFFF4E70320DF
:101A70000090044A2846294601F0E2FFECE7C04600
:101A8000D4A601020E870100548701000010004017
:101A9000556E646566696E6564206D65616E205083
:101AA00052462025640D0A00496E76616C696420F7
:101AB0006D65616E205052462025640D0A000000BD
:101AC000B0B584B00446FAF75AFC1F48016800918B
:101AD0004168019181680291C0680390FFF7E2FDBF
:101AE00000F00EFE1948016804220A430260184DF6
:101AF0006868A021002C01D1884300E00843686099
:101B0000FF200230FAF79CFDFBF72AFC0020FFF7CC
:101B100021FAFDF79FFE6846FEF748F90D48016877
:101B2000C907FCD0012080022968814329600A4846
:101B3000FAF786FDFFF7CCFD4B49086000F0FEFD8B
:101B4000FAF722FC04B0B0BD80A0005010ED00E018
:101B50002C0000402C02004001020000704770473A
:101B600080B50E490E480246083A1268920000D429
:101B7000603142680A4342600A490A6808239A436E
:101B80000A60091F012252040A60032189040268C5
:101B90008A430260FAF724FC80BDC0462000008022
:101BA0002800004004020040B0B5032000072D4982
:101BB0000A6882430125680710180860002420463F
:101BC000FFF7CDFF2046FFF7C9FFEFF31080284055
:101BD00002D1EFF3108172B68021C943224A5368C3
:101BE0000B40536093680B409360D3680B40D36005
:101BF00013690B40136153690B405361002800D1F6
